:100000005446495300010000B44A0200A1C46405EB
:100010001017010316102017443159301017020031
:100020001610201744313030101701121610201707
:100030004431594C030000000000000000000000A3
:100040005446435300200000182202000000000024
:100050000080011001210000252100004122000044
:10006000292100002B2100002D2100003D2100004E
:100070003D2100003D2100003D2100002F21000016
:10008000312100003D21000033210000955A00007D
:100090007B5B0000372100003D210000114C001067
:1000A000372100008F3E0000953E00003D210000FA
:1000B0003D210000BF5600001D4E00009B3E000089
:1000C00045540000372100003D2100003D21000083
:1000D0000000000000000000000000000000000020
:1000E0000000000000000000000000000000000010
:1000F0000000000000000000000000000000000000
:1001000000000000000000000000000000000000EF
:1001100000000000000000000000000000000000DF
:1001200000000000000000000000000000000000CF
:1001300000000000000000000000000000000000BF
:1001400000000000000000000000000000000000AF
:1001500000F003F800F020F8FEE70D480168890878
:100160008900002001C101C101C101C17047000027
:10017000905A0010FEE7FEE7FEE7FEE7FEE7FEE727
:10018000FEE7FEE7FEE703480047FEE7FEE7000064
:10019000202100003D21000000F002F800F068F886
:1001A0000AA090E8000C82448344AAF10107DA45D2
:1001B00001D100F05DF8AFF2090EBAE80F0013F0BC
:1001C000010F18BFFB1A43F0010318470CCB0100C5
:1001D0004CCB01000A444FF0000C10F8013B13F027
:1001E000070408BF10F8014B1D1108BF10F8015B90
:1001F000641E05D010F8016B641E01F8016BF9D183
:1002000013F0080F1EBF10F8014BAD1C0C1B09D1D9
:100210006D1E58BF01F801CBFAD505E014F8016B4B
:1002200001F8016B6D1EF9D59142D6D370470000DD
:10023000103A24BF78C878C1FAD8520724BF30C812
:1002400030C144BF04680C607047000000230024E4
:1002500000250026103A28BF78C1FBD8520728BFD6
:1002600030C148BF0B6070471FB51FBD10B510BD32
:10027000DFF80CD0FFF7F8FF04F0B6FF1BF0A6FE86
:100280000080011003B4FFF7F1FF03BC1BF0A6FED2
:100290001EF0040F0CBFEFF30880EFF3098009F0A4
:1002A000F9BE000008B5002103200B460A46009164
:1002B0001AF09CFE08BD38B5F84D0024AC80EC80E7
:1002C0002C811AF070FE2861FF20A870F4482346A4
:1002D00022460460446004720120E8700320214635
:1002E00000941AF083FE012038BD38B5EB4D02288A
:1002F000AC7822460DD0052810D0A24208BF38BDE8
:10030000002003460246214600901AF06FFEAC70B2
:1003100038BD022914BF01240224EEE7022914BFCC
:1003200064246524E9E738B513460A464FF0010C0A
:1003300000240146604600941AF058FE38BDD748A4
:1003400000697047D549012008707047D34800788C
:100350007047D2490020087070472DE9F0410446EB
:100360000127002503F00700CC4E8846012804BF72
:100370000020308146D0022844D1308904280BD295
:10038000002818BFF06802D11AF051FEF06010F892
:10039000011B2170F0602EE0062808D21AF049FEF9
:1003A0003189C1F10501C900C840207023E0082847
:1003B00008D21AF042FE3189C1F10701C900C840D4
:1003C000207018E00C2808D21AF0EDFD3189C1F137
:1003D0000B01C900C84020700DE00E2808D21AF0A9
:1003E000E4FD3189C1F10D01C900C840207002E06F
:1003F000FF20207000273089401C80B230810E28F9
:1004000028BF012588F800503846BDE8F08130B497
:1004100003F007000024DFF884C201280BD06046F7
:10042000BCF808308088022B0CD2120242EA10205D
:10043000ACF804000CE0ACF80440ACF80640ACF8B2
:10044000084008E0DCF810501844284400F8022C5A
:10045000581CACF808000C7030BC00207047F0B499
:100460000746002003F007048C4D0646012C08BF08
:100470002E8117D0DFF824C2022CBCF806C003D0AE
:1004800013F0070F0AD00DE028892B690CEB00024E
:10049000401C9A5C3A702881012003E0120242EA73
:1004A0001C22EA800E70F0BC704738B503F00700DC
:1004B00000240D4601280AD1784821460B460481C4
:1004C0008480C48002200A4600941AF08FFD2C70AC
:1004D000002038BD2DE9F04182B00446DDE9080670
:1004E0001F460D464FF0010804EB061C002818BFFC
:1004F000022818D0002101287ED003281CBF02B09A
:10050000BDE8F0810F202070032060706180A18021
:10051000E18021816181A181A07B20F00100A07395
:1005200002B0BDE8F0810CF8106C0CF80F0CB5F8B7
:10053000B4002CF80E0CB5F8B6002CF80C0C95F89D
:1005400090002CF80A0C95F891002CF8080C95F8FE
:1005500092002CF8060CA88A2CF8040C92F848108B
:100560001CF8020C61F300000CF8020C95F8EE0088
:1005700001281CBF02B0BDE8F08104F03DFE052853
:100580001CBF02B0BDE8F08109F01BFE042804BFC7
:1005900002B0BDE8F081C0208DF8000095F8990008
:1005A0008DF8010095F8990004EB001030F80E0C5E
:1005B000000A8DF8020095F8990004EB001010F87D
:1005C0000E0C8DF8030095F8990004EB001030F83C
:1005D0000C0C000A8DF8040095F8990004EB00104B
:1005E00010F80C0C8DF805000CF08EFE9DF8001034
:1005F000090908FA01F100E00DE0084204BF02B069
:10060000BDE8F08101230622694607200CF0B2FE06
:1006100002B0BDE8F0810CF8106C0CF80F8C2CF8CF
:100620000E1C2CF80C1C2CF80A1C2CF8081C2CF89E
:10063000061C2CF8041C1CF8020C20F001000CF81D
:10064000020C04F0D9FD05281CBF02B0BDE8F08102
:1006500009F0B7FD042804BF02B0BDE8F081C12055
:100660008DF800008DF801607888000A8DF802008E
:10067000B8788DF80300B888000A8DF8040038793E
:100680008DF805000CF040FE9DF80010090908FAED
:1006900001F10842B6D102B0BDE8F081008000103F
:1006A000348300102B490020487070472948407857
:1006B00070472849012048707047274A11547047F5
:1006C000244800B5006983B04FF00001407810F075
:1006D000020F0AD000918DF804100123052269460B
:1006E00000200CF06EFE03B000BD10F0040F12D01D
:1006F00001208DF800008DF801108DF802108DF8A2
:1007000003108DF8041003460522694600200CF002
:1007100058FE03B000BD10F0C00F4FF001034FF0C2
:10072000000206D003B0012103205DF804EB0CF0B9
:10073000F1BD03B0632107205DF804EB0CF0EABDC6
:1007400070470449002818BF0120C870704701484D
:10075000C078704700800010348300107047FE4856
:10076000D0F8500300F00100704770B5FA4D040056
:100770000AD001F020FB38B9D5F8500310F0010F72
:100780001CBF0020A86005D10120A860002C08BF74
:10079000002000D00120286270BDEF48006A0028C8
:1007A00018BF01207047C00000F1804000F5A04054
:1007B00041637047C00000F1804000F5A040006B2D
:1007C00000F4807070471021C00000F1804000F5F7
:1007D000A04041637047E049D1F8402160F30D2209
:1007E000C1F840217047DC48D0F84001C0F3052033
:1007F000704700F00F0202EB42029201C0F30310B7
:1008000002EB801000F1804000F5A0400029D0F8F4
:10081000401114BF41F0010121F00101C0F8401165
:10082000704700F00F0101EB41018901C0F3031093
:1008300001EB801000F1804000F5A040D0F84001AD
:1008400000F001007047C44900230B6202680A608F
:1008500042684A6082688A60C268CA60426A0A6402
:10086000826A4A6402698A614269CA61826B0A6665
:10087000826C0A67C26C4A67026D8A67426DCA67FA
:10088000826DC1F88020C26DC1F88420026EC1F86B
:100890008820426EC1F88C20426FC1F8B020C26F30
:1008A000C1F8B820C26EC1F8A820D0F89422C1F8CF
:1008B0005023D0F89822C1F85423D0F89C22C1F8D4
:1008C0005823D0F8A022C1F85C23D0F88420C1F8C6
:1008D000F020D0F88820C1F8F420D0F88C20C1F89E
:1008E000F820D0F89020C1F8FC2021224A63CA6386
:1008F000C2694A62C26A8A64026BCA64026FC1F842
:10090000AC20026ACA62426B0A65C26B4A66026C1C
:100910008A66426CCA66826FC1F8B420D0F8802023
:10092000C1F8BC20D0F8A422C1F86023D0F8A822D6
:10093000C1F86423D0F8AC22C1F86823D0F8B02203
:10094000C1F86C23D0F8B422C1F87023D0F8B822D3
:10095000C1F87423D0F8BC22C1F87823D0F8C022A3
:10096000C1F87C23D0F88C2222F48032C1F84023D5
:10097000D0F89022C1F84C23D0F89420C1F800217F
:10098000D0F89820C1F80421D0F89C20C1F80821A3
:10099000D0F8A020C1F80C21D0F8A420C1F8102173
:1009A000D0F8A820C1F81421D0F8C820C1F834210B
:1009B000D0F8AC20C1F81821D0F8B020C1F81C2123
:1009C000D0F8B420C1F82021D0F8B820C1F82421F3
:1009D000D0F8BC20C1F82821D0F8C020C1F82C21C3
:1009E000D0F8C420C1F83021D0F8CC20C1F8402183
:1009F000D0F8D020C1F84421D0F8D820C1F84C213B
:100A0000D0F8E420C1F86021D0F8E820C1F86421D2
:100A1000D0F8EC20C1F86821D0F8F020C1F86C21A2
:100A2000D0F8D420C1F84821D0F8DC20C1F85021FA
:100A3000D0F8E020C1F85421D0F8F420C1F870219A
:100A4000D0F8F820C1F87421D0F8FC20C1F8782142
:100A5000D0F80021C1F87C21D0F83C21C1F8C02198
:100A6000D0F84021C1F8C421D0F84421C1F8C821F0
:100A7000D0F84821C1F8CC21D0F84C21C1F8D021C0
:100A8000D0F85021C1F8D421D0F87021C1F8F42158
:100A9000D0F85421C1F8D821D0F85821C1F8DC2170
:100AA000D0F85C21C1F8E021D0F86021C1F8E42140
:100AB000D0F86421C1F8E821D0F86821C1F8EC2110
:100AC000D0F86C21C1F8F021D0F87421C1F80022CF
:100AD000D0F87821C1F80422D0F88021C1F80C2286
:100AE000D0F88C21C1F82022D0F89021C1F824221E
:100AF000D0F89421C1F82822D0F89821C1F82C22EE
:100B0000D0F8AC21C1F84022D0F8B021C1F844227D
:100B1000D0F8B821C1F84C22D0F8C421C1F8602225
:100B2000D0F8C821C1F86422D0F8CC21C1F86822DD
:100B3000D0F8D021C1F86C22D0F87C21C1F808226D
:100B4000D0F88421C1F81022D0F88821C1F81422ED
:100B5000D0F89C2102E0000000500040C1F8302293
:100B6000D0F8A021C1F83422D0F8A421C1F838224D
:100B7000D0F8A821C1F83C22D0F8B421C1F848220D
:100B8000D0F8BC21C1F85022D0F8C021C1F85422BD
:100B9000D0F8D421C1F87022D0F8D821C1F874223D
:100BA000D0F8DC21C1F87822D0F8E021C1F87C220D
:100BB000D0F8E421C1F88022D0F8E821C1F88422DD
:100BC000D0F8EC21C1F88822D0F8F021C1F88C22AD
:100BD000D0F8F421C1F89022D0F8F821C1F894227D
:100BE000D0F81822C1F8B422D0F8FC21C1F898221C
:100BF000D0F80022C1F89C22D0F80422C1F8A0222B
:100C0000D0F80822C1F8A422D0F80C22C1F8A822FA
:100C1000D0F81022C1F8AC22D0F81422C1F8B022CA
:100C2000D0F81C22C1F8C022D0F82022C1F8C4227A
:100C3000D0F82822C1F8CC22D0F83422C1F8E02222
:100C4000D0F83822C1F8E422D0F83C22C1F8E822DA
:100C5000D0F84022C1F8EC22D0F85422C1F8002389
:100C6000D0F85822C1F80423D0F86022C1F80C2330
:100C7000D0F86C22C1F82023D0F87022C1F82423C8
:100C8000D0F87422C1F82823D0F87822C1F82C2398
:100C9000D0F82422C1F8C822D0F82C22C1F8D022E2
:100CA000D0F83022C1F8D422D0F84422C1F8F02282
:100CB000D0F84822C1F8F422D0F84C22C1F8F8222A
:100CC000D0F85022C1F8FC22D0F85C22C1F80823E9
:100CD000D0F86422C1F81023D0F86822C1F8142398
:100CE000D0F87C22C1F83023D0F88022C1F8342318
:100CF000D0F88422C1F83823D0F88822C1F83C23E8
:100D0000FE4A126832F0FF0C05D1D1F890C062F3B0
:100D1000030CC1F890C0FA4A5370D0F8943213F023
:100D2000010F1CBF01235370D1F8503323F001038E
:100D3000C1F85033D0F8A43213F0010F03D0537828
:100D400043F002035370D1F8603323F00103C1F87C
:100D50006033D0F8B43213F0010F03D0537843F06E
:100D600004035370D1F8703323F00103C1F87033DA
:100D7000D0F8AC0210F0010F03D0507840F008001A
:100D80005070D1F8680320F00100C1F86803704783
:100D9000DB4800787047DA4880787047D849C870D7
:100DA0007047D748C0787047D649D1F8542360F3CC
:100DB0000902C1F854237047D248D0F85403C0F355
:100DC00009007047CE4948607047CE48C0687047F8
:100DD0002DE9F047DFF82893054615F4003F99F810
:100DE000010099F8031000EA010418BF24F001047F
:100DF00015F4802F18BF24F0020415F4002F18BF3B
:100E000024F00404DFF8FC82D8F8400320F480309A
:100E1000C8F8400314F0070F59D0D9F80460D8F887
:100E20004803002740F00100C8F84803D8F84803F9
:100E300020F00100C8F84803D8F8400340F480309F
:100E4000C8F840034FF0630A0DE002F0B4FE5046CC
:100E5000D8F8481311F0010F01D0012703E0011E5B
:100E6000A0F10100F4DC301EA6F1010601DD002F27
:100E7000EBD067B3D8F8500314F0010F0CBF20F08B
:100E8000010040F00100C8F85003D8F8600314F0E6
:100E9000020F14BF40F0010020F00100C8F8600309
:100EA000D8F8700314F0040F14BF40F0010020F0D4
:100EB0000100C8F8700389F80240012089F8000099
:100EC000D8F8400340F48030C8F8400333E0D8F845
:100ED000500320F00100C8F85003D8F8600320F058
:100EE0000100C8F86003D8F8700320F00100C8F8CA
:100EF0007003002089F80200ACB1022089F80000DC
:100F0000D8F8400340F48030C8F84003D8F84803CC
:100F100040F00100C8F84803D8F8480320F0010069
:100F2000C8F8480307E0D8F8401321F48031C8F826
:100F3000401389F80000D8F8400115F0020F20F0A6
:100F40000D0018BF40F0010015F0080F18BF40F069
:100F5000040015F0040F18BF40F00800C8F8400165
:100F600015F0010F21D001F05AF9044601F05AF9A9
:100F70000146D8F80C0000280EBF2046084621463E
:100F80000028D8F8000214BF40F0010020F0010052
:100F9000C8F80002D8F84002002914BF40F0010050
:100FA00020F00100C8F840020BE0D8F8000220F061
:100FB0000100C8F80002D8F8400220F00100C8F88B
:100FC000400215F0200F18BF002417D0204601F072
:100FD00030F900284FEA841000F1804000F5A0406D
:100FE000D0F8C01214BF41F0010121F00101C0F896
:100FF000C012641C022CE9D3BDE8F087D8F8C00207
:1010000020F00100C8F8C002D8F8000320F0010069
:10101000C8F80003BDE8F0872DE9F003024602F0AE
:101020000F01002001EB41018C01C2F3031104EB1D
:10103000811101F1804101F5A041D1F8401111F079
:10104000010F11D142F01001C1F3031104EB811122
:1010500001F1804101F5A041D1F8401111F0010FDB
:1010600004BFBDE8F003704702EB42018E0106F1B8
:10107000804101F5A041D1F82431C3F30809214B87
:10108000DB69D1F8001103F008071FFA81F800218D
:1010900042EA0113C3F3031304EB831303F1804308
:1010A00003F5A043D3F8403113F0010F18D006EB3D
:1010B000811303F1804303F5A043D3F844C1CCF37B
:1010C000080517F1000C1CBFD3F844C1CCF3023C57
:1010D000D3F8403105FA0CFCC3F3054360441844CF
:1010E000491C0229D4D309EBC90100FB08F001EB2C
:1010F0000911BDE8F00300EB41007047E0FE03007A
:10110000148000100050004010B50120FFF784FF4C
:1011100004460220FFF780FF044400F03CFC20441A
:101120004FF47A7148434CF25031B0FBF1F010BDEE
:101130002DE9F041FA4E0546306810F01F0408BF53
:1011400001240120FFF768FF07460220FFF764FF34
:10115000074400F020FC3918F24F002D18BF002979
:101160004ED0D6F85003002210F0010F36D0782070
:10117000B0EB151F08D9D6F85C0320F00F0040F043
:101180000100C6F85C032EE0D6F85403E64BC0F32A
:10119000090060436FF0180C00FB0CF003EB4003F8
:1011A000E248A0FB05C04FEA502CB3FBF1F0102839
:1011B00028BF0F20844598BF6046002808BF012043
:1011C00005D0012884BF00FB1132B2FBF0F2D6F843
:1011D0005C3360F30303C6F85C3304E0B7FBF5F05F
:1011E000884288BF421A32206043B2FBF0F0B0F56B
:1011F000005F28BF41F6FF70726860F30C027260F6
:101200007068C0F30C00604300EBC00202EB0010FA
:1012100001EB4000B7FBF0F0BDE8F081C048D0F82A
:10122000501311F0010F07D0D0F85C0300F00F004D
:10123000C0EB00108001704770B50168406801F094
:101240001F05C0F30C060120FFF7E6FE044602204E
:10125000FFF7E2FE044400F09EFB06FB05F132229C
:1012600001FB02410844AF49B1FBF0F070BDAC484E
:10127000D0F85C0300F00F007047A9494A684B683A
:10128000C2F30C0260F30C034B6010467047A44895
:101290004068C0F30C00704700EB4000800100F193
:1012A000804000F5A040D0F80001A14980B2B1FB18
:1012B000F0F0401C4008704730B49D4B31B1B3FB97
:1012C000F1F1491C4A08B2F5804F01D343F6FF7291
:1012D000B3FBF2F1491C4D0800EB400189015308B2
:1012E00001F1804101F5A041002807BF981FA3F13B
:1012F0000C0CD1F8040180B218BFA2F1060C2CF03E
:10130000010CD1F8004162F30F04C1F80041D1F89B
:10131000002163F31F42C1F80021D1F8042160F3DA
:101320000F02C1F80421D1F818016CF30F00C1F8C5
:101330001801284630BC704700EB4000800100F1E6
:10134000804000F5A040D0F80001000C704700EB91
:101350004002920102F1804202F5A042D2F800312F
:1013600061F31F43C2F80031002818BF70478A1F7D
:10137000901F20F001016A48D0F8043162F30F0396
:10138000C0F80431D0F8182161F30F02C0F8182119
:10139000704700F00F0101EB41018901C0F3031018
:1013A00001EB801000F1804000F5A040D0F844012E
:1013B000C0F30800704700F00F0202EB42029201F6
:1013C000C0F303105B4B02EB801000F1804000F58E
:1013D000A0409B58D0F84421CB1A61F30802C0F812
:1013E0004421D0F844119B1E63F31841C0F8441106
:1013F00070474B49C969504A11F0100F00F00F01B6
:1014000001EB41014FEA8111C0F3031001EB8010A1
:1014100000F1804000F5A0405258D0F84401D2B20B
:10142000C0F3080008BF0022801A0004000C08BFA7
:101430000120704703091B0203EB810101F14051B8
:1014400001F540410007C00E0B6802FA00F0184396
:10145000086070470209120202EB810101F140515C
:1014600001F5404100070968C00E21FA00F000F0C4
:101470000300704700F00F0303EB43039B01C0F32D
:10148000031003EB801000EB810000F1804000F5B9
:10149000A040C0F85021704700F00F0202EB42025A
:1014A0009201C0F3031002EB801000EB810000F109
:1014B000804000F5A040D0F850017047184A002144
:1014C000D26912F0080F10D000F00F0101EB4101BA
:1014D0008901C0F3031001EB801000F1804000F59A
:1014E000A040D0F84401C0F30231084670470C4ACE
:1014F000D36943F00803D36100F00F0202EB42020C
:101500009201C0F3031002EB801000F1804000F55F
:10151000A040D0F8442161F30E32C0F84421704756
:10152000005000400008AF2FD8810C0089888888BF
:10153000A08601001C51004028510040F84A0021BB
:10154000D26912F0080F10D000F00F0101EB410139
:101550008901C0F3031001EB801000F1804000F519
:10156000A040D0F84801C0F302410846704700F09F
:101570000F0202EB42029201C0F3031002EB801053
:1015800000F1804000F5A040D0F8482161F31242FC
:10159000C0F848217047042988BF704710B4002361
:1015A000DF4CE26912F0080F00F00F0202EB42027A
:1015B0004FEA8212C0F3031002EB801000EB04022A
:1015C0001CBFD2F84401C0F302330020D4F81CC081
:1015D0001CF0080F1CBFD2F84801C0F30240C91A22
:1015E0000844042803DD081A011D042003E0002834
:1015F000BCBF014400201944E36943F00803E361E0
:10160000D2F8443161F30E33C2F84431D2F84811B4
:1016100060F31241C2F8481110BC7047C04900285D
:10162000886914BF40F0080020F008008861704706
:10163000BB488069C0F3C000704700F00F0202EBA6
:1016400042029201C0F3031002EB801000F18040CF
:1016500000F5A040C0F84C11704700F00F0101EBFD
:1016600041018901C0F3031001EB801000F18040BB
:1016700000F5A040D0F84C017047A94AD2F85C139D
:10168000022903D110F0010F18BF7047D2F84001B2
:1016900010F0010F0BD0D2F84C01D2F84411002801
:1016A000C1F302311EBF0029C043C2F84C01012121
:1016B00001EB410100204FEA811C0CEB801101F18C
:1016C000804101F5A041D1F8402112F0010F0BD06B
:1016D000D1F84C21D1F84431002AC3F302331EBFA4
:1016E000002BD243C1F84C21401C0228E5D370479F
:1016F0008B4A0021D26912F0080F10D000F00F01C0
:1017000001EB41018901C0F3031001EB801000F1EE
:10171000804000F5A040D0F84801C0F300510846D1
:1017200070470120704710B4022ADDF804C026BFBC
:10173000921E52080022022B26BF9B1E5B0800232C
:10174000784CA4FB0C4C4FEA1C1400F00F0C0CEB73
:101750004C0C4FEA8C1CC0F303100CEB801000F112
:10176000804000F5A040D0F864C161F31B6C62F3C7
:10177000144C63F30C2C64F3070CC0F864C110BC68
:10178000704770B400F00F0404EB4404A401C0F3EC
:10179000031004EB801000F1804000F5A040DDF85C
:1017A0000CC0D0F864010029C0F30366C0F3044400
:1017B000C0F30425C0B218BF0E6012B16100891CCD
:1017C000116013B16900891C1960BCF1000F04BFDE
:1017D00070BC704700EB80008000CCF8000070BC4B
:1017E000704770B491B000224FF480456C10EC4605
:1017F00001E0082A05D2531C03EB8303B5FBF3F386
:1018000004E0D31F03EB8303B4FBF3F35B1A48BF7D
:101810005B424CF82230521C102AEAD30026009B6F
:1018200001215CF821209A42BCBF13460E46491C98
:101830001029F6D300F00F0101EB41018901C0F33B
:10184000031001EB801000F1804101F5A041D1F8B7
:101850006801D1F8682100F00F0066F30302C1F8B7
:101860006821082807D2401C00EB8000B5FBF0F08F
:1018700011B070BC7047C01F00EB8000B4FBF0F0EB
:1018800011B070BC704700F00F0101EB41018901FC
:10189000C0F3031001EB801000F1804000F5A04080
:1018A000D0F8680100F00F00082834BF401CC01FAA
:1018B00000EB800034BF4FF480414FF40051B1FB86
:1018C000F0F0704710F00F0F08BF704700F00F00E6
:1018D00000EB4000800100F1804000F5A0400029AD
:1018E000D0F82C110CBF21F4803141F48031C0F8C4
:1018F0002C117047002110F00F0F0ED000F00F00D8
:1019000000EB4000800100F1804000F5A040D0F8DD
:101910002C0110F4803F18BF0121084670470000D9
:1019200000500040CDCCCCCC00F00F0000EB4000CC
:10193000800100F1804202F5A042D2F83401C2F8E1
:10194000341170472F4B58679967DA6770472D49F4
:101950000028D1F8AC0014BF40F0020020F00200D3
:10196000C1F8AC00704727490028D1F8AC0014BF7B
:1019700040F0010020F00100C1F8AC0070472148A0
:10198000D0F8E00070471F49C1F8E40070471D48D7
:10199000D0F89800704770B41A4E0020D6F8401165
:1019A00011F0010F04BF70BC704711F0040FD6F89E
:1019B000242101F00805D6F800C1C2F308021FFA7D
:1019C0008CF4D6F844C1CCF3080C18BFC1F307401F
:1019D000F369C1F3052113F008031CBFD6F84431A5
:1019E000C3F30233002D18BF491C0CFA03F301FBAB
:1019F0000300604302EBC20170BC01EB021100EB7B
:101A00004100704700500040FEF7C7BE10B5FEF71A
:101A1000C4FE012818BF10BD0020FEF7A6FE21213C
:101A20000020FEF7C0FE2121BDE810400120FEF796
:101A3000BABE10B5FEF792FEFEF7AFFE01280AD13E
:101A40000020FEF792FE21210020FEF7ACFE2121AE
:101A50000120FEF7A8FE0121052001F0EEFB012187
:101A6000052001F0EAFBFF490020087110BD10B508
:101A70004FF4066001F037FCBDE810404FF40660FB
:101A800001F022BCF74A0146107B002818BF012054
:101A9000002918BF012111737047F24A516A506240
:101AA00008467047EF490020C87288704870704738
:101AB000EC490020C87288704870704770B5000704
:101AC000C00E0D46801E00EB400101EB0014E648FD
:101AD0004FF4987200EBC40029461AF085FAE348E7
:101AE00005F5987100EBC400BDE870404FF49872A2
:101AF0001AF07ABA2DE9F0410546FEF774FEDC4F84
:101B0000DFF870830446EDB14C2004FB00F216466A
:101B1000294638461AF068FA324605F50061404613
:101B20001AF062FA04EB440000EB041407EB8400A3
:101B30004C211AF05EFA08EB8400BDE8F0414C211C
:101B40001AF057BA4C21401C41430C4638461AF053
:101B500050FA21464046BDE8F0411AF04ABA10B5A5
:101B6000C04CE061FFF734F9FFF712F9A1696FF398
:101B70000F01A161A269C1B242EA0121A16102285B
:101B800018BF10BDA06940F00100A06110BDBA48A7
:101B90008168BA4A114381600168521C1143016097
:101BA00000F061BE2DE9F041B34A0C46054693684A
:101BB000B248184390601068B1490843106000F0C3
:101BC00052FE0026002C76D00020FEF7CEFD2068C5
:101BD00020B1FEF738FE0020FEF7C7FD2846FFF7CC
:101BE000BEFF0020FEF71DFE70B36068FFF782FFA6
:101BF000A448E16819B102151AF0F6F91DE0A24DEA
:101C00004FF440711AF0F5F90020012329560029FC
:101C100010DB0A09120202EB800202F1405202F5C7
:101C200040420907C90ED2F800C003FA01F14CEA9C
:101C300001011160401C2628E8D39448616959B11C
:101C40004FF400721AF0D0F90120FEF7EAFDDFF838
:101C50001882864F48B904E04FF400711AF0C9F9B0
:101C6000F2E71120FEF7DDFD70B1A56865B14046D1
:101C70004FF4987229461AF0B7F938464FF4987223
:101C800005F598711AF0B0F90220FEF7CAFD18B9EF
:101C90001220FEF7C6FD70B1246964B17C484FF490
:101CA000987221461AF0A0F97A484FF4987204F518
:101CB00098711AF099F96B48C67286704670466240
:101CC000017B002101734FF4066001F00CFBBDE8BD
:101CD000F0414FF4066001F0F7BA10B50020FEF7AE
:101CE00044FD00F0ADFD5F48C078002808BF10BD7E
:101CF0006148016821F0030141F00D7141F080510C
:101D00000160816821F0020141F00D7141F08051C4
:101D1000816010BD4FF4066001F0DBBA10B54FF4DE
:101D2000066001F0D6FAFEF738FD01280AD100203E
:101D3000FEF71BFD21210020FEF735FD21210120AA
:101D4000FEF731FD5448D0F8401321F48031C0F83B
:101D500040130020FEF709FD00F072FD4148C078F5
:101D6000002808BF10BD4448016821F0030141F07C
:101D70000D7141F080510160816821F0020141F054
:101D80000D7141F08051816010BD10B501F0A6FACF
:101D900010F0600018BF012010BD3248C0697047C4
:101DA00030488069704772B62E498A6922EA00007D
:101DB000886162B670472B480078002818BF012060
:101DC000704770B5FEF7E9FC002818BF70BD00240D
:101DD000244DEC72AC706C7021212046FEF7E3FCC0
:101DE00021210120FEF7DFFC2C70BDE870400120AE
:101DF000FEF7BBBC70B50446FEF7CFFC002818BF49
:101E000070BD0021174DE972A97069702121002071
:101E1000FEF7C9FC21210120FEF7C5FC022C3CBFC6
:101E20000120FEF7D0FC012028702C62BDE8704034
:101E3000FEF79BBC10B5FEF7B0FC002818BF10BD24
:101E40000020084CE072A07060702121FEF7ABFC0E
:101E500021210120FEF7A7FC0120FEF7B4FC0120A0
:101E600020701BE01C800010189D003018BD003051
:101E70000080003000A000300080004002003412DA
:101E80000300341200C000304083001000D0003046
:101E9000489E003048BE0030005000402062BDE83F
:101EA0001040FEF762BC0020FEF75FBCFE49002038
:101EB000887048700120FEF758BCFB498862704763
:101EC000F948806A7047002818BF0120F649C862A7
:101ED0007047F548C06A002818BF012070470020ED
:101EE00000F0CEBB012000F0CBBB10B5FFF747FDE3
:101EF0000446FFF748FDED48044208BF10BDEA481C
:101F0000816941F0040181610E2101EAD43104F0BC
:101F100001020A43816962F31F418161E44801685B
:101F200041F02001016010BD002818BF0120DE49EA
:101F3000C8707047DF487047DF487047DA48006B69
:101F40007047D948406B7047D748806B70472DE980
:101F5000F04FD84F4FF0000C8DB007F14C04E6461F
:101F60004FF0FF3807F80C8004F80CE00CF1010C7E
:101F7000BCF1260FF6DB4FF0000C002807DD12F84D
:101F80000C5007F80C500CF1010C6045F7DC0022F6
:101F90000126CDF804E06D46CDF800E0002816DDFE
:101FA00017F902C0BCF1000F0EDBBCF1260F0BD2FB
:101FB0004FEA5C190CF01F0C55F829A006FA0CFC2E
:101FC0004AEA0C0C45F829C0521C8242E8DB002288
:101FD00094460DF108094FEA521A02F01F0B55F80A
:101FE0002AA006FA0BFB1AEA0B0F1ABF09F802C067
:101FF0000CF1010C09F80280521C262AEBDB0022AE
:10200000002810DD17F902C0BCF1000F08DBBCF19D
:10201000260F3ABF19F80CC004F802C004F8028079
:10202000521C8242EEDBDFF880A200220028CAF8B0
:1020300030E009DD14F902C0944502D0CAF83040FE
:1020400002E0521C8242F5DBDFF870B20020ABF1F7
:10205000720404F14C0704F8008007F800E00BF864
:1020600000E0401C2628F6DB0020002904DD1A5C75
:102070002254401C8142FADC0020CDF804E0CDF867
:1020800000E0002912DD2256002A0CDB262A0AD2A3
:10209000530902F01F0255F823C006FA02F24CEA77
:1020A000020245F82320401C8842ECDB0020024657
:1020B000430900F01F0C55F8233006FA0CFC13EA14
:1020C0000C0F1ABF09F80020521C09F80080401CB0
:1020D0002628EDDB002000290BDD2256002A05DB37
:1020E000262A3CBF19F802200BF80020401C884229
:1020F000F3DB0020CAF838E0002909DD1BF90020D5
:10210000824202D0CAF838B002E0401C8842F5DBB7
:1021100011F0010F18BF252015D0420900F01F0350
:1021200055F8222006FA03F31A420AD1420900F0B8
:102130001F0055F8223006FA00F0184345F8220037
:1021400001E0401EE9D500200246430900F01F0CC3
:1021500055F8233006FA0CFC13EA0C0F1ABF09F8E5
:102160000020521C09F80080401C2628EDDB0020CE
:1021700000290ADD2256002A04DB262A3CBF19F872
:1021800002203A54401C8842F4DB0020CAF834E0B4
:102190000029DCBF0DB0BDE8F08F3A56824204D072
:1021A000CAF834700DB0BDE8F08F401C8842F4DBF3
:1021B0000DB0BDE8F08F40F2DB114843404901EB20
:1021C000800070473F49C0EB001001EBC000704732
:1021D000DFF8D4C0012B8CF805008CF8061003D969
:1021E000401C20F0010011468CF807008CF8081004
:1021F00000FB01F24FF6FF7101EA4202ACF8122037
:1022000001EA4000ACF8140070472748007A704794
:102210002548C0797047244A50729172704722480D
:10222000807A70472048407A7047274A1070517072
:1022300070472549085C70472DE9F047DFF8689042
:10224000044699F80C00002804BF99F8010019F021
:10225000D5FE99F80B00002808BFBDE8F0874FF0C5
:102260000008D9F81C0047464646454610F0020FC4
:102270001CBFDFF84C8010F0040F05D0B9F8121025
:102280000F4A21F001018F1810F0010F18BF0D4EF9
:1022900010F0200F18BF0D4DD9F828002060FEF770
:1022A0007AFD10F0010F13E01C8000100100070000
:1022B0005C8000104083001066830010D8830010FB
:1022C000008400106C8B0010298000105C8C0010C2
:1022D00006D0FEF7CCFF022828BF99F8020000D2F2
:1022E0000020E760C4E90108C4E904650120BDE8F5
:1022F000F087FF490020C872704770B50546FEF7A9
:1023000072FA4C2100FB01F21446FA49284619F0F2
:102310006BFE224605F50060BDE87040F64919F0F5
:1023200063BEF0B583B0FEF75EFA044600210846AE
:10233000FFF7B2F8009001210020FFF7ADF800226E
:102340000190002C2AD96E464FF0010C4FF6F07523
:1023500002EB4200002100EB02104B0901F01F07C5
:1023600056F823300CFA07F73B4211D0CB079B0CF1
:1023700003EB80034F0803EB870303F1405303F59E
:1023800000431B889BB2AB4202D903B00020F0BDD2
:10239000491C2629E1D3521CA242D9D303B0012003
:1023A000F0BD70B50D460107C80E811E01EB41005E
:1023B00000EB0114D1484FF4987200EBC401284699
:1023C00019F012FECE484FF4987200EBC40105F5E7
:1023D0009870BDE8704019F007BE2DE9F04F00F08D
:1023E0000F07780083B0A0F1020B0025E9464FF0FB
:1023F00001084FF6F07647EA051A5046FEF711FA43
:10240000002843D05046FFF759F808FA00F4022C90
:1024100088BF022400215046FFF73EF800900121BA
:102420005046FFF739F800210190002C2ED90BEB14
:102430000500982200FB02FA01EB4102002002EBAA
:10244000011C420900F01F0359F8222008FA03F387
:102450001A4215D000F001020AEB423202EB8C0264
:10246000430802EB830202F1405202F51042B2F837
:10247000182D92B2B24203D903B00020BDE8F08F0C
:10248000401C2628DDD3491CA142D5D36D1C022D4A
:10249000B1D303B00120BDE8F08F2DE9F041002653
:1024A000934D00280C4640D000F00F01C0F30310FC
:1024B00001290EBF00210229BDE8F081022828BFB2
:1024C000BDE8F0810F18FEF768F95FEA00081CBF4D
:1024D0000020FEF74AF90023982007FB00FC03EBDD
:1024E0004300002200EB031702F001000CEB403028
:1024F000510800EB870000EB810000F1405000F52F
:102500001040521CC0F8184D262AEDD35B1C022B3C
:10251000E5D3B8F1000F08BFBDE8F081AE706E7072
:10252000BDE8F0410120FEF720B9FEF736F95FEA79
:1025300000081CBF0020FEF718F9002303EB43003E
:10254000002200EB031CD007800C510800EB8C002C
:1025500000EB810707F1405707F50047521C3C602C
:10256000262AF0D35B1C312BE8D3B8F1000FD5D16C
:10257000BDE8F08110B5FEF73CFF5D49088210BD53
:102580005B4AC1B200F47F43128A914288BF114670
:102590004FF0640C01FB0CF1B1FBF2F11A0A02FBE3
:1025A0000C1110F4803F12BF08B2484200B27047CD
:1025B00010B54FF44071534C534819F01AFD0020E8
:1025C00001232156002910DB0A09120202EB8002C6
:1025D00002F1405202F540420907C90ED2F800C08C
:1025E00003FA01F14CEA01011160401C2628E8D3EE
:1025F00010BD10B5434C4FF44071434819F0F9FC3D
:10260000002001232156002910DB0A09120202EBE7
:10261000800202F1405202F540420907C90ED2F889
:1026200000C003FA01F14CEA01011160401C2628A8
:10263000E8D341F678712F4819F0DBFCBDE8104073
:1026400041F678712C4819F0D4BC294810B5808B1C
:1026500000F48170FFF783FA4FF440712A4819F0B3
:10266000C8FC41F61851234819F0C3FC41F6185133
:10267000214819F0BEFCBDE810400020FEF7FDBD6A
:1026800070B51B4C0546A06A401CA062E16A002997
:1026900018BFFEF7F2FF207850B1206A10B1206A0F
:1026A000401E2062206A002804BF0020FEF75DF86B
:1026B00020212846FEF777F8616A00291CBF2846CA
:1026C0008847FEF765FB022826D11048D0F848134A
:1026D00011F0010F20D0D0F8481341F00101C0F8EB
:1026E0004813D0F8481321F00101C0F848130FE057
:1026F0001C8000100080003000A00030189D0030C9
:1027000018BD00304083001000C000300050004071
:10271000A06940F00200A0610248016841F0200178
:10272000016070BD5C800010F0B40024634E012392
:1027300082B0002808BF33701CD00128347018BF45
:10274000747017D05E4D28685E4908432860317860
:102750005D4A002914BF49F608305C48D06014BFB8
:102760005B484FF0BB7090605A48006830F0FF0C37
:1027700008D101E07370E5E7D2F80CC060F3030CF8
:10278000C2F80CC040F2E24CA9B1906840F01800C9
:1027900090600120009004E00198471E0197FBD251
:1027A0000098471E009728BFCDF804C0F4D2906867
:1027B00040F4805090600120009004E00198471E92
:1027C0000197FBD20098471E009728BFCDF804C0A0
:1027D000F4D2707818B1D06840F03000D060D2F8F0
:1027E000B00040F00100C2F8B0000120009004E009
:1027F0000198461E0196FBD20098461E009628BFFF
:10280000CDF804C0F4D2D3674FF4E0601061C2F891
:102810008840002918BFC2F89430D06820F03000FA
:10282000D060906820F480509060286820F0040008
:1028300040F00D7040F08050286002B0F0BC70474E
:102840002148C16821F03001C160816821F48051C4
:1028500081601B48016821F0040141F00D7141F0D5
:1028600080510160704716480268164911430160A3
:10287000124915480A783AB1826842F0180282601B
:10288000826842F480528260497819B1C16841F08F
:102890003001C160D0F8B01041F00101C0F8B010B3
:1028A00070470D49C0B241EA0020074908647047EB
:1028B00005494FF020400864704700005880001020
:1028C00000800040040034120060004005F4010064
:1028D00020009B00D0FE0300130000A042484149A5
:1028E0008161891CC1614A1E4263036823F00303AE
:1028F00043F00D7343F080530360436923F00103F9
:1029000043F00D7343F08053436103691A4302613E
:10291000364A8260364AC260C2681143C160354996
:1029200000200860704710B501F03DF93148046897
:10293000002C08BF30BFFAD00021016001F037F948
:10294000204610BD10B501F02EF92648294B264926
:10295000421C1C682CB10020186001F028F92046A8
:1029600010BD72B648638A6120BF88614A6362B64F
:10297000BFF36F8FBFF34F8FEBE71B48016821F068
:10298000030141F00D7141F0805101601A498160ED
:1029900001691A4A1143016130BF704772B611498B
:1029A00011484163C91CC161891E816162B67047CB
:1029B0000D480168124A1143016070470A480168D6
:1029C00021F0030141F00D7141F080510160704729
:1029D00072B6044904488161891CC161491E416382
:1029E00062B6704700003412008000403C00341290
:1029F000280034125C8000100800341201003412E8
:102A000003003412704770470022B2EBD10F26D278
:102A10000368B3F1FF3F04BF4368B3F1FF3F17D131
:102A20008368B3F1FF3F04BFC368B3F1FF3F0FD129
:102A30000369B3F1FF3F04BF4369B3F1FF3F07D11F
:102A40008369B3F1FF3F04BFC369B3F1FF3F01D016
:102A5000002070472030521CB2EBD10FD8D3012098
:102A6000704710B40023B3EBD20F30D2D0F800C0BF
:102A70000C68A44522D1D0F804C04C68A4451DD1EF
:102A8000D0F808C08C68A44518D1D0F80CC0CC6828
:102A9000A44513D1D0F810C00C69A4450ED1D0F8CC
:102AA00014C04C69A44509D1D0F818C08C69A4455C
:102AB00004D1D0F81CC0CC69A44502D010BC0020C1
:102AC0007047203020315B1CB3EBD20FCED310BC4B
:102AD000012070472DE9F041054601F06CF8002017
:102AE00021264FF4825784464FF4E0221660C5F841
:102AF00000C0116841F004011160116811F0040F69
:102B0000FBD1176080232C460021D4F80080B8F157
:102B1000FF3F04BFD4F80480B8F1FF3F1DD1D4F8C3
:102B20000880B8F1FF3F04BFD4F80C80B8F1FF3F34
:102B300013D1D4F81080B8F1FF3F04BFD4F814804B
:102B4000B8F1FF3F09D1D4F81880B8F1FF3F04BFB6
:102B5000D4F81C80B8F1FF3F08D0C2F800C0401C78
:102B6000C0B20828C2D30220BDE8F081491C20343D
:102B7000B1EBD30FC9D3C2F800C00120BDE8F0818A
:102B80002DE9F041054601F016F80020092684469B
:102B90004FF4E0231E60C5F800C0196841F004013D
:102BA0001960196811F0040FFBD12C464FF48062B4
:102BB00000212768B7F1FF3F04BF6768B7F1FF3F07
:102BC00017D1A768B7F1FF3F04BFE768B7F1FF3F30
:102BD0000FD12769B7F1FF3F04BF6769B7F1FF3F26
:102BE00007D1A769B7F1FF3F04BFE769B7F1FF3F1E
:102BF00008D0C3F800C0401CC0B20328CAD30220CA
:102C0000BDE8F081491C2034B1EBD20FD1D3C3F819
:102C100000C00120BDE8F0812DE9F05F88468146C3
:102C200004274FF07F0A4FF0020B4FF4E02600F02C
:102C3000C2FF4946424653464FF0060CC6F800B064
:102C400052F8040B41F8040BC6F800C0306810F0CD
:102C5000040FFBD15B1EF1D2002030604C4645468C
:102C60001F20D4E900C3D4E90221D5F800E0E645ED
:102C700004BFD5F804C09C4505D1AB68934204BF9E
:102C8000EA688A4208D07F1E03D34846FFF722FF36
:102C9000CDE70220BDE8F09F10341035401EE0D291
:102CA0000120BDE8F09F70B50D46044600F083FF9B
:102CB0004FF400722146284619F096F9012070BDA4
:102CC0002DE9F0410546C005ADF5007D14460E46E0
:102CD000C00D25D0A8466FF308086F4600F06BFFC3
:102CE0004FF400724146384619F07EF9C5F30800EA
:102CF000C0F50077A74288BF274668443A46314668
:102D000019F081F94046FFF7E5FE022844D06946F4
:102D10004046FFF781FF022843D03D443E44E41B78
:102D2000B4F5007F19D34FF400723146684619F0AC
:102D30006AF92846FFF7CEFE02282DD069462846BC
:102D4000FFF76AFF02282CD0A4F5007405F5007582
:102D500006F50076B4F5007FE5D2C4B16F4600F009
:102D60002AFF4FF400722946384619F03DF92246F1
:102D70003146684619F047F92846FFF7ABFE0228AE
:102D80000AD069462846FFF747FF022809D00DF50B
:102D9000007D0120BDE8F0810DF5007D0A20BDE831
:102DA000F0810DF5007D0B20BDE8F0812E49086013
:102DB000086100F010B82C490860486100F00BB8B9
:102DC0002949486770472849886770472648012184
:102DD0000166016570474FF04022116B10F0010F42
:102DE00018BF21F4404110F0020F1CBF21F44051E4
:102DF00041F4805110F0040F18BF21F4406110F02D
:102E0000080F18BF41F4407110F0100F18BF41F0C7
:102E1000C00110F0200F18BF41F0300110F0400F3A
:102E200018BF41F00C0110F0800F18BF41F00301F2
:102E300041F4BE0141F020411163D2F8901010F42A
:102E4000807F1CBF21F0030141F0020110F4007FDC
:102E50001CBF21F00C0040F0080141F4BE0040F01E
:102E60002040C2F890007047001000407047D048E2
:102E70008268D0490A438260C2681143C1604169D7
:102E8000CD4A114341617047C948416921F00101B0
:102E900041F00D7141F080514161C16821F0400164
:102EA00041F00D7141F08051C160816821F0400115
:102EB00041F00D7141F080518160704710B5BC4CFC
:102EC000A168BC480143A160E1680843E060606913
:102ED000B94908436061B94843F63F71C1600021B8
:102EE00081638164C0F8B01003210A2000F0A5F9C5
:102EF0000A2000F0C5F9606920F0010040F00D7073
:102F000040F080506061E06820F0400040F00D70BB
:102F100040F08050E060A06820F0400040F00D706C
:102F200040F08050A06010BDA44A1060516048433A
:102F300090607047A14A10605160484310F0010F43
:102F400018BF401C906070479C49C1F8B0007047A2
:102F50009A49002818BF0120886470479749886300
:102F6000C86840F00200C8607047DFF850C2CCF873
:102F70002000CCF82410CCF82820CCF82C300120EC
:102F8000CCF83000DCF8340010F0010F05D020BF81
:102F9000DCF8340010F0010FF9D110F0020018BF76
:102FA0004FF0FF3070478548C16821F00201C160D1
:102FB00070478248C16841F00101C16070477F4B92
:102FC000186259629A6201201864586C10F0010F5F
:102FD00004D020BF586C10F0010FFAD110F0060099
:102FE00018BF4FF0FF3070477448C16821F00101ED
:102FF000C16070477148C16841F00401C160704709
:10300000027C017B02F03F0241EA02416B4A91657A
:1030100001685162416891628168D1620121116544
:10302000516D11F0010F04D020BF516D11F0010F4F
:10303000FAD1D36D8382D36D1B0CC382136E0383CD
:10304000136E1B0C4383536E8383526EC2F30E4286
:10305000C28311F0020018BF4FF0FF30704757488D
:10306000C16821F00401C16070475448C16841F053
:103070000801C1607047DFF844C1CCF87820CCF873
:103080002000CCF82430CCF828100120CCF87000B7
:10309000DCF8740010F0010F05D020BFDCF87400DC
:1030A00010F0010FF9D110F0060018BF4FF0FF30FB
:1030B00070474248C16821F00801C160704701684B
:1030C0004FEA31423D49C1F89C204068C1F8A00058
:1030D000C86840F02000C860704701684FEA31427C
:1030E0003649C1F89C208088C1F8A000C86840F02B
:1030F0002000C8607047314B18625A629962012003
:10310000C3F89400D3F8980010F0010F05D020BF49
:10311000D3F8980010F0010FF9D110F0060018BF95
:103120004FF0FF307047254A106251620120C2F80B
:103130009000D2F8980010F0010F05D020BFD2F80F
:10314000980010F0010FF9D110F0060018BF4FF0F1
:10315000FF3070471948C16821F02001C1607047F5
:103160001648C16841F01001C1607047A3F1050C19
:10317000124BC3F888C018625A6299620120C3F8E2
:103180008000D3F8840010F0010F05D020BFD3F8E1
:10319000840010F0010FF9D110F0060018BF4FF0B5
:1031A000FF3070470548C16821F01001C1607047C9
:1031B00000800040400034120100341200900040B2
:1031C0001B4810B5022140F8501F01210161102158
:1031D000416241F206014161002181610421816364
:1031E00090214163416B41F0010141634FF48171D2
:1031F00001610161032000F043F80021032000F089
:103200001CF8002010BD10B5032000F045F8084858
:103210004FF480710166002101661021816702214F
:103220004165002010BD0349002008707047000070
:103230000030004060800010704700F00303DA00A7
:103240004FF0FF0C0CFA02F24FF0050C0CEBC3032D
:1032500001FA03F300F00C0101F1E021002807DA84
:10326000D1F8140D90431A401043C1F8140D704763
:10327000D1F8000490431A401043C1F8000470478D
:1032800000F01F01012202FA01F14009800000F163
:10329000E020C0F80011704700F01F01012202FA7F
:1032A00001F14009800000F1E020C0F88011704772
:1032B00000F01F01012202FA01F14009800000F133
:1032C000E020C0F8801270474FF0E021C1F8000103
:1032D00070474FF0E021C1F8800170474FF0E020C7
:1032E000D0F8000170474FF0E021C1F8800270472C
:1032F000084800687047074A116810600846704720
:10330000044A126800F1100352F8230042F8231017
:103310007047000008ED00E002210C20FFF78DBF90
:10332000B8488268B8490A438260C2681143C160E4
:103330007047B448816821F4805141F00D7141F02B
:1033400080518160C16821F4805141F00D7141F0DC
:103350008051C1607047AD4881B0016F11F4007FAA
:10336000FBD1816E11F0010F1CBFD0F884100091C9
:1033700004D0D0F88410009A9142FAD0016F11F471
:10338000007F04BF4CF27101016642F24131816657
:1033900001B070479D4981B04FF40D528A660A6FA3
:1033A000CA66012898BF012005D9401EB0F5803FAC
:1033B00028BF4FF6FF7082B24FF05C5040EA022007
:1033C00048664FF01140C1F88000086F10F4007F8C
:1033D000FBD1886E10F0010F1CBFD1F88400009063
:1033E00004D0D1F88400009A9042FAD0086F10F40B
:1033F000007F04BF4CF27100086642F241308866DB
:1034000001B07047814881B0016F11F4007FFBD19A
:10341000816E11F0010F1CBFD0F88410009104D010
:10342000D0F88410009A9142FAD04FF40D51816681
:1034300001B070477348806810F4805008BF70472F
:103440007248806E00F0010070477048406EC0F313
:103450000F2070476D48D0F88400704710B50C20DD
:10346000FFF726FF0C20FFF70BFF68490220486793
:1034700010BD664910B5032088670C20FFF70CFFCC
:10348000BDE810400C20FFF713BF614A11681060BF
:10349000084670475D4810B5016FC1665C4800681A
:1034A000002818BF80475B48016841F480510160E3
:1034B00010BD574840687047524810B5826852495D
:1034C0000A438260C2681143C16050490320886783
:1034D0000C20FFF7E1FE0C20FFF7EAFE00F05CF99C
:1034E0004D4B0420C3F888004FF6FF70C3F88C00E2
:1034F00072B66033FFF74EFF4FF40070186062B68B
:1035000010BDF8B572B64148016F11F4007FFBD1D0
:10351000816E11F0010F1CBFD0F88410009104D00F
:10352000D0F88410009A9142FAD04FF40D51816680
:1035300039494FF400320A6662B6D1F80412314DAF
:10354000002946D0324C4FF6FF73591AA160AA6980
:10355000D5F81CC002F00F020CF00F0C6244121DD3
:1035600001FA02F2A2F54341DFF8B0C051396145DA
:103570002FD2D0F88400191AE160B1F5803F28D22B
:10358000274B4FF0000CA1FB03070CFB037301FB5F
:103590000C31634618F03CFD401C40082061B0F53A
:1035A0007A7F38BF4FF47A701E4B9968002908BFA4
:1035B00098605A681A609968C3E901108A421BD959
:1035C000824205D9814201D9616002E0606000E079
:1035D000626000F0EDF8A86820F4805040F00D70B3
:1035E00040F08050A860E86820F4805040F00D70F2
:1035F00040F08050E860F8BD8242E9D88142E5D8C9
:10360000E2E70000008000400010341200C00040DB
:10361000648000105C80001000A000404F62250014
:1036200000E1F505D48C00100F4881680F4A114362
:1036300081600F48016841F404710160001F016856
:1036400041F004010160016841F010010160704720
:10365000084908607047BFF34F8F08490648086063
:10366000BFF34F8FFEE700000080004004003412DB
:1036700014ED00E008ED00E00400FA050CED00E0B8
:1036800015488168154A114381601003416941F072
:1036900001014161016A21F00F0211490A430262EE
:1036A000104B8A1EC3F8C420016570474FF04020BC
:1036B000006900F0700070474FF040200A4940F860
:1036C000301F0A4941600A4901660A49416670474C
:1036D0004FF04020406870470080004004003412E2
:1036E00003005FA000600040C0845FA095995FA0C8
:1036F0000A005FA000005FA0022824BF00207047DE
:10370000E04B53F8202043F820101046704770B566
:10371000DD4C206FDB4D10F0010F05D00120E0667D
:103720002868002818BF8047206F10F0020F08BFDC
:1037300070BD0220E0666868002808BF70BDBDE863
:1037400070400047D14810B58268D1490A43826071
:10375000C2681143C160CC4902220A6501230B668D
:103760000323CB664A65816821F0800141F00D7129
:1037700041F080518160C16821F0800141F00D71FC
:1037800041F08051C1600920FFF77AFD0221BDE8B8
:1037900010400920FFF751BDBC488268BC490A436C
:1037A0008260C2681143C160B74902200865704752
:1037B000B54902204865B548816821F0800141F093
:1037C0000D7141F080518160C16821F0800141F0AC
:1037D0000D7141F08051C1607047AC488068C0F302
:1037E000C0107047A848016F11F4007F14BF4FF458
:1037F00040714FF480710166704710B5A24CE06FC4
:1038000010F0020F4FF0010018BF0320606700F0B6
:103810006EF99E498A69C96902F00F02D04001F031
:103820000F01C8400521B0FBF1F04FF4057100090C
:10383000C4F8801018F0F1FB964A974B18F0F2FB91
:1038400018F0F5FBC4F88400206F10F4007F14BF5B
:103850004FF440704FF48070206610BD8A48016FAD
:1038600011F4807F14BF4FF440714FF40071016672
:103870007047854B30B4DA6F12F0010F14BF03228A
:1038800002225A6700EB4005C5EBC010C1EBC00037
:103890004FF4FA744C43C0EB001000EB40007F493A
:1038A00004EBC000A1FB0010784900224FF0020C8D
:1038B0008C69C008C96904F00F0401F00F012144AC
:1038C000C8400521B0FBF1F0B0F5803F05D3511C95
:1038D0004008CAB2B0F5803FF9D242EA0C2141F06B
:1038E0001001C3F88810C3F88C00186F10F4807FA3
:1038F00014BF4FF440704FF40070186630BC70472E
:103900006148016F11F4003F14BF4FF440314FF490
:103910008031016670475C48016F11F4803F14BF2D
:103920004FF440314FF40031016670475648006F44
:10393000C0F3002070475448006FC0F34020704728
:1039400052498968C1F3C011002904BF00207047A3
:103950004D4900280CBFD1F80002D1F8040270478D
:103960004A4B9A68C2F3C012002A04BF0020704775
:10397000454A00280CBFD2F88000D2F88800C0F376
:103980000A200CBFD2F88020D2F8882002F00F0263
:10399000D3F818C0DB690CF00F0C03F00F0363447D
:1039A0001A449140012202EB400048433C49A1FBEC
:1039B0000010000970473B4901200870704770B43F
:1039C000324B322251439A69D3F81CC002F00F02E5
:1039D0000CF00F0C6244121DD14008BF012104D02D
:1039E000B1F5803F28BF4FF6FF719A68C2F3C0124D
:1039F000002A1CBF70BC7047D3F808C0244A4CEAA8
:103A0000020CC3F808C0D3F80CC04CEA0202DA601A
:103A10001D4A4FF0020CC2F850C04FF40034146637
:103A20000425C2F88850C2F88C101F4DD566C2F824
:103A300074C01E4902283CBF124E46F820100021D7
:103A4000184801704FF400711166017819B920BF50
:103A500001780029FBD014669567D566C2F854C07A
:103A6000986820F0800040F00D7040F08050986021
:103A7000D86820F0800040F00D7040F08050D86091
:103A800070BC70477C80001000A0004000800040A7
:103A9000800034127B14AE47E17A843FCDCCCCCC8D
:103AA0001F85EB5178800010020002026759000068
:103AB0004FF0E0210020886108611F49486070478D
:103AC00010B54FF0E02460610020A0610221401E8B
:103AD000FFF7B3FB0720206110BD4FF0E02100206D
:103AE0000861704714480188491C018070471248DA
:103AF000806870472DE9F0410F4C0027054627806C
:103B0000A0684FF47A71B0FBF1F04FF0E026401E50
:103B10007061B7610221C81EFFF78FFB072030617B
:103B20002188A942FCD33761BDE8F08103494843AD
:103B300001498860704700008480001040420F00F7
:103B4000704770B505464FF40D500406A06603207B
:103B5000E066264860664CF2710020662448C4F88E
:103B6000800042F24630A06602210020FFF765FB8C
:103B70000020FFF785FB002D08BF70BDA06E42F24C
:103B800041310843A06670BD012110B588078167E7
:103B90004FF40D5181660020FFF77EFBBDE8104019
:103BA0000020FFF785BB012081074867704701208F
:103BB0008107886770474CF271008107086670477B
:103BC0000C4A11681060084670470A4808B500683A
:103BD00018B18047002818BF08BD4CF27101880752
:103BE0000166016FC166006F009008BD075E5F3718
:103BF00000AF2F919080001070B5FF4C00254FF45E
:103C0000E46125706570E570FC4818F0F2F94FF436
:103C1000E461FB4818F0EDF9A56025714C21F948E5
:103C200018F0E7F94C21F84818F0E3F965717421B0
:103C3000F64818F0DEF97421F54818F0DAF9E56075
:103C4000A5717421F34818F0D4F97421F24818F0E2
:103C5000D0F9256170BDE849002048707047E648FA
:103C600040787047E4480079002818BF0120704769
:103C7000E1488079002818BF01207047DE4840796C
:103C8000002818BF01207047DB48C078002818BF03
:103C900001207047DF48704770B5E04A054610784C
:103CA00051784218520014462946DA4818F0ABF908
:103CB00022462946D84818F0A6F9CF490120887134
:103CC00070BDCD4800697047CB48407800EB40019B
:103CD000C1EB4010CD4901EB800070472DE9F04168
:103CE000C54D0446C9496A78CD4F02EB4200C0EB8E
:103CF0004210CC4E01EB80033A78307821461044D4
:103D00004200184618F07FF96A78C14902EB420078
:103D1000C0EB421001EB80033A7830782146104422
:103D20004200184618F06FF901206871BDE8F08173
:103D3000B148C0687047B0484078C0EBC001C1EBE3
:103D40008010AE4901EB401070472DE9F041AA4EBA
:103D500007463078002814BFB348B448047814BF2D
:103D6000B348B448057804FB05F8FFF780F8294606
:103D70002046FFF7D9F87078A14CC0EBC001C1EB29
:103D8000801004EB4012A4F5E46101EB40103B46C7
:103D90000146FFF7EAF8FFF777F870784FEA480234
:103DA000C0EBC001C1EB801004EB4010394618F0A5
:103DB0002AF90120F070BDE8F0812DE9F0478E4D21
:103DC00004468E496A78DFF86082C2EBC200C0EB1D
:103DD000821001EB40132878DFF85092944E954FF3
:103DE000002815BF98F8000099F8000032783A785A
:103DF00000FB02F04FEA40022146184618F003F992
:103E00006A787F49C2EBC200C0EB821001EB401C14
:103E100028782146002815BF98F8002099F800203E
:103E200033783B7802FB03F04FEA4002604618F01B
:103E3000EAF80120E870BDE8F0876F4880687047B5
:103E400070B57D4C0546014622786E48520018F048
:103E5000DAF82278294652006B4818F0D4F86649FF
:103E60000120087170BD2DE9F04FDFF88C81ADF2B3
:103E7000647D98F80300CDF8440798F80400CDF865
:103E8000400798F80500CDF83C0798F80600CDF8F3
:103E9000380701F0B1F90446FDF7B6FDCDF85C072F
:103EA000FDF789FFCDF85807FDF7F1F9CDF8540774
:103EB000FCF771FFCDF84807FCF76AFF0746FDF7EE
:103EC000A5FDDDF8480710F0010F02D0FDF779FFDE
:103ED00004E00020FDF7D1F9FDF7ACFF98F80200EF
:103EE0001E250026002804BF0420C8F8180016D09C
:103EF000022C18BF0A200ED109F058FE38B10FF07D
:103F0000ACFE012806D00FF0A8FE082802D0C8F8A1
:103F1000185002E00F20C8F8180088F802604FF02F
:103F2000010A022F0ED1022C18BF052C0AD1FDF771
:103F300075F908300009022C18BFC8F818503AD09B
:103F400088F802A0D8F818000428BCBF0420C8F8DC
:103F5000180098F80200B8F81810000240EA014072
:103F600040F0010200239121072009F0D3F93746E0
:103F70004FF0000B05F047F8012826D00DF5E4605E
:103F8000FEF75AF9002800F0A5820DF5E46005F06F
:103F900003FF002088F80100D8F81800C01E8642F0
:103FA000CABF874201240024DDF82C0710B3DDF8D6
:103FB000400770B15DE04FF47A7141434FF47A707D
:103FC00091FBF0F0C8F81800BAE74FF0010B00F0D1
:103FD0006ABADDF82C9774B1174D4946287842002B
:103FE000084818F010F8287849464200064818F0AA
:103FF0000AF823E03DE024E094800010E08C0010FB
:104000000094001040A200108CA20010D8A2001052
:104010004CA3001034A40010A8A40010D4800010F9
:10402000D1800010D2800010CF800010CC80001012
:10403000D0800010CD800010D380001088F804A03C
:1040400017E0FEF714FFFF4D01212878FEF76CFF03
:10405000FD4A4B46A2F14C010846FEF786FFFEF7EB
:1040600013FF287849464200F74817F0CCFF88F83C
:1040700004A0DDF82807002800F0D780DDF8440709
:10408000002840F0D28098F80000DDF82857E0BB07
:10409000D8F80890B9F1000F24D0EC480078CDF89A
:1040A0005007EB480078CDF84C07FEF7E0FEDDF84E
:1040B0004C17DDF85007FEF73DFF29464A460846F3
:1040C000FEF77DFFFEF7E0FEE2480078022804BF1D
:1040D000484605F034FBDF480078092804BF28462D
:1040E00005F02DFBDC480078012816D9DFF8649331
:1040F00099F80000042804BF284605F020FB294653
:10410000684617F099FF054600E006E099F80000C0
:10411000052804BF284605F012FBCCB398F801002F
:1041200098F80020C0EBC001C1EB8011CB48002AF9
:1041300000EB411029460CBFC94AC44A137814BF8A
:10414000C34AC84A127803FB02F24FEA420217F050
:104150005AFF98F80100C0EBC001C1EB8011C248C2
:1041600000EB411398F800002946002814BFB74817
:10417000BB48007814BFB64ABA4A127800FB02F076
:104180004FEA4002184617F03EFF88F803A03DE0D2
:10419000FFE7CDF84C5798F80000002814BFAB4853
:1041A000AF4890F8009014BFA948AE48057809FBC5
:1041B00005F0CDF85007FEF75AFE29464846FEF7AF
:1041C000B3FE98F80100A84DC0EBC001C1EB801010
:1041D00005EB4012A5F5E46101EB40100146DDF866
:1041E0004C37FEF7C2FEFEF74FFEDDF850074200E7
:1041F00098F80100C0EBC001C1EB801005EB401046
:10420000DDF84C1717F0FFFE88F803A091480078FE
:1042100003280AD198F80100C0EBC001C1EB80115E
:104220008E4800EB411005F08AFADDF830070028CF
:104230007DD0DDF83C07002879D198F80000DDF842
:10424000305748BBD8F80C90B9F1000F24D08748FC
:104250000178874800780844401C400801900220FB
:104260000090FEF704FEDDE90010FEF763FE29462C
:104270004A460846FEF7A3FEFEF706FE7D48007894
:10428000022804BF484605F065FB7A4800780928F3
:1042900004BF284605F05EFB4CB398F80100DFF838
:1042A000D09100EB4001C1EB4011734800EB81035A
:1042B0006E482946027899F80000104442001846DA
:1042C00017F0A1FE98F80100684A00EB4001C1EB2D
:1042D00040116A48127899F8003000EB81001A44C6
:1042E0002946520017F08FFE88F805A030E05F489D
:1042F000009501785E4800780D18FEF7B8FD681C3F
:1043000040080221FEF710FE98F80100DFF86C91DA
:1043100000EB4001C1EB4010A9F1740109EB8002F0
:1043200001EB80010846009BFEF71FFE00E01EE047
:10433000FEF7AAFD98F801006A0000EB4001C1EB0E
:10434000401009EB8000009917F05DFE88F805A089
:104350004848007803280AD198F8010000EB400192
:10436000C1EB4011444800EB810005F0F3FADDF8A1
:104370003407002863D0DDF8380700285FD198F8AB
:104380000000DDF8345740BBD8F81090B9F1000FA9
:1043900023D03B48017840780844401C40080190F5
:1043A00002200090FEF763FDDDE90010FEF7C2FD7C
:1043B00029464A460846FEF702FEFEF765FD3148EB
:1043C0000078022804BF484605F0DEFB2D4800783F
:1043D000092804BF284605F0D7FB29480178407812
:1043E00074B10844440022462946274817F00BFEC2
:1043F00022462946254817F006FE88F806A017E051
:104400000C18FEF734FD601C40080221FEF78CFDFD
:104410001E4A2B46A2F174010846FEF7A6FDFEF7E0
:1044200033FD62002946194817F0EDFD88F806A013
:1044300014480078032804BF134805F0A5FBFDF7D6
:1044400058FF25E0D38000108CA20010CF80001010
:10445000D08000103D810010CE800010E08C001054
:10446000CC800010CD80001000940010D18000108E
:10447000D280001042810010D8A200104CA300107E
:10448000D48000104781001034A40010A8A40010AC
:10449000D8F81800761C7F1C8642A8BF874211DB23
:1044A000D8F8140070B1FDF7B1FADDF85407FCF745
:1044B000E4FEDDF85C0790B1DDF8580768B1FDF760
:1044C000B9FC0CE0DDF8480710F0010F08BFFDF75C
:1044D000B1FC4FE500F0DDFE4CE5FDF772FCBBF1F1
:1044E000000F04BF0420C8F818000FD0DDF84407FF
:1044F00088F80300DDF8400788F80400DDF83C0781
:1045000088F80500DDF8380788F80600B8F81810B4
:104510004FEA0B2040EA014200239121072008F0D6
:10452000F9FE0DF2647D5846BDE8F08F10B5002409
:10453000FDF733FCFF4910F0020F0AD0CA78002AB9
:1045400008BF012410F0040F03D00A79002A08BF25
:10455000012410F0010F03D04A79002A08BF01247A
:1045600010F0200F03D08879002808BF0124002014
:10457000002C08BF10BD00200870BDE8104072E498
:1045800008B50F2100F03AFF012804D1FFF7CEFF54
:10459000009001F0A2F8E748C17800291CBF4179DA
:1045A000002906D0817900291FBF00790028012049
:1045B00008BD002008BD08B50F2100F01FFF01282D
:1045C00004D1FFF7B3FF009001F087F8D948C17814
:1045D00000291CBF4179002906D0817900291FBF1D
:1045E00000790028012008BD002008BD7047D1498E
:1045F00000220028CA700A714A718A711CBF01200A
:10460000887000F011BD10B54FF4E461CA4817F08E
:10461000F0FCBDE810404FF4E461C84817F0E9BC75
:104620002DE9F041C34D069A2978002914BFC449E9
:10463000C4490978D21A4A4303FB01F4697852004D
:10464000C1EBC103C3EB8111BB4B164603EB411118
:1046500001EB440300EB44010F46184617F0D3FC6E
:1046600068783246C0EBC001C1EB8010B34901EB62
:10467000401000EB4400394617F0C5FC0120E870FB
:10468000BDE8F0812DE9F047AA4F804608983978B7
:10469000002914BFAA49AB490D78A0EB030905FB1B
:1046A00009F603FB05F4FEF7E2FB49462846FEF750
:1046B0003BFC7878A14DC0EBC001C1EB801005EB4D
:1046C000401101EB4402A5F5E46101EB401000EB61
:1046D000440008EB440843460146FEF746FCFEF75B
:1046E000D3FB78787200C0EBC001C1EB801005EB02
:1046F000401000EB4400414617F085FC0120F870A3
:10470000BDE8F087002818BF01208A49C8707047AB
:1047100010B5884C002804BFA06010BDDFF828C287
:1047200087490B7889490A7801465A435200604606
:1047300017F069FC8448A06010BD10B54C21844876
:1047400017F057FCBDE810404C21824817F051BCCF
:104750007F487047002818BF0120764908717047CC
:1047600010B574217C4817F044FCBDE8104074215A
:104770007A4817F03EBC002818BF01206D494871E7
:10478000704710B56B4C002804BFE06010BD742268
:104790000146734817F037FC7148E06010BD10B552
:1047A0007421704817F025FCBDE8104074216E4854
:1047B00017F01FBC002818BF01205E4988717047A0
:1047C00010B55C4C002804BF206110BD67490A7811
:1047D000497811444A000146654817F014FC6448C2
:1047E000206110BD70B5534C00210546E170217168
:1047F0006171A17100F018FC002D14BF0120002090
:104800002070BDE87040FFF72EBB2DE9F04F89B056
:104810004FF4E4614C4817F0ECFB7421504817F05A
:10482000E8FB7421524817F0E4FBFDF7B6FA0446A2
:10483000FDF7EAF80890FDF7BEFA0190FCF727FDB6
:104840000090FDF7E3F80020FCF717FDFDF7F2FA02
:1048500000252E4604F0D7FB012868D002A8FDF7FA
:10486000EBFC002864D002A805F096FA14F0020FC1
:104870001CD03348DFF8D0B0DDF8109090F80080FD
:104880003248DA460778FEF7F2FA0120FEF760FBBD
:1048900039464046FEF74EFB524649465846FEF71B
:1048A0008EFB0020FEF754FBFEF7EEFA14F0010F2A
:1048B00020D03048DFF8A8B04FF0020801782E4829
:1048C000DA46DDF8189000780844401C4708FEF7E7
:1048D000CEFA0120FEF73CFB41463846FEF72AFBA4
:1048E000524649465846FEF76AFB0020FEF730FB69
:1048F000FEF7CAFA14F0200F47D01C48DFF870907A
:104900004FF0020B01784078C8460844401C4FEA3B
:10491000500A079FFEF7ABFA0120FEF719FB594634
:104920005046FEF707FB42463946484626E034E04B
:1049300040E0000094800010E08C00100094001013
:10494000CF800010CC800010209B0010D080001081
:1049500040A200108CA20010D8A200104CA300109E
:10496000C0A3001034A40010A8A40010D48000102C
:104970001CA50010D1800010D2800010FEF71FFB94
:104980000020FEF7E5FAFEF77FFAFDF7B2FC6D1C9A
:10499000102D03D2FDF74EFA5CE70126FDF736F83D
:1049A0000098FCF76AFC089848B1019828B1FDF717
:1049B00041FA04E000F06DFC4CE7FDF702FA96BB0B
:1049C000F84D14F0020F4FF001070DD0F648009794
:1049D00010230178F548007801FB00F2F4490846FD
:1049E00017F02FFBF248A86014F0010F0CD0F1482B
:1049F000009710230178F04800780A18EF4908461C
:104A000017F01FFBED48E86014F0200F0BD0EC48C6
:104A100000971023017840780A18EA49084617F0F1
:104A200010FBE848286109B03046BDE8F08F01204E
:104A300070472DE9F0414FF43F300027D0E90015D1
:104A4000D0E903464BF6BB38ADF5007D41452BD090
:104A50004FF40071684617F0CCFAFF224FF4007152
:104A6000684617F0F3FAFF2060F307052D2060F386
:104A7000070460F30F24282060F31744CDF800806A
:104A8000CDE90346CDE901574FF43F342046FEF708
:104A900021F869462046FEF7BFF801281EBF002016
:104AA0000DF5007DBDE8F08101200DF5007DBDE82C
:104AB000F0814FF43F3070474FF43F31042804BF7A
:104AC000C87A704710DC002804BF087970470128B5
:104AD00004BF087A7047022804BF487A7047032849
:104AE00004BF887A70470BE0142804BF087B704726
:104AF000152804BF487B7047162804BF887B704781
:104B0000FF2070472DE9F0434FF43F3CADF5017DA8
:104B1000DCE9015461F3070462F30F24DDF820920D
:104B2000DCE9037860F3070563F3174469F31F6456
:104B3000FF224FF400716846DCF8006017F086FA37
:104B40000096CDE90154CDE903784FF43F34204677
:104B5000FDF7C0FF69462046FEF75EF8012818BF42
:104B600000200DF5017DBDE8F0832DE9F04F4FF4F5
:104B70003F33ADF5017DD3E90274D3E90056904689
:104B800089468246FF224FF400716846D3F810B080
:104B900017F05CFA6AF3070469F30F2468F317440B
:104BA000CDE90274CDE900564FF43F34CDF810B092
:104BB0002046FDF78FFF69462046FEF72DF80DF5DC
:104BC000017DBDE8F08F2DE9F04F0027ADF5017DA7
:104BD0007D4C42F20F783D461420FFF76DFF40B246
:104BE00002901520FFF768FF4FFA80F91620FFF7B3
:104BF00063FF40B201901620FFF75EFF404240B2D3
:104C00000090FDF7CAF8DFF89CA1834600208AF8DF
:104C100003008AF804008AF805008AF8060000F00C
:104C200003FA00208AF80000FFF71DF91BF0010FBE
:104C300004D017F010FA012808BF01271BF0020F5B
:104C40007ED062489AF80110002690F800C06048B3
:104C5000C1EBC102C2EB811100785E4A002802EB71
:104C60004112C8BFACF1010A1DDD0021BAF1000FED
:104C700016DD01F1010B01FB00630BFB006B32F849
:104C8000133032F81BB0A3EB0B031BB2002BB8BFE1
:104C90005B421BB2AB42C8BF1D46491C5145E8DB15
:104CA000761C8642E1DBA945B8BF47F00207002623
:104CB000B146BCF1000FC8BFA0F1010A1BDD002105
:104CC000BAF1000F13DD09FB001332F813B002EB49
:104CD00043035B88ABEB03031BB2002BB8BF5B4203
:104CE0001BB2B342C8BF1E46491C5145EBDB09F15C
:104CF0000109E145E3DB0299B142B8BF47F0020781
:104D00004FF00009BCF1000F13DD002300280CDD7B
:104D100009FB003132F91110A142C8BF0C464145D0
:104D2000B8BF88465B1C8342F2DB09F10109E1450B
:104D3000EBDB0198A04202DB0098404503DD00E078
:104D400001E047F002074FF43F32C8F10001D2E919
:104D5000018066F3070065F30F20D2E903AB64F32B
:104D6000174061F31F600446D2F8009067F307080C
:104D7000FF224FF40071684617F068F9CDF80090F3
:104D8000CDE901844FF43F342046CDE903ABFDF774
:104D9000A1FE69462046FDF73FFF0DF5017DBDE808
:104DA000F08F000094800010CF800010D0800010A1
:104DB000209B0010D1800010D2800010C0A30010F2
:104DC000D48000101CA50010F1D8FFFFCD8000108A
:104DD000CC800010E08C0010FA4880897047F948B8
:104DE000C089704770B515460E46044608F05BFE54
:104DF000002C18BF70BD042806D0F348006890F856
:104E00002400A84288BF70BD3046BDE8704017F04E
:104E100027B9DDF800C0084312BF52EA03000020A2
:104E20008CF800007047E74840697047E549012069
:104E300048617047E3490020486170470143E148F9
:104E400018BF142AD4BF0121002141617047DD48F9
:104E50000021C171018270472DE9F04790468946D3
:104E6000044608F0CBFD0027D64E002802BFF7719C
:104E70003782BDE8F087B6F910008442C8BF34829B
:104E8000204617F0F2F804460D46B6F9100017F068
:104E9000ECF8CE4ACE4B17F0C5F822462B4617F059
:104EA00021FA13D2B9F1010F10D0F079401CC0B231
:104EB000F071032898BFBDE8F087F77137820120B1
:104EC0003071801EC8F80000BDE8F087F771BDE8BA
:104ED000F0872DE9FF5F0546BE480A26002490F8BA
:104EE0000090BD48B74FDDF838B090F8008092468A
:104EF000012B08BFBBF1000F1BD008F07FFD01287C
:104F00001DD0B889012888BF1E2336D97989002091
:104F1000A1421CBF7C81B871002119EB08021FD08F
:104F200035F911C09C4517DDB87104B00020BDE80B
:104F3000F09FB879052828BF05201ED31CE0BBF1DF
:104F4000010F08BF4123E1D03C2301240526BAF11B
:104F5000000FC8BF3323D9E7491C89B28A42DFD882
:104F6000B979491CC9B2B971B14206D901994FF05A
:104F7000FF320A6001213971B87104B00020BDE828
:104F8000F09F70B51E4615460C4608F037FD012807
:104F90001AD10021DFF82CC2002DC2BF8CF80510F9
:104FA000002070BD012E0FD09CF80500401CC0B23F
:104FB0008CF805000A2807D94FF0FF302060012047
:104FC0008CF804008CF80510002070BD00207D4A8C
:104FD000034601291CBF137070471078401CC0B2F3
:104FE0001070042826BF137002200120704708B5F6
:104FF00002237A490A787A490978891E00910021AA
:10500000FFF70EFB012008BD744908B50A78744902
:1050100002230978891E00910021FFF733FB01204C
:1050200008BD6848007A704710B508F0E7FC002812
:1050300008BF10BD08F0E5FC00230121BDE81040C9
:105040001A46022008F066B9664A028042800021B2
:105050008280C1800181534243818181C18101826B
:105060004182017501834183C28270472DE9FF4F60
:1050700083B01446DDE910A70546DDF848B008F016
:1050800012FD0195DFF83C8100252E4688F8085076
:1050900008F08CFD4FF0010948BB08F057FE0146AF
:1050A00001AA1398FFF7D8FE3B46524601A9CDF856
:1050B00000B00498FFF70DFF08F0A0FC012816D1FE
:1050C000BAF1000FC8BF88F8056010DC012F0ED0C0
:1050D00098F80500401CC0B288F805000A2806D9D7
:1050E0004FF0FF30019088F8049088F8056008F0D0
:1050F00080FE012808D1D8F8140028B10025012F1E
:1051000018BF88F800600CD00198344A3449B0F1D7
:10511000FF3F04BF98F8040001280FD0022D2DD0C6
:1051200036E098F80000401CC0B288F8000004285F
:1051300026BF88F8006002250125E5E788F80460AD
:1051400088F80890012D18BF022D08D0002C04BF4C
:1051500007B0BDE8F08F2046FEF72FFE18E0002CC8
:1051600004BF07B0BDE8F08F204609781278891E89
:10517000009102230021FFF753FA09E044B10978B6
:105180001278891E0091204602230021FFF77AFA47
:105190000198002807BF98F80200012807B0BDE871
:1051A000F08F88F8026088F80890002C1CBF204619
:1051B000FEF7CBFD0698002818BF16F05BFF07B07E
:1051C000BDE8F08FB0800010D4810010CDCCCCCCE5
:1051D000CCCCE43FD1800010D2800010CC800010F5
:1051E000CD800010F1D8FFFF10B505F08DFD05F062
:1051F00038FE002010BD0000FE4800787047FD48D2
:1052000040787047FB480078022805D005281CBF6D
:105210000020704704F0D5BF08F045BCF549087080
:10522000704770B5F34E04460D463078A04212D058
:1052300002281AD0052814BF002004F0C2FF44EA57
:1052400005213278002341EA024141EA00626121EE
:10525000072008F05FF87570072C28BF70BDDFE8E5
:1052600004F016070B13160F160008F01CFCE6E7F7
:10527000284600F03FFA0AE0284608F00FFC06E056
:10528000284604F093FF02E0284608F0EBF834705B
:1052900070BDD94900200968B1F8641011F4807F0D
:1052A00008BF7047FDF73FBBD34900200968B1F83C
:1052B000641011F4807F08BF7047FDF743BBCE49EF
:1052C00000200968B1F8641011F4007F08BF70472E
:1052D00016F0D5BEC84900200968B1F8641011F471
:1052E000806F08BF704716F0CFBEC249887800288B
:1052F0001CBF401E8870704770B5C049D1F8CC0003
:10530000BC4C10F0030F0AD040F4BE0040F0204027
:10531000C1F8C800A078002804BF0120A070B848D8
:105320008068B54D10F0020F296807D14FF040207A
:10533000406910F0010F01D0A07840B1B1F86410BD
:10534000002011F4807F18BFFDF7FCFA07E0B1F8E8
:105350006410002011F4806F18BF16F095FEA94963
:10536000084208BF70BD2968496E090CA17070BD64
:1053700010B572B6FEF708FCBDE81040FEF76BB939
:1053800010B5012802D0022805D008E04FF44330C0
:10539000FDF7A0FB03E04FF040219B48086772B681
:1053A000FEF7F2FBBDE81040FEF755B99149002821
:1053B00018BF0120C87070478E48C078002818BFF9
:1053C000012070478B48406970478A4800697047E0
:1053D0008849886170478748806970478549C861F6
:1053E00070478448C06970478348026802F5C073FB
:1053F000118A508A02F5A072FCF7A9BD2DE9F04F81
:10540000DFF8F09197B08A46C9F8140005F0ACFBBC
:10541000C9F81000002800F0A58090F800C089F8B5
:1054200004C0417889F80510837804460CF1010026
:1054300089F8063000F0FE0089F80700E27889F864
:105440000820207989F80900607989F80A0009F1B3
:105450000C05A0792870E0796870207889F80B0035
:105460006046FCF7B5FE99F80A1099F80900FCF7B8
:10547000D2FE69782878FCF7D8FE6946204605F008
:1054800096FB608AD9F8185000281CBF6843050BAA
:10549000B4F81A80D9F81C60B8F1000F08BF4FF4B7
:1054A0008058678C002F08BF4FF4805700201AF0F7
:1054B000040F18BF4FF485701AF0080F18BF40F0A2
:1054C00004001AF0020F1CBF40F2012108431AF039
:1054D000010F18BF40F48460616A6FF30F0A08403F
:1054E0006FF30F0108434AEA000A009810900498ED
:1054F0001190089812900C981490019813900798A6
:10550000159010A95046FCF74DFB1AF0020F65D01C
:1055100005F03BF85FEA000B31D005F04DF8684329
:10552000050B59460020FBF7C7FE218A00291CBF46
:105530000020FBF740FF05F05FF87043000B00F51B
:105540000060010A0820012202FA00F30B4201D197
:10555000401EF9D5061FA07B002818BFA0F1010B43
:1055600017D112E024480068B0F8640010F4807F7E
:1055700018BFFDF7E7F9002017B0BDE8F08FB4F8C9
:105580000CB0BBF1000FCCD1CFE70020FBF796FFAA
:105590008346E07B002814BF401EFBF7CFFF0BEBD8
:1055A0000601042903DD711A0E1D042103E0002900
:1055B000BCBF761A00210644042E03DD301FC5400F
:1055C000042604E0002E02DA704285400026002006
:1055D000FBF78DFF31460020FBF7C9FF1AF0010FE2
:1055E00030D0A18A00291CBF0120FBF765FE268B65
:1055F000A6B10BE0C8800010D4810010006000400C
:105600000080004008000300AD2007B031460120B3
:10561000FBF7D1FE31461120FBF7CDFEA67D3EB152
:10562000711E0120FBF763FF711E1120FBF75FFF66
:10563000E67D3EB1711E0120FBF799FF711E11201E
:10564000FBF795FF1AF0200F23D0A18B00291CBF78
:105650000220FBF731FE268C3EB131460220FBF7DB
:10566000AAFE31461220FBF7A6FEA67F3EB1711EB0
:105670000220FBF73CFF711E1220FBF738FFE67F8C
:105680003EB1711E0220FBF772FF711E1220FBF764
:105690006EFFE07A00281CBF0001FBF749FD02986D
:1056A00004F04FFF039830B12B4699F8052099F884
:1056B000041016F0EEFC3A464146284616F0EEFC81
:1056C0000598FFF725F80998FFF75BF80D98FFF7A5
:1056D00077F817B00120BDE8F08F10B5FCF71EFB7E
:1056E00004F037FF024900200861012010BD0000CE
:1056F000C8800010FE4908707047FD480078704768
:10570000FC4810B4FC4A0168914218D14168B1F5D7
:10571000887F14D80022D0F808C003461146B2EBA7
:105720009C0F24BF10BC704753F82140491C2244F1
:10573000B1EB9C0FF8D3002A04BF10BC70470020C7
:1057400010BC7047EB48FDF7C5B9E9490120087066
:1057500070472DE9F34FE5B0002045908A465590FB
:10576000549072B6FCF719FB0646FEF736F848B1BE
:10577000FEF7DCF85590FEF7C3F8FEF7DCF854901E
:10578000FEF7C9F8FCF703FAFCF73EF95C90FCF76A
:1057900012FB5B90FCF73AF9FCF79BFB5D90002055
:1057A000FCF791FBFDF746FE5A90FDF72BFE4FF4F8
:1057B0009350FDF798FD62B60020074636AD45F8D8
:1057C0002070401C0628FAD3DFF8308316F0020F51
:1057D0004FF001040AD041F618514046369416F0B5
:1057E00008FC41F61851C64816F003FCDFF8149384
:1057F00016F0010F15D04FF41871C34816F0F9FBDD
:105800004FF41871484616F0F4FB0120FBF709F835
:10581000002818BF38941120FBF703F8002818BFA0
:10582000399416F0200F15D04FF41871B64816F0C1
:10583000E0FB4FF41871484616F0DBFB0220FAF744
:10584000F0FF002818BF3A941220FAF7EAFF002868
:1058500018BF3B94DFF8B492A54E36984FF0405BEA
:1058600068B300210846FBF717FE009001210020D5
:10587000FBF712FE019099F800008DF80800A4488B
:105880000078012894BFA348A34800788DF8090048
:105890000020FBF72DFF002818BF4FF0FF300490C9
:1058A0008DF80AA07088ADF80C000020FBF7A1FD70
:1058B000ADF80E009948CDF81880CDE907B03798BB
:1058C0004FF0FF0A68B300210846FBF7E5FD099099
:1058D00001210020FBF7E0FD0A9099F800008DF807
:1058E0002C008DF82D400D978DF82EA07088ADF806
:1058F00030000020FBF77DFDADF832009DF8090077
:1059000000EB400101EB001108EB81010F919DF8C4
:10591000081048430BEB40011091804901EB400017
:1059200011907F4FDFF8FC81389870B3002101207F
:10593000FBF7B2FD012112900846FBF7ADFD139075
:10594000FBF743FA00280CBF98F8000038788DF870
:1059500050000120FBF7B2FD04FA00F08DF8510071
:105960000120FBF77AFEC04316908DF852A0B08854
:10597000ADF854000120FBF73CFDADF8560062483D
:1059800018906948199069481A90399870B30021A5
:105990001120FBF781FD1B9001211120FBF77CFDFD
:1059A0001C90FBF712FA00280CBF387898F800001A
:1059B0008DF874001120FBF781FD04FA00F08DF8DA
:1059C00075001120FBF749FEC0431F908DF876A0AB
:1059D000B088ADF878001120FBF70BFDADF87A0028
:1059E000534821905348229053482390534F3A985C
:1059F00040B300210220FBF74FFD2490012102203B
:105A0000FBF74AFD259038788DF898000220FBF7C7
:105A100055FD04FA00F08DF899000220FBF71DFEF9
:105A2000C04328908DF89AA0B088ADF89C00022061
:105A3000FBF7DFFCADF89E0041482A9041482B90CF
:105A400041482C903B9840B300211220FBF724FDE5
:105A50002D9001211220FBF71FFD2E9078788DF8F4
:105A6000BC001220FBF72AFD04FA00F08DF8BD00FF
:105A70001220FBF7F2FDC04331908DF8BEA0B08834
:105A8000ADF8C0001220FBF7B4FCADF8C2002F48FF
:105A900033902F4834902F4835909DF851000227BD
:105AA000022888BF8DF851709DF87500022888BFC4
:105AB0008DF875704FF055361F9601201696FBF73E
:105AC000CCFD18B171000120FBF7B7FD1120FBF7E9
:105AD000C4FD20B14FF0AA311120FBF7AEFD9DF8B7
:105AE0009900022888BF8DF899709DF8BD0033E0B9
:105AF000E880001000FE020054435246008000304F
:105B000000A0003018BD0030189D0030CF8000107C
:105B1000CE800010CD800010D080001000400030FA
:105B2000D1800010D2800010CC090030CC49003068
:105B3000B09D0030CC0E0030CC4E0030D480001030
:105B4000489E00304C1800304C580030E09E003029
:105B50004C1D00304C5D0030022888BF8DF8BD70B0
:105B6000319602202896FBF778FD20B14FF0AA313C
:105B70000220FBF762FD1220FBF76FFD20B14FF012
:105B8000AA311220FBF759FDBDF8540000F58060E2
:105B9000ADF85400BDF8780000F58060ADF87800ED
:105BA000BDF89C0000F58060ADF89C00BDF8C00019
:105BB00000F58060ADF8C000FBF73AFD5E90012073
:105BC000FBF72CFD0120FBF7ACFD61900020FBF7FB
:105BD00064FF60900020FBF755FF5F900020FBF70B
:105BE0004CFB6290FCF726F90020539052903D90B8
:105BF00044904598002840F0988303F004FA012867
:105C000000F093835398802800F28F8346A8FCF716
:105C100013FB002800F0838346A804F0BDF85298D7
:105C2000401C529000F07283002052905398401C08
:105C3000539000203EAA012142F82010401C062863
:105C4000F8D33D98002808BF3C9013D0012804BF2A
:105C500000203C9000F0E480022804BF00203C902B
:105C600000F00782032804BF0120459000F02D8337
:105C700000F05BBB3C9936A850F8210000287DD08D
:105C800001EBC101684600EB81000021449A4D916F
:105C900001684E9141684F91077A417A4C91D0E961
:105CA0000681B0F90C600069C2F108055090FAB1A4
:105CB000002D7DDB4C984FF0000A002861D905F1DA
:105CC0000800012202FA00FBE81D02FA00F05690DB
:105CD0000123509803FA0AF2104018BF0120002255
:105CE00057900AEB4A0000EB0A10944651907EE070
:105CF0004C980024002888BF4FF0010E7FD950989F
:105D00000EFA04F2024214BF4FF0010B4FF0000BE9
:105D1000002004EB440202EB04128446519228E076
:105D200043094EAA52F8232000F01F030EFA03F392
:105D30001A421BD000F0010208EB4233519A4FEA9D
:105D4000500903EB820A31F9023B5AF829209B1BC8
:105D50000CF1010CBBF1000F18BF5B42002BC8BF58
:105D600042F4803242F400424AF82920401C26289E
:105D700001D2BC45D4D3641C4C9800E048E0844276
:105D8000BDD33CE053094EA802F01F0450F8233065
:105D90000120A040034227D002F0010008EB40336D
:105DA00051984FEA520903EB800454F8290000E0AF
:105DB00029E031F9023BDDF85CE19B1B0CF1010CA1
:105DC000BEF1000F18BF5B4210F4803F02D0002BE1
:105DD00004DA01E0002B01DD20EA0B00002DC4BF36
:105DE000569B184344F82900521C262A01D2BC4570
:105DF000C8D34C980AF1010A8245FFF469AF002D1F
:105E000004BF01204D903EA93C9A4D9841F82200D4
:105E10003C98401C3C900628FFF42CAF00F055BA8B
:105E20003C9936A850F82100002800F01A813C98CF
:105E3000449900EBC002684600EB820000225092B9
:105E400002684C9242684D92037A457A847A4F9464
:105E5000D0E906C2B0F90C8004695194C0894F9C06
:105E6000C1F1080600EA0407E9B1002E75DB4FF026
:105E7000000A002D70D9012000FA06FB701E0121D6
:105E800001FA00F059900124519804FA0AF10840EF
:105E900018BF012000214E900AEB4A0000EB0A10C7
:105EA0008946589092E04FF0000A002D54D9012401
:105EB000519804FA0AF1084018BF012000214E90C1
:105EC0000AEB4A0000EB0A10894657903EE04C0965
:105ED0004CA801F01F0B50F82440012000FA0BF0F1
:105EE000044230D001F001000CEB403457984FEAE7
:105EF000510B04EB8000569032F9024BDDF838E18B
:105F000050F82B00A4EB080409F10109BEF1000FC1
:105F100018BF644210F4803F09D0002C0EDA10F450
:105F20007F4018BFA0F5807040F4803006E0002C60
:105F300004DD10F47F4018BFA0F5807040F08000B1
:105F4000569C44F82B00491C262901D29945BED302
:105F50000AF1010AAA45AAD33FE042E04C094CA845
:105F600001F01F0E50F82440012000FA0EF0044208
:105F700029D001F001000CEB40345898DDF838E1ED
:105F800004EB80004C08CDE9564050F8240032F96B
:105F9000024B09F10109A4EB0804BEF1000F18BF80
:105FA000644210F4803F02D0002C04DA01E0002C9F
:105FB00001DD20EA0B00002EC4BF599C2043DDE91F
:105FC000564E4EF82400491C262901D29945C5D3C6
:105FD0000AF1010AAA45FFF456AF002EC8BF509837
:105FE0003BDC0026002D36D94F98C0F5807A40F46E
:105FF000807E002006EB4601024601EB061B25E0F1
:1060000044094CA900F01F0851F82440012101FA6D
:1060100008F10C4217D000F001010CEB413101EB0B
:106020008B094FEA5008521C59F82840E1B201EBA5
:106030005A0101EA0E01B94288BF394624F0FF0433
:10604000214349F82810401C262801D29A42D7D370
:10605000761CAE42CDD3012050903C9A3EA941F827
:1060600022003C98401C3C900628FFF4D9AE00F07A
:106070002CB93C9936A850F82100002800F01F8167
:1060800044984F9001EBC101684600EB810000216C
:106090004E91016850914168519190F808A0417A61
:1060A0004C91817AB0F90C9082695792D0E90784BB
:1060B000C289006956904F98C1F5807602EA0107BF
:1060C00010F0010F14D04C984FF0000B002870D93D
:1060D0000122569802FA0BF1084018BF0120002156
:1060E0004D900BEB4B0000EB0B108C466390D4E013
:1060F0000020FBF716FB05464C9800FB0AF1032035
:1061000000EB410020F003024146204615F07BFFE2
:106110002846FBF706FB4C984FF0000B002848D9A7
:106120000122569802FA0BF1084018BF0120002105
:106130004D900BEB4B0000EB0B100D4659904BE0D4
:106140004A0950A801F01F0350F82220012098406E
:1061500002423ED038F9020B6D1CA0EB09034D98AA
:10616000002818BF5B4201F0010257984FEA510E18
:1061700000EB4232599802EB8000589050F82E20E4
:10618000C2F3072002F0FF0C12F4803F02D0002B74
:1061900002DB04E0002B02DDACEB060401E00CEBBB
:1061A0000604BC4206DDFF283ABF0024401C3C46E2
:1061B00007E07AE0002C04DA0028C6BF3C46401E07
:1061C000002402F4803242EA0020589A204342F828
:1061D0002E00491C262901D25545B1D34C980BF10C
:1061E000010B83459CD360E04A0950A801F01F03CE
:1061F00050F822200120984002424BD034F9020B83
:106200004D9AA0EB09000CF1010C002A18BF404286
:1062100038F9022BA2EB090218BF52420028B4BF82
:1062200043420346002AB8BF52429A4232D9579A93
:1062300001F0010302EB4333639A03EB82024B0844
:10624000CDE9583252F82330C3F30722DDB213F4FC
:10625000803F02D0002802DB03E0002801DD354446
:1062600000E0AD1BBD4205DDFF2A3ABF0025521CF0
:106270003D4606E0002D04DA002AC6BF3D46521E08
:10628000002503F4803040EA0220DDE9582328434A
:1062900043F82200491C262901D2D445A4D34C98A6
:1062A0000BF1010B8345FFF413AF4F98032826BF72
:1062B00001204E904E983EA93C9A41F822003C980D
:1062C000401C3C900628FFF4D4AE012300203EA9D8
:1062D00051F82020EAB1401C0628F9D3CBB13D98F3
:1062E0001F2811D2401C012101FA00F23D9065984F
:1062F000024209D13D98401C3D90032804D801FA80
:1063000000F265980242F5D000204490459818B1FB
:106310000BE04498401CF8E7FBF78CFD6DE4FEF7BA
:10632000C3FF459800283FF468ACFBF76FFB5D980E
:10633000FBF7C9FD5E98FBF771F96198FBF7F1F97E
:106340006098FBF7AAFB5F98FBF79CFB6298FAF753
:1063500094FF5C9830B15B9810B1FBF76BFD01E0E6
:10636000FBF72FFDFDF739FA48B15598002818BF03
:10637000FDF738FA5498002818BFFDF76FFA5A98BD
:10638000002818BFFCF7E7FF459800280CBF012044
:10639000002067B0BDE8F08F2DE9F05FADF5A85D96
:1063A0000646002001AF054607F5805807F59359CA
:1063B00000909EE0284604F0D7FB00287ED000899C
:1063C00000EA060424F0CC0030F47C4076D00F21A3
:1063D0002846FFF713F8002870D0FBF7DEFC009981
:1063E00000296CD1FBF7BBFBFF210F20FFF7B1F9B0
:1063F0000090FBF70BFB0098002877D114F0010FF9
:106400000DD0FEF7E2FF82464FF0040B3846FBF753
:1064100074FF9AF92C103A46584604F0F3FB14F036
:10642000100F0ED0FEF7D1FF82464FF0080B414609
:106430000120FBF7B6FF9AF930104246584604F0A7
:10644000E1FB14F4807F0ED0FEF7BFFF82464FF0D1
:106450000C0B49460220FBF7A4FF9AF934104A4678
:10646000584604F0CFFB009848BB24F0990030F464
:10647000794006D0FEF7C9F90090FBF7C7FA0098FB
:10648000E8B914F0020F0DD0FDF7D7FC8246FEF7F5
:106490009CFF05235FEA0A0204D090F92D101846EC
:1064A00004F0B0FB14F0200F10D0FDF741FC824641
:1064B000FEF78BFF09235FEA0A0201E018E015E00E
:1064C00004D090F93110184604F09CFB14F4007FBE
:1064D0000CD0FDF7F6FB0446FEF777FF0D232200F4
:1064E00004D090F93510184604F08CFBFFF7F5F84E
:1064F0006D1C04F035FBA842009803D900283FF436
:1065000059AF06E0002802BF01200DF5A85DBDE8E7
:10651000F09F00200DF5A85DBDE8F09F2DE9F04F3C
:106520009C48ADF50D7D0478FEF766FE012840F02D
:10653000CB8099480068B0F93610B0F9340015F0F6
:10654000B2FD14F0020F7DD00DF5007BFFF7D8F8F7
:106550003026924F4FF488784FF050094FF0FF3AB1
:10656000002578B1B0E80E108BE80E10B0E80E10E0
:106570000DF5047B8BE80E100FC80DF5087B8BE83A
:106580000F0013E0FF223021584615F05FFDCDE9E2
:106590008495CDE98265CDF82CA2CDF828A2CDF85E
:1065A00024A28695CDE9875ACDE98078DFF8F0B14D
:1065B0005846FCF78FFA8598401C859040F277701A
:1065C000FFF7EAFE012803D1FEF731FA01281FD0B8
:1065D00087980023401C87901A462121CDF81092FD
:1065E000072006F097FE00231A461946FE20009564
:1065F000FEF788FA0DF5007904F096FA90B18169FA
:106600008891C169899141698A91C0688B9011E034
:1066100014F0080F14BFA220A12084908698401C7B
:106620008690E7E7CDF82CA2CDF828A2CDF824A2D9
:10663000CDF820A2CDE98265CDE9807800214A46D7
:10664000084600E029E0D9F8083052F820C0401C84
:106650006144B0EB930FF8D34D42FF224FF4007129
:106660006846C9F80C5015F0F1FCD9F80820F9E893
:1066700004018DE82700B9E80F0004AD85E80F009C
:1066800099E80F0008AD85E80F005846FCF722FA9C
:1066900069465846FCF7C0FA0DE014F0100F0AD016
:1066A0004FF4E060FFF778FE28B900230122212192
:1066B000072006F02FFE0020FDF799FF0023224659
:1066C0004021072006F026FE0DF50D7DBDE8F04FB8
:1066D00002F052BC2F49488070472E49888070478D
:1066E00070B50126FFF70CF820B10069A12818BF8A
:1066F000A22801D0002070BD002404F031FA002847
:1067000042D9204604F030FA00281EBF058925F042
:10671000CC0030F47C4032D00F212046FEF76EFED4
:1067200068B315F0010F0AD0FBF7FBFD38B944F44C
:10673000807200232021072006F0ECFD002615F0D2
:10674000100F0BD00120FBF748FE38B944F48052FB
:1067500000232021072006F0DDFD002615F4807FB0
:106760000BD00220FBF739FE38B944F48032002305
:106770002021072006F0CEFD0026FEF7AEFF641CA8
:1067800004F0EEF9A042BCD8304670BD002070473E
:1067900000207047E8800010D48100105443524616
:1067A00000FE020070470020704710B503F007009C
:1067B000042808BFFEF7DCFD002010BD70B503F013
:1067C00007020025F84CF94B012A02D0022A14D006
:1067D00011E0052018709D60FCF77AFF22685321B4
:1067E00011702268452151702268010A9170216858
:1067F000C87020680571002070BD1A78052A13D171
:106800009A68052A28BF104607D2D4F800C01CF8A1
:1068100002C080F800C0501C9860052804D10120F7
:106820009D60087003201870012070BD2DE9F041B3
:1068300003F0070201260025DB4CDC4B012A02D0C5
:10684000022A3BD037E0052018709D60FCF740FF1E
:106850002168AC270F702268010A51702168887086
:1068600004F018F9DFF8488380B1D8F8000004F08C
:106870000DFA58B1D8F8000090F8200010F0020F7F
:1068800004D0206847702168432088702068C67053
:106890002068057104F0FEF850B1D8F8000004F04B
:1068A000F5F928B1D8F800002168007E487102E0AF
:1068B0002168FF2048710020BDE8F0811A78052A80
:1068C00012D19A68062A28BF104607D2D4F800C011
:1068D0001CF802C080F800C0501C9860062803D144
:1068E0009D600E70032018700120BDE8F08103F058
:1068F0000702022A1CBF00207047202202700120DC
:10690000087070472DE9F041A84F0D46064613F078
:10691000070F04D003F00700022808D004E012F0AB
:10692000040F1CBF0020B8700020BDE8F08102F009
:106930001DFB002814BF0124002402F01AFB0028CC
:1069400014BF0222002242EA0403B878002814BFD0
:106950000422002242EA0300307001202870BDE8C2
:10696000F08170B503F0070C0026904C8E4DBCF101
:10697000010F0AD0204613F0070F00780DD0BCF1AC
:10698000040F08BF062818D029E0A6602868067002
:10699000286846700520207021E005281FD1A068D6
:1069A000022803D22B681A54401CA060022816D17A
:1069B0000120A6600870062010E02868007855289D
:1069C0000BD128684078AC2818BFBC2805D12868AE
:1069D0000122411C062002F0AFFA032020700020A3
:1069E00070BD70B503F0070200256F4C6F4B012A94
:1069F00002D0022A24D021E0052018709D6002F008
:106A000070FA41F6E8710144B0F53C3F10D8CA78FD
:106A1000086862F31F60674A904208BF002007D1F0
:106A20000A18236812791A54401C1428F8D305E078
:106A3000002021680D54401C1428FAD3002070BD9A
:106A40001A78052A13D19A68142A28BF104607D24B
:106A5000D4F800C01CF802C080F800C0501C986038
:106A6000142804D101209D600870032018700120B3
:106A700070BD70B503F0070200254B4C4B4B012A4B
:106A800002D0022A3FD03CE0052018709D6002F041
:106A900028FA41F6E8710144B0F53C3F2BD8CA789A
:106AA000086862F31F60434A904224D12268087C40
:106AB00010702268487C50702268887C9070206832
:106AC000CA7CC27020680A7A02712268487A5071C2
:106AD0002268887A90712268C87AD0712268087D0D
:106AE00010722268487D50722268887D9072C87D3D
:106AF0002168C87205E0002021680D54401C0C2854
:106B0000FAD3002070BD1A78052A13D19A680C2A8E
:106B100028BF104607D2D4F800C01CF802C080F885
:106B200000C0501C98600C2804D101209D600870A2
:106B300003201870012070BD70B503F00702002516
:106B4000194C1A4E012A02D0022A3FD03CE003F031
:106B5000EBFF40B3D0E906212368C0681A70D4F86F
:106B600000C0130A8CF80130D4F800C0130C120EC8
:106B70008CF802302368DA702268117123680A0ADF
:106B80005A7123680A0C090E9A712268D171216822
:106B900008722268010A51722268010C9172010E7A
:106BA0002068C1720DE007E0D0E60100F880001017
:106BB000D481001034CD12AB21680D54401C0C2838
:106BC000FAD305203070B560002070BD3278052AF8
:106BD00010D1B2680C2A28BF104604D223689B5CEF
:106BE0000370501CB0600C2804D10120B5600870FF
:106BF00003203070012070BD70B503F0070200243F
:106C0000F84DF94B012A02D0022A3ED03BE0052084
:106C1000187000269C6002F064F900F50051B0F590
:106C20003C3F98BF11F0030F27D1F04A086890420B
:106C300004BF0022104620D151F82030401C1A44D5
:106C40000728F9D302B1C6B128680A7C02702A6805
:106C5000487C50702A68887C90702A68C87CD07004
:106C60002A68087D10712A68487D50712A68887DDD
:106C70009071C87D2968C87105E0002029680C540E
:106C8000401C0828FAD3002070BD1A78052A13D1B9
:106C90009A68082A28BF104607D2D5F800C01CF809
:106CA00002C080F800C0501C9860082804D1012060
:106CB0009C60087003201870012070BD2DE9F04120
:106CC00003F0070C0027C84E4FF00508BCF1010F78
:106CD0000DD013F0070F0FD03246BCF1020F12781F
:106CE00010D0BCF1040F08BF062A26D058E086F861
:106CF00000807770B76053E07270BD48B0620620C4
:106D000030704DE0052A15D1B268042A28BF10461C
:106D100009D2C2F10303D6F828C0DB002CFA03F332
:106D20000370501CB060042804D10120B7600870C3
:106D3000032030700120BDE8F08170780125002427
:106D400010F0010F11D002F0CCF8B0F53C3F23D881
:106D50006A030021B1EB900F07D252F8043B491CA3
:106D60001C44B1EB900FF8D3B5B1707810F0020F5E
:106D70000ED003F0D9FE78B182680021B1EB920FFA
:106D800006D250F8043B491C1C44B1EB920FF8D3D7
:106D9000002D18BFB46200D1B762777086F800800A
:106DA0000020BDE8F081F0B503F0070C00268D4D02
:106DB0008D4C83B0BCF1010F0ED013F0070F1DD026
:106DC000224603271278BCF1020F26D0BCF1040F33
:106DD00008BF062A36D03CE002AA01A9684602F0A4
:106DE000D9FB05202070296801980870296800984F
:106DF0004870296802988870A6602AE0A068032875
:106E000003D229680A54401CA060022821D306211D
:106E10002170032808BFA6601BE0052A0FD1A268D5
:106E2000032A28BF104604D22B689B5C0370501CB9
:106E3000A060032803D10120A6600870277003B06A
:106E40000120F0BD286882780178407802F095FB37
:106E5000277003B00020F0BD08B503F0070001283B
:106E60000AD103F017FE38B101208DF80000024668
:106E700069460D2002F060F8002008BD08B503F057
:106E8000070001280AD103F005FE38B100208DF873
:106E90000000012269460D2002F04EF8002008BDD6
:106EA00008B503F00700012809D103F0F3FD30B164
:106EB00003208DF800000122694602F03DF8002011
:106EC00008BD0020704708B503F0070001280AD16B
:106ED00003F0E0FD38B10B208DF800000122694677
:106EE000032002F029F8002008BD1FB513F0070F9A
:106EF0000ED103F0CFFD58B19DF80800F0280AD05C
:106F000003F0C8FD20B1012202A9092002F014F803
:106F100004B0002010BDFEF715FCF9E708B503F03A
:106F2000070001280AD103F0B5FD38B110208DF813
:106F3000000001226946032001F0FEFF002008BD89
:106F400070B503F00700274C274D012808D013F037
:106F5000070F12D0042804BF2878062816D01FE097
:106F60000020A86021680870216848702168887036
:106F70002168C8700520287012E0A86804280FD284
:106F800021680A54401CA860062008E003F082FD36
:106F900030B104221046216801F0CEFF0320287092
:106FA000002070BD10B503F00700012804D102F0E5
:106FB000C7FF0D4900200871002010BD10B503F077
:106FC000070C094CBCF1010F06D013F0070F11D0CC
:106FD000BCF1020F20D01DE00020A06006F091F966
:106FE000A06117E0D0E60100F88000105446495334
:106FF000EFBEADDEA068002804BF1002A06106D07D
:10700000012804D1A0691043A06106F079F9A068B5
:10701000401CA060002010BDA26812B1012A04D05B
:1070200007E0218B090A017003E0237E0370012031
:107030000870501CA060012010BD10B503F0070CB3
:10704000FE4CBCF1010F06D013F0070F09D0BCF1C4
:10705000020F18D015E00020A06006F055F9A061DD
:107060000FE0A068002804BF1002A06106D001282C
:1070700004D1A0691043A06106F049F9A068401C42
:10708000A060002010BDA26812B1012A04D007E060
:10709000218B090A017003E0237E03700120087030
:1070A000501CA060012010BD70B5064603F007001B
:1070B000E24C0D46012808BF00200DD013F0070F49
:1070C00002D002280BD008E0A068002804BF1046B8
:1070D00011F0FBFEA068401CA060002070BD11F004
:1070E000F1FE30700120287070BD70B503F0070C00
:1070F000D24D0E460446BCF1010F06D013F0070F27
:1071000007D0BCF1020F18D015E00020A860E8609D
:1071100011E0A868002804BF1002A86108D0012867
:1071200006D1A869104381B2A861E8880CF0AEFDD1
:10713000A868401CA860002070BDE86802280ED234
:10714000E8880CF0A7FDEB6882B2002B04BF100AA0
:10715000207004D0012B02D1227001203070E86829
:10716000401CE860012070BD10B403F0070CB34C64
:10717000BCF1010F08BF00200BD013F0070F03D0A4
:10718000BCF1020F09D005E0A068002808BFE2802A
:10719000401CA06010BC00207047A2681AB9A379F7
:1071A000037001200870501CA06010BC01207047C3
:1071B0002DE9F047064603F00700A04F8946012855
:1071C00008BF002039D0DFF878829E4D13F0070FFA
:1071D00002D0022835D031E0B868002808BF7A70A4
:1071E00029D0012804BF1002B86124D0022822D17E
:1071F000B8691043B8617E7884B203F04BFCD0B11B
:10720000062E18D2DFE806F00306090C1014A8F8C1
:107210000E4010E0A8F80C400DE0286884860AE0D3
:107220002868A0F80C4106E02868A0F8504002E069
:107230002868A0F85240B868401CB8600020BDE83B
:10724000F087F86802282CD297F801A0002403F0F8
:1072500021FCD8B1BAF1060F18D2DFE80AF0030614
:10726000090C1014B8F80E4010E0B8F80C400DE00E
:107270002868848E0AE02868B0F80C4106E0286887
:10728000B0F8504002E02868B0F85240F868002892
:1072900004BF200A307004D0012802D1347089F86C
:1072A0000000F868401CF8600120BDE8F0872DE977
:1072B000F0411C4615460E46074603F0EBFB80B135
:1072C0005F4814F0070F04D004F0070102290BD027
:1072D00007E0002D1ABF90F86C00C008002009F0EC
:1072E00048FC0020BDE8F08190F86C00C0083870C0
:1072F00001203070BDE8F0812DE9F0411C461546B3
:107300000F46064613F0070F08D103F0C3FB28B160
:10731000022D3CBF284607F006FB03E004F00700FF
:10732000022802D00020BDE8F08107F0F5FA3070A5
:1073300001203870BDE8F08170B503F00702002627
:10734000414C3E4D012A02D0022A15D012E006F02F
:10735000C8FB21680870FDF74FFF2168487003F0F3
:1073600011F921688870FDF74DFF2168C87005206C
:107370002870AE60002070BD2A78052A10D1AA6856
:10738000042A28BF104604D223689B5C0370501C5B
:10739000A860042804D10120AE6008700320287082
:1073A000012070BD70B503F00702274C0025234E65
:1073B000012A02D0022A4BD03FE0FEF7A1F90028B3
:1073C00028D04169FF292CBFFF21C9B22268117062
:1073D0008169FF2934BFC9B2FF2122685170C16998
:1073E000FF2934BFC9B2FF21226891702268017C55
:1073F000D170226890F820101171018C2268090A5E
:107400005171016A2268090C9171006A2168000EAD
:10741000C87111E02068057020684570206885708B
:1074200021685020C8702168FF20087121684871C8
:10743000216888712168C871B56007E0F880001084
:10744000E4F80010D4810010D0E60100002070BDE7
:10745000B268082A28BF104604D223689B5C0370D8
:10746000501CB060082802D10120B56008700120CE
:1074700070BD03F00702FC4B4FF0000C012A08BF5F
:10748000C3F808C001D0022A01D0002070479A68D2
:10749000022A3DBF80F800C0501C986010460228A8
:1074A00003D10120C3F808C00870012070472DE9FE
:1074B000F047064603F00700EB4F89464FF00008FF
:1074C000012808BFC7F8088001D0022802D0002098
:1074D000BDE8F087B86880BB0024254601F001FDB7
:1074E00000F50051A1F1180340214FF40052B0F50E
:1074F0003C3F1ED893F803A0D3F800C06AF31F6C7A
:10750000DFF868A3D44514D1001FB4EB900F07D265
:1075100052F804CB641C8CEA0505B4EB900FF7D34A
:10752000DA7D586962F31F60A84204BF8020307082
:1075300000D03170B868401CB860012803D1C7F88A
:10754000088089F800000120BDE8F0872DE9F041AE
:1075500003F007020026C64CC34D012A02D0022ABE
:1075600056D052E0FCF7B4F80520287003F092FAE8
:10757000002849D0BF4F386803F088FB002843D06B
:107580000CF063FB80460CF064FB39680A7E12F055
:10759000040F11D0C98A2268090A1170396822685B
:1075A000897D517039682268898A090A9170396821
:1075B0002268097DD17010E0898A2268090A117059
:1075C00039682268097D517039682268C98A090AB8
:1075D000917039682268897DD17022684FEA18213C
:1075E0001171216881F805802268010A9171216872
:1075F000C87138682268817C11722268017C5172DE
:10760000008B2168000A8872AE600020BDE8F0811E
:107610002A78052A10D1AA680B2A28BF104604D25E
:1076200023689B5C0370501CA8600B2804D10120C8
:10763000AE600870032028700120BDE8F0812DE9BC
:10764000F04703F007020026894D874B012A02D03C
:10765000022A5DD059E00520187000249E6001F0D8
:1076600040FC00F50053B0F53C3F98BF13F0030F0A
:1076700045D1814A1968914204BF0022114608D1C0
:1076800053F821C0491C62440729F9D3002A08BFD6
:1076900001249F7C93F8138084B341F6E871014480
:1076A000B0F53C3F07D8CA78086862F31F606F4A9C
:1076B000904208BF012491F8129091F813A0002C79
:1076C00008BF002014D003F02FFA2968806981F8E0
:1076D0000090296881F801A02A68010C000E9170C1
:1076E0002968C87028680771286880F805800CE050
:1076F00029680E54401C0628FAD306E0FFE7002054
:1077000029680E54401C0628FAD30020BDE8F087F3
:107710001A78052A13D19A68072A28BF104607D27B
:10772000D5F800C01CF802C080F800C0501C98605A
:10773000072804D101209E600870032018700120E2
:10774000BDE8F08710B503F0070C474CBCF1010F02
:1077500006D013F0070F0AD0BCF1020F1AD017E0C1
:107760000020A060E0600CF0E9FAA06110E0A068E1
:10777000002804BF1002A06107D0012805D1A0692C
:107780001043A06180B20CF0D6FAA068401CA06043
:10779000002010BDE268022A0BD212B1012A04D0E7
:1077A00007E0218B090A017003E0237E03700120AA
:1077B0000870501CE060012010BD70B503F0070197
:1077C0000026294D0446012908BFEE6201D0022996
:1077D00001D0002070BDE86A002804BF274814F0DB
:1077E00067FCE96A082928BF267002D22348405C5A
:1077F0002070481CE862012070BD2DE9F04103F0C3
:1078000007010026184D0746012908BFEE6201D086
:10781000022902D00020BDE8F08195F82C0000F08C
:1078200007042879204304D1144814F041FC0120B6
:107830002871052C28BF2E711048005D3870E86A49
:10784000401CE8620120BDE8F08170B5044603F0F9
:1078500007000D4602281CBF002070BD14F02DFC4F
:1078600020700120287070BDF880001034CD12AB5C
:10787000D0E60100D48100105446495328810010FD
:1078800070B503F007020025F94C012A02D0022A44
:1078900012D00FE005202070002211461046A5608E
:1078A00001F078FE4FF6FF7101EA4000206101F01F
:1078B00084FE6062002070BD2278052A17D1D4F8BA
:1078C00010C0A268624528BF104607D212F0010F0F
:1078D0001CBF637803700CD0501CA060604506D1BB
:1078E0000120A56008700320207001F073FE0120C4
:1078F00070BD666A22F00103F35A1E0A06706370B7
:10790000EAE770B503F007020025D94C012A02D03E
:10791000022A11D00EE0D74805220068B0F91210F3
:10792000B0F91000227008444000A560206101F009
:10793000C4FF6062002070BD2278052A17D1D4F8F8
:1079400010C0A268624528BF104607D212F0010F8E
:107950001CBF637803700CD0501CA060604506D13A
:107960000120A56008700320207001F0B4FF012001
:1079700070BD666A22F00103F35A1E0A0670637036
:10798000EAE7F8B503F007020025B94C012A02D056
:10799000022A13D010E000216A46084601F0FAFDE1
:1079A00005202070A56000984FF6FF7101EA4000A5
:1079B000206102F0B4F860620020F8BD2278052A48
:1079C00017D1D4F810C0A268624528BF104607D26C
:1079D00012F0010F1CBF637803700CD0501CA06024
:1079E000604506D10120A56008700320207002F0D8
:1079F000A4F80120F8BD666A22F00103F35A1E0ABA
:107A000006706370EAE77FB51C460E46054613F024
:107A1000070F08D103F03EF828B1012202A90C207B
:107A200001F08AFA03E004F00700022802D004B053
:107A3000002070BD06F055F828700120307004B0A9
:107A400070BD7FB51C460E46054613F0070F08D1E2
:107A500003F020F828B1012202A90F2001F06CFAEE
:107A600003E004F00700022802D004B0002070BD3B
:107A700011F01EF800F00F0040F0100028700120F7
:107A8000307004B070BD10B503F00702784C012AC5
:107A900002D0022A0DD00AE003F093FA0021E0613F
:107AA00000281ABF4FF4056020622162A160002007
:107AB00010BD236AA2689A4228BF104607D2D4F8A4
:107AC0001CC01CF802C080F800C0501CA060984286
:107AD00004BF01200870012010BD10B413F0070F7F
:107AE0004FF0402C04D003F00702022A13D00FE01D
:107AF000012A04BFDCF8140040F0010006D0002A7F
:107B000004BFDCF8140020F0010001D1CCF814000F
:107B100010BC00207047DCF8142002F00102027053
:107B20000120087010BC704770B514460E4605461B
:107B300013F0070F04D003F00700022813D010E061
:107B4000002C14BF0120002002F0ECF94CB14FF0E2
:107B50004020016B21F4405141F4BE0141F020412D
:107B60000163002070BD02F0E4F9002814BF012277
:107B700000222A700120307070BD70B503F007003C
:107B80003B4D1446012808BF002015D013F0070F05
:107B900013D1A868002808BF6A700BD0012809D14A
:107BA0006878FBF703F96878334900EA04020A634E
:107BB000A0434863A868401CA860002070BD70B551
:107BC000044603F007000D4602281CBF002070BDCC
:107BD00005F014FF20700120287070BD70B50D46AF
:107BE000044613F0070F04D003F00700022805D065
:107BF00002E0104605F00AFF002070BD05F009FF05
:107C000020700120287070BD70B50D46044613F039
:107C1000070F04D003F00700022805D002E0104649
:107C2000F9F7BCF8002070BDF9F7BBF8207001200F
:107C3000287070BD10B403F007020024DFF830C0D4
:107C4000012A08BFCCF808400FD0022A03D013F055
:107C5000070F05D009E004700120087010BC7047C0
:107C6000DCF80800401CCCF8080010BC002070476D
:107C7000F8800010D48100100010004070B5044658
:107C800003F00700FE4D0E46012804BF0020A86047
:107C900014D013F0070F02D0022811D00EE0A8680C
:107CA000F84904283CBF0B681A54401CA8600428FB
:107CB00004D104220968112001F03EF9002070BDB2
:107CC0000AF064F9AA68002A04BF000E20700FD0E1
:107CD000012A08BF000C06D0022A08BF000A02D001
:107CE000032A02D004E0207002E0207001203070EE
:107CF000501CA860012070BD70B503F0070CE04D6A
:107D00000E460446BCF1010F04BF0020A86015D048
:107D100013F0070F03D0BCF1020F11D00EE0A868DA
:107D2000D84902283CBF0B681A54401CA86002289E
:107D300004D102220968122001F0FEF8002070BD73
:107D40000AF0FCF8AA68002A04BF000A207004D0D8
:107D5000012A02D1207001203070501CA86001203F
:107D600070BD70B5044603F00700C54D0E460128EE
:107D700004BF0020A86014D013F0070F02D002281F
:107D800011D00EE0A868BF4904283CBF0B681A5404
:107D9000401CA860042804D104220968132001F0C3
:107DA000CBF8002070BD0AF024F9AA68002A04BFAD
:107DB000000E20700FD0012A08BF000C06D0022A46
:107DC00008BF000A02D0032A02D004E0207002E0BB
:107DD000207001203070501CA860012070BD70B56B
:107DE000044603F00700A64D0E46012804BF0020FC
:107DF000A86037D013F0070F02D0022834D031E04A
:107E0000A868A04C002804BF21680A70216809787E
:107E1000012901D039B11BE0002818BF04283CBF5C
:107E200021680A5414E00AF002F921680009487038
:107E30000AF0EEF8C0F303260AF0F9F8216846EAE2
:107E4000001088700AF0E4F82168C8700320A86068
:107E5000A868401CA860042804D1042214202168CA
:107E600001F06AF8002070BD0AF0EDF8AA68002A57
:107E700004BF000E20700FD0012A08BF000C06D0EE
:107E8000022A08BF000A02D0032A02D004E02070B0
:107E900002E0207001203070501CA860012070BDED
:107EA00010B503F00702764C012A02D0022A27D02F
:107EB00024E003F086F80023002804BFE361236276
:107EC0001BD000F15001E1614168B1F5887F90F865
:107ED00020100CD390F8212001EB020C01FB02C111
:107EE00090F8222090F823001044084404E090F811
:107EF00022000A1801FB00202062A360002010BDB0
:107F0000236AA2689A4228BF104607D2D4F81CC040
:107F10001CF802C080F800C0501CA060984204BF4A
:107F200001200870012010BD03F00702012A02D0D1
:107F3000022A05D002E052490020886000207047E4
:107F4000012202700A701046704710B513F0070F37
:107F500004D003F00702022A05D002E0104601F027
:107F600046FB002010BD484A1278027001200870BC
:107F700010BD10B513F0070F04D003F00702022A5A
:107F800005D002E0104601F0CBFC002010BD3F4AB6
:107F9000127802700120087010BD10B513F0070FA1
:107FA00004D003F00702022A05D002E0104601F0D7
:107FB000D1FD002010BD364A1278027001200870F1
:107FC00010BD1FB513F0070F07D102F063FD20B1FC
:107FD000012202A90B2000F0AFFF04B0002010BD69
:107FE00070B503F00700264C1546012804BF002099
:107FF000A06024D013F0070F21D102F04BFDF0B1A7
:10800000A068204E03283CBF31680D54401CA0607E
:10801000032814D1F9F7BBFD3068B0F8010045BA68
:10802000F9F7F2FC040018BFF9F73DFF3068294664
:108030000078F9F741F9002C18BFF9F737FF002055
:1080400070BD70B503F007000D4C1646012804BF43
:108050000020A06034D013F0070F31D102F01AFDD8
:1080600070B3A068074D02283CBF29680E54401C1D
:10807000A060022824D1F9F78AFDF9F7C5FC09E0D0
:10808000F8800010D0E601003D8100104281001010
:1080900047810010040018BFF9F705FF2868007831
:1080A00080B129684978F9F786F92868417800781D
:1080B00040F01000F9F77FF9002C18BFF9F7F6FE31
:1080C000002070BD286841780020F3E77FB51C468A
:1080D0000E46054613F0070F08D102F0DBFC28B16D
:1080E000012202A9182000F027FF03E004F0070096
:1080F000022802D004B0002070BD05F0CAFC0028A0
:1081000014BF012200222A700120307004B070BD1B
:108110007FB51C460E46054613F0070F08D102F046
:10812000B9FC28B1012202A9192000F005FF03E0E3
:1081300004F00700022802D004B0002070BD05F052
:1081400095FC28700120307004B070BD70B503F04C
:108150000700FB4C1546012804BF0020A06019D081
:1081600013F0070F16D102F095FC98B1A068F549FD
:1081700003283CBF0A681554401CA060032809D19D
:1081800008680968B0F80100097840BA00B219B16E
:10819000FEF7A3FA002070BDFEF79CFAFAE770B56F
:1081A00003F00700E64C1546012804BF0020A0603C
:1081B00017D013F0070F14D102F06CFC88B1A0683F
:1081C000E04B03283CBF19680D54401CA0600328F5
:1081D00007D11868B0F8010041BA18680078FAF7BA
:1081E0005CF9002070BD10B503F00702D44C012AE1
:1081F00002D0022A07D004E00020A060FBF759F962
:10820000A061002010BDA268042A07D2C2F10303B6
:10821000D4F818C0DB002CFA03F30370501CA060E4
:10822000042804BF01200870012010BD10B503F020
:108230000700012807D102F02DFC20B100221146D1
:108240001D2000F079FE002010BD2DE9F04103F063
:108250000705BB4E174688460446012D04BF002083
:10826000B0601BD013F0070F16D102F013FC98B1C9
:10827000B068B44B03283CBF19680F54401CB06071
:1082800003280BD1186890F9022090F9011090F999
:108290000000FCF76AFC01E0022D02D00020BDE8DE
:1082A000F081B06820B1012807D002280AD010E080
:1082B0001420FCF701FC20700BE01520FCF7FCFB00
:1082C000207006E01620FCF7F7FB2070012088F8EC
:1082D0000000B068401CB0600120BDE8F08170B5BE
:1082E0000D46044613F0070F04D003F007000228E0
:1082F00005D002E0924900208860002070BD002077
:10830000FCF7DAFB20700120287070BD70B503F017
:10831000070C00268B4C8A4DBCF1010F06D013F0E0
:10832000070F0CD0BCF1020F1FD01CE005F0E8FCD9
:10833000AE60216808702168000A487013E0A868E0
:10834000022803D221680A54401CA86002280AD1DE
:10835000AE602068007810F0010F04D002221A20CD
:10836000216800F0E9FD002070BDAA68022A28BF3C
:10837000104604D223689B5C0370501CA86002283E
:1083800004D10120AE60087003202870012070BD68
:108390002DE9F0411C4617460E46054613F0070F1F
:1083A00006D102F077FB18B138460BF0B9FC03E0B8
:1083B00004F00700022802D00020BDE8F0810BF095
:1083C0004CFC287001203070BDE8F0817FB51C4660
:1083D0000E46054613F0070F08D102F05BFB28B1EB
:1083E000012202A91F2000F0A7FD03E004F007000E
:1083F000022802D004B0002070BD0BF099FC287058
:108400000120307004B070BD7FB51C460E46054695
:1084100013F0070F08D102F03DFB28B1012202A999
:10842000212000F089FD03E004F00700022802D0BB
:1084300004B0002070BD44480078287001203070DE
:1084400004B070BD7FB51C460E46054613F0070FFD
:108450000ED102F01FFB58B19DF80800002818BF8C
:108460000BF06FFC012202A91E2000F065FD03E065
:1084700004F00700022802D004B0002070BD0BF009
:1084800063FC28700120307004B070BD002070477C
:108490002DE9FF412A4E1C460F46054613F0070FF3
:1084A0001CD102F0F7FAC8B19DF80800002818BFE7
:1084B000012802D0022807D014E0F070012202A99E
:1084C000082000F039FD0DE0F07004208DF8080060
:1084D000012202A9082000F02FFD03E004F00700AC
:1084E000022803D004B00020BDE8F081F0782870A5
:1084F0000120387004B0BDE8F0817FB51C460D4600
:10850000064613F0070F08D102F0C4FA28B1012281
:1085100002A9082000F010FD03E004F00700022883
:1085200002D004B0002070BDFCF766FE801E052856
:1085300014D2DFE800F0030D0F0B110000200EE055
:10854000F8800010D0E6010030810010012006E024
:10855000022004E0032002E0042000E0FF2030704D
:108560000120287004B070BD2DE9F0411C4617466B
:108570000E46054613F0070F0BD102F08BFA40B1FF
:10858000384605F035FA00221146012000F0D4FCEF
:1085900003E004F00700022802D00020BDE8F081CB
:1085A00005F029FA287001203070BDE8F08110B57F
:1085B000104613F0070F08BF05F081FA002010BD28
:1085C00010B5104613F0070F08BF05F07FFA002022
:1085D00010BD70B5044603F007000D4602281CBF0D
:1085E000002070BD05F07AFA20700120287070BD5F
:1085F00003F0070230B4FF4B4FF0000C012A05D006
:10860000022A04BF1A78022A0BD01EE0022018703A
:10861000F948C3F808C06FF07F410068081A9861F4
:1086200013E09A68042A28BF104606D29D69D40038
:1086300025FA04F40470501C9860042805D1012028
:10864000C3F808C008700320187030BC01207047C0
:1086500013F0070F04BFE94802700020704710B5FF
:1086600003F00700E349012804BF0020886013D00D
:1086700013F0070F10D18868E14B04283CBFD3F8F2
:1086800000C00CF80020401C8860042804D104229B
:108690001020196800F050FC002010BD2DE9F047B3
:1086A000164603F007020024D24F012A04BFBC6023
:1086B000FC6064D0DFF84C8313F0070F07D0022A68
:1086C00033D0042A04BF387806284FD058E0BD685C
:1086D000002D08BFFE6125D0012D06D0D7F81090DF
:1086E000AC1E4C4516D284B908E0701C3861F9699B
:1086F0000844B0F5007F88BF3C6113E04FF400727E
:108700004FF43E31C04813F06FFCBD49F869096869
:1087100020440E54601C484504D1BB48C0F8FC817D
:1087200006203870681CB8602AE0FF2202703B699E
:10873000CBB1D7F81CC0FA689444BCF5007F10D2C6
:10874000B24D2D68454518BF047005D10CF53C3C71
:108750009CF800C880F800C0501C984204BF01205B
:108760000870501CF8600120BDE8F0874FF43E30DF
:10877000FAF7B0F9A4494FF43E30FAF74DFA3C70DD
:108780000020BDE8F08770B503F00700994C15464E
:10879000012804BF0020A06014D013F0070F11D1EE
:1087A00002F078F970B1A068954902283CBF0A68C8
:1087B0001554401CA060022804D10222096805203B
:1087C00000F0BAFB002070BD2DE9F041054603F032
:1087D00007008B4C874E0F4601280AD013F0070F75
:1087E00014D002281BD0042804BF3078062834D0C7
:1087F0003FE00020B060216808702168487021685F
:1088000088702168C8700520307032E0B068042894
:108810002FD221680A54401CB060062028E0B068BE
:1088200060B905F0DCF8216808702268010A51700F
:108830002268010C000E91702168C870B06804288D
:108840003ABF2168095CFF21297024BF01213970DA
:10885000401CB0600120BDE8F08102F01BF940B17E
:108860002068C178006861F31F6005F0B3F8032049
:1088700030700020BDE8F08170B503F007015D4C59
:10888000064601290BD05E4D13F0070F0CD00229CC
:1088900014D0042904BF207806281DD025E000202C
:1088A000A0600520207020E0A068B0F5007F1CD2F9
:1088B00029680A54401CA060062015E0A06818B979
:1088C0000021286813F0FEFB2868A168405C307026
:1088D000481CA060012070BD02F0DCF828B1A1683E
:1088E000286813F0F4FB03202070002070BD1FB532
:1088F00013F0070F04D1012202A91B2000F01CFB7A
:1089000004B0002010BD03F007003A49012806D04A
:1089100013F0070F04BF0878012806D014E00120E7
:1089200008700020886048610DE08868042805D23E
:108930004B69401C42EA03224A618860042803D143
:10894000032008704869C8610020704703F00700E1
:10895000DFF8A0C0012807D013F0070F04BF9CF870
:108960000000022809D01EE002208CF80000002040
:10897000CCF80800CCF8180015E0DCF80800022854
:1089800008D2DCF81810401C42EA0121CCF818107B
:10899000CCF80800022806D1DCF81800CCF820003A
:1089A00003208CF800000020704770B403F0070229
:1089B0000025104C012A02D0022A06D002E0022033
:1089C0002070A56070BC002070472278022A2BD14D
:1089D000D4F820C0A268624528BF10461DD212F00C
:1089E000030F04D1E36953F8046BC4E90663237EE3
:1089F00003700DE0F88000108880001020800010C7
:108A0000D0E60100554E564D90A50010FCF902002D
:108A1000A069000AA061501CA060604504D101203B
:108A2000A56008700320207070BC0120704770B5ED
:108A300003F007000025FF4C0E46012806D013F076
:108A4000070F04BF2078022805D02BE002202070F9
:108A5000A560A56126E0216AA068884219D2A169B3
:108A6000090A41EA0262401CA26110F0030FA060F3
:108A70000FD1E069B0F5443F28BF026006D2B0F5DF
:108A8000005F03D30422EC49FAF71AF9E069001DEC
:108A9000E061216AA068884204D10120A56030709D
:108AA00003202070002070BD30B403F007040025BF
:108AB000DFF880C3012C08BFCCF8085035D013F084
:108AC000070F02D0022C33D02FE0042A08BF4FF446
:108AD000403028D013DC002A08BF4FF4005022D0C9
:108AE000012A08BF4FF443301DD0022A08BF4FF4BB
:108AF0001C3018D0032A08BFD04814D010E0052A33
:108B000008BF4FF43E300ED0CD48102A00680AD07E
:108B1000112A08BFCB4806D0202A08BFB43002D0A3
:108B2000CCF8145001E0CCF8140030BC00207047A1
:108B3000DCF80820042A07D2C2F10303DCF8144051
:108B4000DB0024FA03F30370501CCCF8080004285F
:108B500024BF01200870012030BC704770B403F0BE
:108B6000070CB44DBCF1010F07D0B74C13F0070F41
:108B700007D0BCF1020F21D01DE00020A860E86002
:108B800019E0A86805283CBF21680A54042810D1C0
:108B900023682268D4F800C0D3F8013069691278DC
:108BA0001BBA9CF804C023F0FF0343EA0C0341F80E
:108BB0002230401CA86070BC00207047EB6873B185
:108BC000042B07D22268032B1A445278027004BF88
:108BD00001200870581CE86070BC012070472268B2
:108BE000D5F814C012785CF8222026684FEA126C7F
:108BF00086F801C026684FEA124C86F802C0266843
:108C00004FEA122C86F803C0D4F800C08CF8042078
:108C1000D8E710B503F00700012804D1002211465F
:108C20000E2000F089F9002010BD2DE9F04103F07D
:108C30000704804E174688460546012C04BF0020D5
:108C4000B06017D013F0070F12D101F023FF78B1F5
:108C5000B0687D4902283CBF0A681754401CB060C8
:108C6000022807D102220968072000F065F901E017
:108C7000022C02D00020BDE8F081B26812B1012AB6
:108C800004D009E0FCF7B8FA287005E0FCF7BAFA5E
:108C90002870012088F80000B068401CB0600120F6
:108CA000BDE8F08170B503F007000025614C012894
:108CB00008D013F0070F0BD0042804BF2078062833
:108CC00025D02DE06561A5616570A560257027E060
:108CD000A068022807D2616942EA012161616178D6
:108CE0001144617010E0042807D2A16942EA012111
:108CF000A16161781144617006E0052804D26178B1
:108D00008A4204BF06212170401CA06008E0D4E91B
:108D1000050101F0F9F9002804BF0120A0702570B9
:108D2000002070BD10B5434C13F0070F07D003F0BF
:108D30000700042804BF2078062822D02BE0A06872
:108D4000022807D2616942EA012161616178114418
:108D5000617013E03D49091808D23B490968014494
:108D600001F8022C61781144617007E03849091854
:108D700004D261788A4204BF06212170401CA060A1
:108D800009E03449606901F0E1F9002804BF0120DD
:108D9000A07000202070002010BD03F0070CBCF173
:108DA000010F00D0BEE72349002048614870886069
:108DB0000870704730B403F007050024DFF874C072
:108DC000012D07D013F0070F0DD0022D50D0042D28
:108DD00068D083E0CCF81440CCF81840CCF80840B8
:108DE0008CF800407AE0DCF8080002280BD2DCF8AE
:108DF000141042EA0121CCF814109CF8011011441F
:108E00008CF801102DE004282BD2DCF81810032870
:108E100042EA0121CCF818109CF801301A448CF871
:108E200001201ED106228CF80020DCF8142011430A
:108E300012E00000F88000101081001000FE020017
:108E4000D4810010E4F80010D0E60100FEFDFFFF21
:108E5000FDFDFFFF90A5001004BF4FF4C471CCF8D6
:108E600018102849401CCCF82810CCF8080035E030
:108E7000DCF80820042A28BF10460AD2C2F10303F6
:108E8000DCF82850DB0025FA03F30370501CCCF803
:108E90000800042803D10120CCF80840087030BC39
:108EA000012070479CF80000062815D1DCF814005A
:108EB00000224102DCF8180043021046B2EB930F87
:108EC00006D251F8045B401C2A44B0EB930FF8D350
:108ED000CCF828208CF80040CCF8084030BC0020AA
:108EE00070474FF443300168880A424211EB8222F6
:108EF00018BF401C404201EB8000C01C20F0030062
:108F000070470000EFBEADDEF7480022427082706D
:108F1000C270427182710271DFF8D0C3114601EB59
:108F2000410300200CEB43031A54401C0628FBD3DA
:108F3000491C2029F3D3704713F0CEB82DE9F04136
:108F400015460E460746FAF7C9F900F0080408204E
:108F5000FAF7BFF92A463146384613F0BDF8054600
:108F60002046FAF7B1F92846BDE8F081DE48C0781E
:108F70007047DD4880787047DB4900208870704773
:108F8000D9490820C871704770B50026F8F708FF66
:108F9000044610F00F0531D02846F8F704FF012DE4
:108FA00018D0FCF72FF944EA00640023224603217D
:108FB000072004F0AFF914F0060F1FD00126FCF7CC
:108FC0001BF9044604F06FFD0546022C18BF052C62
:108FD00009D013E0FCF710F9C349CA79904218BFD1
:108FE000C871DED1E7E70120FBF701FB022D05D0B8
:108FF000022C4FF0020003D001F0D8F8304670BDCB
:1090000004F04CFDFAE72DE9F84F0027FAF7D3FDFD
:1090100004F095FD002818BF0127FCF7EDF80228A1
:1090200004D101F003FD002818BF0127FFF7ACFFB2
:10903000002818BF0127AC4EF078002800F04F82BE
:10904000B0686D464FF0FF344FF0000838B1B26899
:1090500000230121084604F05DF9C6F80880FAF7FC
:109060003DF900F0080A0820FAF733F93079DFF803
:109070007CB2F0B1B07900EB4001401CC0B20BEB08
:109080004101B071202828BF86F806803079401E43
:1090900030714C7891F800900020002C05DD0A1802
:1090A00092782A54401C8442F9DC81F8008081F8CF
:1090B00001805046FAF708F9002CC0F2018209F04D
:1090C000FF000024222880F0BD81DFE800F0C231DB
:1090D000F51A24341140F647C27E8499DA89F3F2F6
:1090E000F1F0EFC2C2C2AEBEC3C8C2EEEDECC2EB3D
:1090F0009DF80000AC280CBF01200220FCF740F9CD
:1091000016E09DF800100120FCF78BF80120B070EC
:10911000044600F097B99DF80310009861F31F60B2
:1091200001F04CFF01210320FCF77BF80120B07017
:10913000012400F087B9BDF8000040BA04F052FCE9
:1091400002210320FCF76DF80120B070F0E79DF8D4
:1091500001109DF80000FCF764F8E9E74FF0010A00
:1091600086F802A0707860BBF8F70FFE48B39DF850
:10917000005086F801A015F0040F18BFFDF706FB9C
:1091800015F0020F07D0FF210F20FCF7E2FAFBF7E2
:109190003CFB45F0010515F0010F10D0FCF72CF851
:1091A000022802D104F07FFC48B1FCF725F805281D
:1091B00002D101F006F810B10020FBF713FB86F88E
:1091C000018086F8028000F03DB99DF80000401E45
:1091D00001F062FAACE79DF8000004F085FCA7E717
:1091E0009DF8000000F00F000FF065FC9DF80000F6
:1091F00010F00F0018BF01200FF060FC00F022B942
:109200009DF8000060B1FBF7F7FF022818BF0124AA
:1092100004F04FFC01460220FCF703F800F012B9FD
:1092200000210620FBF7FDFF82E79DF800000028E3
:1092300018BF012004F023FC9DF80000002818BF8F
:10924000012000F0A9FF00F0FDB89DF8000004F037
:1092500002FCF7E0BDF8000004F0FCFC68E79DF8B4
:10926000000020B101284DD0022805D0EAE04FF4DB
:109270004330F9F72FFCE5E001F04FFC002104201A
:10928000D0E7FAF72BF800F008040820FAF721F8E5
:109290003079002808BF86F803802046FAF714F8D2
:1092A0000121BEE7A3E082E074E02CE05AE04BE04D
:1092B00044E02BE01CE000E075E09DF80000012890
:1092C00004BF02210520ADD0022804BF00210320E5
:1092D000A8D0032804BF00210420A3D004281CBF69
:1092E000022108469CD09DE73081001090A7001015
:1092F0009DF80300009A002360F31F62622107209B
:1093000004F008F89EE0FBF75EFC11E79DF8000012
:109310009DF80110000140EA111008F01EFE9DF8B2
:1093200001109DF8020001F00F0140EA012008F051
:109330001AFE9DF8030008F022FE83E0BDF800004D
:1093400040BA08F0FEFD7DE09DF8000008F02AFE1E
:109350009DF8010008F035FEBDF8020040BA08F0A3
:109360003FFE6FE09DF8000008F04FFE9DF8010001
:109370009DF80210000140EA111008F05BFE9DF814
:1093800002109DF8030001F00F0140EA012008F0EF
:1093900042FE57E09DF800000AF0D3FC9DF8000063
:1093A00000287FF4C5AE0020FBF721F9C0E60AF0E3
:1093B000BFFC05469DF8004004F0A2FC012C0AD039
:1093C000022C08BF40F4807005D0042C14BF082C78
:1093D00040F4007001D104F010FC20460AF0A3FC18
:1093E000082D12BF082C022004F093FBA0E69DF884
:1093F0000050F6F7A4FF027815F0010F114614BFD4
:1094000041F0020121F00201337814BF43F002035E
:1094100023F00203337015F0020F14BF41F0040172
:1094200021F00401337814BF43F0040323F0040354
:109430003370914206D0017000220123114610467C
:10944000F7F733F80CB101273AE0B0686D464FF0FA
:10945000FF3438B1B26800230121084603F05AFFF7
:10946000C6F80880F9F73AFF00F0080A0820F9F773
:1094700030FF3079F0B1B07900EB4001401CC0B250
:109480000BEB4101B071202828BF86F806803079A7
:10949000401E30714C7891F800900020002C05DDC2
:1094A0000A1892782A54401C8442F9DC81F8008022
:1094B00081F801805046F9F707FF002CBFF6FFAD99
:1094C000F9F70CFF00F008040820F9F702FF3179E2
:1094D000002908BF86F803802046F9F7F5FE002F23
:1094E00014BF01200020BDE8F88F000002460020D4
:1094F000022928BF704772B101EB4103C3EB411150
:10950000012A08BFFA4803D0022A0CBFF948704765
:1095100000EB8100704740F2DB104843F64901EB55
:109520008000704770B5F9F7D9FE00F008060820F2
:10953000F9F7CFFEF14C00256078FF2806D240F6FF
:10954000D861ED4812F055FDA570E570A079FF28AF
:1095500005D2E821E64812F04CFDE5712572E07A6B
:10956000FF2805D2E821E34812F043FD2573657317
:109570003046BDE87040F9F7A7BEDFF884C300FBB2
:1095800001F31CEB030C88BF7047DC4B9A61C3E905
:1095900004017047DFF864C30028DCF8103018BFFE
:1095A0000360D6480029406918BF0860002A1CBF24
:1095B000DCF81810116058437047D0480121017140
:1095C000007840F2DB1180F001004843CA4901EB0A
:1095D00080007047C9488278002132B1C27822B930
:1095E000027882F001020270817001717047C349F4
:1095F0001E284A78487008BF002003D01F2808BFE3
:10960000012000D1087010467047BC48007840F235
:10961000DB1180F001004843B74901EB800070473F
:10962000F0B4B64E96F800C040F2DB140CFB04FC1C
:10963000B14C356904EB8C0C03FB05F40CEB440CCA
:109640008D4234BF2C460C467669F31A934238BFDC
:109650001A460026002A9CBFF0BC70470023002C4D
:1096600006D930F813702CF813705B1C9C42F8D8A4
:10967000761C0CEB450C00EB41009642EED3F0BC9F
:1096800070472DE9F0419D4F14468C4601467A788B
:1096900006981D468A4218BFBDE8F0810121F97085
:1096A000012802D0022824D029E0387840F2DB11CA
:1096B000484391493E6901EB8001A64234BF3246DE
:1096C00022467869A84238BF05460023002D16D9E6
:1096D0000020002A06D91CF8007021F81070401CE8
:1096E0008242F8D85B1C01EB4601A444AB42EFD3A5
:1096F00005E000232A4621466046FFF791FFBDE8BA
:10970000F04100F0A1BB002808BF70477B497D4BAA
:109710004A787D491B78002A097818BF022A05D0AB
:10972000042A18BF092A01D0012279E7774A127862
:10973000012A84BF764A1378012200F09FBB2DE9ED
:10974000F04FDFF8B8A183B001218AF80310714906
:109750006E4C6F4D0F786B490E789AF801101129F5
:1097600030D00EDC002918BF02291DD0042918BFF3
:10977000092919D098B1002332463946FFF750FF26
:109780000DE0122918BF13291CD0212918BF222946
:10979000F0D120B10023B21C3946FFF741FF03B0DE
:1097A000BDE8F04F00F050BB2178012902D95A4999
:1097B0002E780F780028F2D000233246394600F088
:1097C0005DFBECE7F8F7E3F9F8F71EF900900028E5
:1097D00018BFF8F768FB2078012888BF2E78F8F7C3
:1097E000DCFA10F0040F18BF761CDFF830919AF8FD
:1097F0000100A0F111089AF8000040F2DB11484383
:109800003D4901EB8004DAF81000B84238BF074642
:10981000DAF81400B04238BF0646F8F78DFB019025
:109820000020F8F7A7FE0025002E39DD4FF0000AD2
:10983000002FC4BF05EB450000EB051B29DD019897
:1098400010F90A00262824BF002024F81A001CD290
:1098500000F0010109EB413100EBD07001EB8B010D
:109860004010B8F1000F51F820104FF0FF301DD01C
:10987000B8F1010F08BFC8B205D0B8F1020F04BF9C
:109880000846F8F77DFE24F81A000AF1010ABA45E5
:10989000D5DB1A486D1CB542006904EB4004C5DBFA
:1098A0000098002818BFF8F701FB78E711F4803F13
:1098B000C1F3072018BF4042E5E71048012141727B
:1098C000407980F0010000EB4001C1EB40100849F5
:1098D00001EB800070470948C279002132B1027A59
:1098E00022B9427982F001024271C171417270471E
:1098F00028B7001010B8001050A800103C810010CC
:109900004AFCFFFFCD800010D3800010CE800010F5
:10991000D0800010CC800010CF800010008000307C
:10992000F9491E288A79887108BF002003D01F28B2
:1099300008BF012000D1487110467047F2484079B5
:1099400080F0010000EB4001C1EB4010EF4901EB5A
:10995000800070472DE9F04FED4985B0012291F864
:109960000080EC4991F80090E7490A728979E74C48
:1099700011291CBF1229132929D090B1E249497934
:1099800001EB4102C2EB411104EB8102002119EB12
:10999000080306D030F811C022F811C0491C8B42D0
:1099A000F8D8F9F79BFC00F008050820F9F791FCBE
:1099B000D54C607A002818BF01217CD0E17128467F
:1099C000F9F782FC0020207205B0BDE8F08FF8F7AF
:1099D000DEF8F8F719F80190002818BFF8F763FAD5
:1099E000C9488179A1F11105C1690091407900EB65
:1099F0004001C1EB401004EB8006F7F7E6F9C64FD3
:109A0000C6494FF0110A002804BF8B46012004D03C
:109A1000BB4650460F464FF0010AF8F7ABFDF8F78A
:109A200089FA00240390B9F1000F28D900984C213D
:109A30004843029003980057262824BF002026F8A8
:109A4000140019D200F001010BEB413200EBD07091
:109A50000299401001EB8000002D11584FF0FF30AB
:109A600049D0012D08BFC8B204D0022D04BF08465A
:109A7000F8F786FD26F81400641C4C45DAD306EB93
:109A800049065046F8F776FDF8F756FA0024824664
:109A9000B8F1000F29D900984C2100FB01F94FF0D3
:109AA000000B1AF90400262828BF26F814B019D292
:109AB00000F0010100E02CE000EBD070401007EB5B
:109AC000413109EB800009584FF0FF30D5B1012D2D
:109AD00008BFC8B204D0022D04BF0846F8F750FDF5
:109AE00026F81400641C4445DBD30198002818BFF5
:109AF000F8F7DCF955E711F4803FC1F3072018BFF0
:109B00004042B7E711F4803FC1F3072018BF40423D
:109B1000E6E7607980F00100607100214EE77A4845
:109B200001218173807A80F0010000EB4001C1EBDC
:109B300040107B4901EB800070477348027B002195
:109B400032B1427B22B9827A82F0010282720173C1
:109B5000817370476C491E28CA7AC87208BF0020FA
:109B600003D01F2808BF012000D18872104670471B
:109B70006548807A80F0010000EB4001C1EB4010A5
:109B8000674901EB800070472DE9F04F5E4987B0CF
:109B900001224A73C97A624D624C11291CBF1229F5
:109BA000132930D0C8B15849897A237801EB410292
:109BB000C2EB411105EB810294F801C0002113EBC7
:109BC0000C0F0AD030F8113022F81130237894F8B5
:109BD00001C0491C63448B42F4D8F9F77FFB00F0C5
:109BE00008060820F9F775FB474CA07B00250028E4
:109BF0001CBF012121737DD03046F9F765FB6573E9
:109C000007B0BDE8F08FF7F7C2FFF7F7FDFE04904D
:109C1000002818BFF8F747F9434805902078617885
:109C2000394A00EB0108D07A917AA0F11109D06984
:109C300001EB4103C3EB411105EB810B91694145F8
:109C400038BF88460221029112210391002500EBC2
:109C500040012E4601EB001A02AC54F82600F8F73A
:109C600089FC54F826000021F7F716FC009054F800
:109C700026000121F7F710FC019006EB460005993C
:109C800000EB0610002401EBC0072EE0E01704EB08
:109C9000D060421120F01F005DF82210221A01202E
:109CA0009040014220D004F0010007EB403004EB6B
:109CB000D47100EB8A00491000EB810141F6486045
:109CC000B9F1000F09584FF0FF302FD0B9F1010F53
:109CD00008BFC8B205D0B9F1020F04BF0846F8F7B3
:109CE0004FFC2BF815006D1C641C4545B8BF262C95
:109CF000CCDB00E021E0761C022EADDB04980028CE
:109D000018BFF8F7D3F868E73C81001028B70010B7
:109D1000D1800010D2800010B09D0030189D00301E
:109D200010B80010D48000100080003011F4803F83
:109D3000C1F3072018BF4042D3E7A07A80F00100AA
:109D4000A072257358E770B50D466F490122CA709D
:109D50006E4A497816786E4A212914781EBF222946
:109D6000232970BD002818BF002D11D000232246E2
:109D70003146FFF755FC631C012221462846FFF7B8
:109D80004FFC05EB4400A31C01223146FFF748FCC1
:109D9000BDE8704000F058B870B55B4D0446687877
:109DA00068B9E06858B15B490978012994BF5849FE
:109DB00059490B7859490122097800F05FF8E87A8F
:109DC000112804BF0020FFF7DFFEE87A122804BF45
:109DD0000020FFF7D9FEE87A132804BF0020FFF720
:109DE000D3FE6878002804BFA068FFF7A8FC687855
:109DF000112804BF0020FFF7A2FC6878122804BFD6
:109E00000020FFF79CFC6878132804BF0020FFF7B0
:109E100096FC206920B1A979002908BFFFF79AFDB7
:109E2000A879112804BF0020FFF794FDA879122813
:109E300004BF0020FFF78EFDA879132818BF70BD5E
:109E40000020BDE8704085E570B5F9F747FA00F0ED
:109E500008060820F9F73DFA2B4C20790025002848
:109E600001BF207880F001002070A5701CBF012088
:109E7000A0703046F9F728FAE57070BD2DE9F0477B
:109E8000994616460D460446F8F75BF85FEA000C63
:109E90001CD01D49087840F2DB125043204AD1F80B
:109EA000108002EB800009FB08F200EB4200454500
:109EB00094BF2F4647464969A1EB0901B14238BF1B
:109EC0000E460021002E09D8BDE8F0874B463246E9
:109ED00029462046BDE8F047FFF7A2BB0023002F2C
:109EE00008D91CF9032034F8122020F813205B1C39
:109EF0009F42F6D8491C00EB480004EB4504B142F0
:109F0000ECD3BDE8F08700003C810010CC8000104D
:109F1000CD800010CE800010D0800010D3800010C3
:109F200050A800105949002814BF002001200870D3
:109F300070475648007800280CBF01200020704769
:109F40005248017829B14FF040214A6942F001029C
:109F50004A61002141608160C160016141617047D7
:109F60004A48017829B14FF040214A6942F0010284
:109F70004A61002141608160C160016141617047B7
:109F800070B50446F9F7AAF900F008050820F9F7BA
:109F9000A0F93E4A3E490023106901EBC001401C74
:109FA0001061B0F5807F28BF136120780870607859
:109FB0004870A0788870E078C8702079087160795E
:109FC0004871A0798871E079C8715069B0F5807FD7
:109FD0003CBF401C506116D31D2008700120487002
:109FE000207888706078C870A0780871E07848712F
:109FF000207988716079C871D068401CD060B0F554
:10A00000807F28BFD360506840F001005060107816
:10A0100028B14FF04020416921F0010141612846FB
:10A02000F9F752F9012070BD00B50178427883B08C
:10A03000890141EA82018DF80010418809098DF8F3
:10A040000110818809098DF80210817801F00F0252
:10A05000017962F31F118DF80310017A8DF8041055
:10A06000417A8DF805108179C27901F03F0102F043
:10A070000C0241EA02118DF80610C07980018DF8BA
:10A0800007006846FFF77CFF03B000BD5C8100104D
:10A0900058B90010194A002112684FF0402312F0FD
:10A0A000804F26D0164AD2F800C05FEA1C4C04D07C
:10A0B00011686FF30F0141F00101D2F800C01CF4E8
:10A0C0007F4F0CD011684FF0020C01F47F414CEA35
:10A0D0000121DFF830C0DCF800C0C3F874C0D2F84A
:10A0E00000C01CF0FF0F04D011680322C9B242EA7D
:10A0F000014199678069D867FEE700002CED00E018
:10A1000028ED00E038ED00E070B50E460446FBF7A0
:10A1100073F8042811D1A4F59C7050280DD2A01911
:10A12000A0F23910502808D265020024002E04D96C
:10A130002846F8F7CFFC012801D0002070BD641C30
:10A1400005F50075B442F3D3012070BD70B50D461E
:10A150000446FBF751F804280AD1A4F59C70502856
:10A1600006D260022946F8F757FD012808BF70BDE6
:10A17000002070BD10B5074CFEF745FF012808BF51
:10A1800010BD206800F082FD002818BFFBF78CF896
:10A19000F2E70000D4810010E34A0028516814BFA0
:10A1A00041F0010021F0010050607047DE4B59681A
:10A1B0000A0E120721F07F4142EA0060084358600E
:10A1C0007047D9484068C0F303607047D64840687C
:10A1D000000F7047D44800697047D34901200861D7
:10A1E0007047D1490020086170472DE9F043AFB0B6
:10A1F00000270EF07AFE0646A02102A811F0F9FE13
:10A20000002425464FF003084FF00109305D10F09F
:10A21000800F17D0601CC1B28DF8A9108DF8AF5017
:10A220008DF8A880ADF8AC50ADF8AA508DF8AE50BE
:10A230003555CDE90091002201272AAB114602A82D
:10A24000F6F748F9601CC4B20A2CDFD3012F06D1FF
:10A25000102302AA06210120009510F0C7FE0EF07F
:10A2600053FC2FB0BDE8F0832DE9F04FDFF8BC823E
:10A2700087B0D8F80000B0F90E11B0F90C0111F058
:10A2800012FF0120FAF7B3F90020F7F71CFE0EF0D9
:10A290000DFE042000F010F9FAF78DF9FAF7ACFF83
:10A2A00005285ED1DFF888B29F4F4FF000094FF0CC
:10A2B000402A7868C7F80890C0F30366C7F80C9086
:10A2C000D8F80000B100D0F8F80020FA01F101F050
:10A2D0000F04C0F30321C0F303358C4222D10F2DAC
:10A2E00020D003F074FC20B109F022FD082818BF2B
:10A2F0002C467869A04215D009F01AFDAC420CBF7B
:10A300000121002141EA002509F0A7FC45EA0045AA
:10A3100009F01AFD45EA006200238421072002F0BB
:10A32000F9FF7C613146052003F072F8002E7DD0E4
:10A33000022E1FD0042E7AD078680A2E4FEA1061C0
:10A3400020F07F404FEA017118BF41F000710843CF
:10A350007860FEF758FE012803D0FAF74DFF052874
:10A36000A7D00EF0D1FBFAF741F907B0BDE8F04FE6
:10A370000EF0A1BD0D212046FBF740F80028E8D0E3
:10A3800011F0AFFE11F0B2FEFAF7D0F8040065D17B
:10A39000F6F773FF6748F7F780FB0120F7F772FBCA
:10A3A000F8F7BEFF6448F9F770F8F9F757F8F9F7CE
:10A3B00080F8D8F800104000B1F80621B0FBF2F0A8
:10A3C000401CC0F34F00788091F80811397059B1E2
:10A3D000F9F76FF8D8F800104000B1F80411B0FB9D
:10A3E000F1F0401CC0F34F00F8F7D4FF5348CAF80F
:10A3F0001800F7F7CCFBF7F71DFD387838B1401E91
:10A4000010F0FF00387004BF7888F8F7C3FF786851
:10A41000C0F3036529460520F5F767FFFEF7F3FD56
:10A42000012809D07868C0F3036001E03CE03FE018
:10A43000A84208BF002C18D0CAF818B0F8F7E2FFFD
:10A44000F9F717F80020F9F720F8F8F772FFF7F797
:10A450009EFBF7F7DBFA0020F7F71FFB11F046FE33
:10A4600011F049FEFBF739F973E76846F7F7E4FEA8
:10A4700070B16846FFF790FC0198F9F7ECFB68466D
:10A4800011F03EFE0446F7F734FFFAF72EFFC5E75A
:10A49000D8F80000406E10F0704F02D0FAF704FFB9
:10A4A000BCE7FAF729FFB9E7204611F02EFE50E786
:10A4B000204603F0B7FD4CE770B51C4980000968E1
:10A4C000D1F8F81021FA00F000F00F04C1F30320D6
:10A4D000C1F30335844224D10F2D22D003F077FB42
:10A4E00020B109F025FC082818BF2C460E4E7069D3
:10A4F000A04216D009F01CFC0146AC420CBF012062
:10A50000002040EA012509F0A8FB45EA004509F0D2
:10A510001BFC45EA006200238421072002F0FAFEBA
:10A520007461204670BD000074810010D481001059
:10A5300000005FA0413A0010D733001007005FA071
:10A540007047002808BF704780220146014811F07B
:10A550004BBD704758C10010704708283CBFFE49EA
:10A56000087070470020FC4988604860FB4800681C
:10A5700090F88100082838BF087070470020F6491D
:10A5800048607047F4480078704770B5F34D002478
:10A59000286890F86C0010F0020F0BD0FAF72CFE30
:10A5A000022807D1EC482968007801EB8000B0F858
:10A5B000840084B2204670BD70B5E84D4FF48054DD
:10A5C000286890F86C0010F0020F0DD0FAF714FE16
:10A5D000022809D1E0482968007801EB8000D0F812
:10A5E0008400000CC0F31304204670BDDA48807864
:10A5F000002818BF012070472DE9F041FAF7FCFD53
:10A60000022803D103F04FFA022803D04FF4805000
:10A61000BDE8F0814FF480552E4603F062FADFF872
:10A620003C830446CC4FD8F8000090F86C1011F031
:10A63000010F0CD0B0F87600B9684042814206DCC8
:10A640002CB10020641EB860204603F04DFAD8F803
:10A65000001091F86C0010F0040F18BF002C0AD005
:10A66000B1F87C00621E9040B1F87E20824238BF73
:10A670001046C0F31306D1F8A40010F0020F1CBF5F
:10A68000B978002902D0000CC0F31305B54298BF79
:10A6900035462846BDE8F0812DE9F04FDFF8BCA231
:10A6A00087B0DAF8001091F86C2012F0020F0DD08C
:10A6B000A94A91F88090DFF8A8B21778002809DB42
:10A6C000484503D2B84218BF064643D107B0002020
:10A6D000BDE8F08F3E464FF0FF38F7F797F9F7F7F0
:10A6E000B4FF0025B9F1000F34D9DAF800000024D6
:10A6F00000EB8500B0F8840081B22046F6F7DCFD5F
:10A70000F7F798FB6846F7F797FD002866D00298A0
:10A7100078B1014693489BF8002000785043421ED0
:10A7200007D331F9020B0028B8BF40420444521E3F
:10A73000F7D2F7F7DEFDF7F769F9002322469221F9
:10A74000072002F0E7FDA04584BF2E46A0466D1C01
:10A750004D45CAD3B74244D0082E3CBF7E490E7047
:10A76000DAF80000B0F8821039B300EB870200EB92
:10A770008600B2F88420B0F8840092B280B2801AC9
:10A78000484340F30F34F9F7D6FA774B9BF8002093
:10A79000002193F800C002FB0CF2002A0DD930F81A
:10A7A0001120224420F811209BF8002093F800C0CB
:10A7B000491C02FB0CF28A42F1D84FF0806003F092
:10A7C000C8FADAF80000002300EB86008021B0F818
:10A7D000840082B2072002F09DFD09E0FAF764FDD3
:10A7E00090E703F07EF903283CBF401C03F07CF99E
:10A7F000012007B0BDE8F08F584857490068B0F80D
:10A800007600424288688242BCBF401E8860704722
:10A810002DE9F04F93B093460E4604464FF0000AE0
:10A8200003F05FF9DFF834814B4F0500D14610D1BA
:10A8300011F070FCD8F80010B1F87810884208D3F5
:10A840000120C7F8089003F04FF913B00120BDE8CC
:10A85000F08F002E1FDDB8680028B8BFC7F8089039
:10A8600007DBD8F80010B1F874108842BCBF401C58
:10A87000B860D8F80000B968B0F87400884215DCF8
:10A88000032D13D2681CC7F8089003F02DF913B0FC
:10A890000120BDE8F08F09D1D8F80000B0F87600AB
:10A8A0004142B8688842C4BF401EB860B87850B111
:10A8B000D8F8000090F8A40010F0040F1EBF00208C
:10A8C00013B0BDE8F08FD8F80000B0F972108C42D8
:10A8D0000EDD796821447960B0F86E00884210DCA2
:10A8E0004FF0FF30C7F80490FFF7D6FE824608E02D
:10A8F0007868002805DD002CD4BF01212146401ACC
:10A900007860DFF8689099F8000007283BD1184874
:10A91000594600784200684611F075FBADF80040DA
:10A92000ADF80260ADF804503889ADF80600B8887B
:10A93000ADF80800D8F80000B0F87210ADF80A10B1
:10A94000B0F87410ADF80C10B0F86E10ADF80E1031
:10A95000B0F876000EE00000C0810010D481001035
:10A96000CC800010D0800010CD8000103D81001000
:10A97000D3800010ADF8100099F80000072804BF3C
:10A980006846FEF7C0FE504613B0BDE8F08F3E4863
:10A9900010B50068D0F8A40010F4807F06D0C0F392
:10A9A0000330012101FA00F0F8F705FA37490020D9
:10A9B0004870887010BD70B5344D0024A878002808
:10A9C00014BF01260026687828B903F099F80028FA
:10A9D00008BF002100D001218E4225D00A1C18BFDB
:10A9E0000122AA7028480068D0F8A43013F0040FA0
:10A9F0000ED021B1C3F30310082808D206E00021CD
:10AA0000A960696090F88100082800D228700124AC
:10AA100013F0020F18BF0124002A18BF01220023DF
:10AA20008221072002F076FC204670BD16490020E6
:10AA30000968D1F8A41011F4807F08BF7047DFF8CF
:10AA40004CC09CF80120131C18BF012330B4104CDB
:10AA5000C1F30332E46B012505FA02F2224011F43E
:10AA6000007F01D00AB102E00AB1002100E001211B
:10AA70008B4204BF30BC7047081C18BF01208CF803
:10AA8000010030BC97E70000D4810010C0810010A5
:10AA9000001000406948007870476848406800F539
:10AAA000407070476548406800F58070704770B529
:10AAB000624C4FF41C32624962601068884204BFE5
:10AAC0005068B0F5087F26D1D2F808C0BCF5084F11
:10AAD00021D85C49D06888420DD000231146184621
:10AAE000B3EB9C0F07D251F8045B401C6B40B0EBFA
:10AAF0009C0FF8D37BB9012502F5807000F0C6F8F1
:10AB000048B1606800F5407000F0CFF800281EBF23
:10AB10002570012070BD002070BD484900200870DC
:10AB20004FF41C30F7F7D6BF4448017841B1406874
:10AB3000434A0168914202BF4168B1F5087F7047FE
:10AB4000002070473D4B5B6803F580731844F8F7AD
:10AB5000B7B83A4B5B6803F540731844F8F7B0B8E0
:10AB60003648406800697047344949680A6982423A
:10AB70009CBF00207047C0EBC00001EBC00000F597
:10AB8000806070472D4A526802EB80035B6A1A446A
:10AB90002D4B53F820C0403333F810000CEB00036A
:10ABA000401E5B1E23EA000000FB012070472DE9D8
:10ABB000F003224B244F00225C6807F140069046C8
:10ABC000831893F928C0BCF1000FB8BF41F8228068
:10ABD00012DBD3B204EB830557F8239036F8133019
:10ABE0006D6A99445B1EA9F10109254429EA030312
:10ABF00003FB0C5341F82230521C102AE0D3BDE86D
:10AC0000F00370470029B8BF704730B494460B4A30
:10AC10000E4C526802EB80035B6A13440A4A52F8F6
:10AC2000202034F810001418401E641E24EA00008E
:10AC300001FB003030BC6146F8F742B8CC8100100F
:10AC400054465053EFBEADDED4E6010014E70100D8
:10AC500010B5FFF72CFFA8B1FFF71FFF0146D02268
:10AC6000174811F0C1F9FFF71DFF164C01464FF4CC
:10AC7000E272206811F0B8F92068406DBDE810401C
:10AC800002F0CABE0220FAF77BFBE2E758B10E4A97
:10AC90000168914207D1406820F00F00B0F5107FA5
:10ACA00004BF012070470020704730B1006820F0D9
:10ACB0000F00602804BF012070470020704700008B
:10ACC000E4F80010D481001041505352B34810B53D
:10ACD000806810F0020F15D0F6F796FE90B1F6F7E7
:10ACE00056FE0402FAF788FA44EA0044FAF78AFAB0
:10ACF00044EA00604EF2AF0108434FF04021C867BC
:10AD0000012010BD002010BD10B572B60120F7F76C
:10AD1000E5FDF8F789FCF8F7B3FC4FF0FF30F8F7E2
:10AD2000D8FA9F4880234FF40052002152F821C0E6
:10AD300040F821C0491CB1EB930FF7D3F8F7DBFAC9
:10AD4000F8F7FEFEF8F720FF9648F8F739FF0120E4
:10AD5000F8F7F7FEF7F756FE1E20F8F7E7FEF8F7CC
:10AD6000ABFCF8F733F8F8F7A3FEF8F7EBFCF8F7CD
:10AD7000D3FAF8F7A3F8F6F75CFEFFF769FFF8F7E8
:10AD800052FAF8F71DFAFEF7BFF8FBF70BFDFFF7D5
:10AD9000E7F862B684480DF097FE844C2068B0F95D
:10ADA0000C010EF081F8F5F786FAFFF7D5FBF8F7FE
:10ADB00023FFFAF7CAFC2068018BC1F30722418AFE
:10ADC000008AFEF7DAFB2068806E000C02F09FFA22
:10ADD000FFF7B6FB11F0A3F9FAF706FB206890F82D
:10ADE000640000F00F00F7F79FFC206890F8200047
:10ADF00010F0010F04BF0021032003D002F059FE20
:10AE000001460220FAF70DFA4FF040242069002392
:10AE100000F070021946022002F07CFA206910F05E
:10AE2000200F17D0226F00230521072002F072FAAD
:10AE3000626F00230521072002F06CFAA26F002345
:10AE40000521072002F066FAE26F002305210720A2
:10AE500002F060FAFFF79BFDF9F7EBFD0020206799
:10AE600010BD534CFEF7CFF8012806D0FAF7C4F90D
:10AE7000032802D102F0F9FA40B3002C05DC02F0FD
:10AE800018FE01460220FAF7CCF9DFF82C810127E1
:10AE9000484E4FF04025A8F10309FAF7ADF90446F2
:10AEA000FAF7B0F90146204602F0B2FAFAF7AAF929
:10AEB00001462046F5F719FAFEF762F8072C68D22A
:10AEC000DFE804F0671A082427172A00641E002C04
:10AED000C8DCD4E7307848B9FBF702FC30B900236E
:10AEE0001A462021072002F015FA377003F05BFBA9
:10AEF000D3E7FFF7B9F9D0E7FBF710FBFAF77CF9D6
:10AF0000012804BF0220FAF789F9C6E702F027FDFD
:10AF1000C3E7FFF72FF9C0E70024C5F81880FEF754
:10AF200072F8012806D1FAF767F9062802D0C5F8A9
:10AF30001890B2E7FAF763F940B3002C04DCFAF793
:10AF4000C9F943F22054EAE7641E00BF00BF00BF06
:10AF500000BF00BF00BF00BF00BF00BF00BF00BFF9
:10AF600000BF00BF00BF00BF00BF00BF00BF00BFE9
:10AF700000BF00BF00BF00BF00BF00BF00BF00BFD9
:10AF800000BF00BF00BF00BF00BFC8E7FAF78CF9E1
:10AF9000C5E70220FAF7F4F97FE7000000800040DF
:10AFA00000FC00107DCC0000E4F80010D4810010FB
:10AFB000FF700200D881001003005FA0FE49086006
:10AFC000704710B44FF44030FC4A016891421CD1E4
:10AFD0004168B1F5007F18D3836800228446B3F539
:10AFE000056F88BF4FF405630021B1EB930F24BFB9
:10AFF00010BC70475CF82140491C2244B1EB930F10
:10B00000F8D3002A04BF10BC7047002010BC704762
:10B0100070B54FF440310446E84D0868A84217D196
:10B020004868B0F5007F13D38B6800228C46B3F5D7
:10B03000056F88BF4FF405630020B0EB930F08D273
:10B040005CF82060401C3244B0EB930FF8D302B19F
:10B05000002149B18A68B2F5056F88BF4FF40562D7
:10B06000204610F0C1FF1CE0FF224FF4056120468E
:10B0700010F0ECFF4FF40870C4E900504FF4056085
:10B08000A0600020E06084F8200084F8210084F8AB
:10B09000220084F8230040F2FF71C4E90410A0618B
:10B0A000E061012070BD70B50021C160D0F808C01A
:10B0B0000B460446BCF5056F88BF4FF4056C0022B3
:10B0C000B2EB9C0F06D254F82250521C2B44B2EB28
:10B0D0009C0FF8D35942C1604FF440304FF40562E1
:10B0E0002146F7F7EDFD012818BF002070BDFF22B3
:10B0F00070B50025044605614FF40061503010F032
:10B10000A5FFA584E584E562A56265632563E56323
:10B11000A56365642564E5640120A56470BD70B411
:10B1200002684FF408715160016801F1500291F812
:10B1300021C091F820300CFB03F102EB4101002209
:10B14000BCF1000F08D900EB4204521CB4F8EA40ED
:10B1500021F8024B9445F6D80022002B08D900EBC9
:10B160004204521CB4F8124121F8024B9342F6D823
:10B170000468002294F82240002C0BD900EB420412
:10B18000521CB4F8BE4321F8024B046894F82240E4
:10B190009442F3D80468002294F82340002C0BD981
:10B1A00000EB4204521CB4F8CE4321F8024B046871
:10B1B00094F823409442F3D80022BCF1000F08D940
:10B1C00000EB4204521CB4F8704021F8024B944545
:10B1D000F6D80022002B08D900EB4204521CB4F828
:10B1E000984021F8024B9342F6D8B0F8E62021F8B7
:10B1F000022BB0F8E82021F8022BB0F8E42021F867
:10B20000022B00240022BCF1000F0ED904EB4405F0
:10B2100005EB041500EB850505EB4206521CB6F85C
:10B220005E6121F8026B6245F6D30022002B0ED935
:10B2300004EB440505EB041500EB850505EB420620
:10B24000521CB6F88E6221F8026B9A42F6D3641C47
:10B25000042CD7D30023D0F800C000229CF822C0D1
:10B26000BCF1000F88BF00EB031C0BD90CEB4204B0
:10B27000521CB4F8DE4321F8024B046894F82240D3
:10B280009442F3D8D0F800C000229CF823C0BCF14F
:10B29000000F88BF00EB031C0BD90CEB4204521CBF
:10B2A000B4F8FE4321F8024B046894F8234094421A
:10B2B000F3D85B1C022BCED370BC70472DE9F74F3F
:10B2C00088B000250A992C462E460968049101F1A0
:10B2D00050030999002984BF3949D1F800801CD94D
:10B2E0000022002888BFB8F9CE700DD933F9021BAF
:10B2F0000029B4BFC1F1000C8C46BC45BCBF0D4455
:10B30000641C521C8242F1D30999761C8E42E7D309
:10B31000002CC8BF95FBF4FA08DC4908414301EB57
:10B320005002049901EB4201B1F950A000210291B1
:10B33000019104995031009100210391099900294C
:10B3400075D91F49009E069609684FF0000B4FF013
:10B350000109B1F9C0E0D1F8B4105F46C1F307416B
:10B36000D846CDF814B00791002830D9B6F900209E
:10B370004FF0000C06999344634600280DD9B1F9AB
:10B380000040A51A48BF151B7545B8BF0CF1010C4C
:10B3900001EB49015B1C8342F1D307998C4503D330
:10B3A00005997F1C1144059108F1010806EB490637
:10B3B0008045DBD3002F05E0DC81001053454C466F
:10B3C000D4810010C4BF059991FBF7F101DC9BFB10
:10B3D000F0F1039B0A9A09B202EB4302A2F8701043
:10B3E000FE4A1268B2F9BA30AAEB030399420ADDA9
:10B3F000B2F9B82052448A4205DD019A1144019104
:10B400000299491C02910099099A01EB40010091AF
:10B410000399491C0391914293D30299002906DDB7
:10B42000DDE9011291FBF2F1019103E0FFE75146E2
:10B43000CDF804A00A9AA2F8E61000210291039127
:10B4400004995031009100210491002868D9E34902
:10B45000009F069709684FF0000B099EB1F9BCE008
:10B46000D1F8B410D846090ED946CDF814B00791DA
:10B47000002E2BD9B7F900204FF0000C0699934409
:10B480006346002E0DD9B1F90040A51A48BF151B1F
:10B490007545B8BF0CF1010C01EB40015B1CB342D8
:10B4A000F1D307998C4504D3059908F1010811449B
:10B4B000059109F1010907EB4007B145DAD3B8F16D
:10B4C000000FC4BF059991FBF8F101DC9BFBF6F17D
:10B4D000049B0A9A09B202EB4302A2F89810BF4AF1
:10B4E0001268B2F9BA30AAEB030399420ADDB2F945
:10B4F000B82052448A4205DD039A1144039102990F
:10B50000491C02910099891C00910499491C0491DD
:10B5100081429CD302980028C4BF039991FBF0FAA2
:10B520000A98A0F8E8A001980A99504400B200EBEC
:10B53000D0704010A1F8E4000BB0BDE8F08F2DE909
:10B54000F04F146889B015460E460746A1F1200851
:10B55000202928BF4FF0FF3A05D24FF0010000FA32
:10B5600006F0A0F1010A38BF4FF0000B05D34FF0F1
:10B57000010000FA08F0A0F1010B202F3DBF0120CF
:10B58000B840401E4FF0FF3038BF002207D3A7F16C
:10B5900020024FF0010101FA02F1A1F10102C6F10E
:10B5A0002009202E34BF20FA09F100FA08F1B24038
:10B5B0001143B040CDE90001206920F4FE60206114
:10B5C0008748007810F0010F7ED02A463146384671
:10B5D00001F026FA0020A8616861002F84BFDFF81F
:10B5E000FCE101221BD905EB4001B1F998100029BB
:10B5F000B8BF494209B2DEF80030B3F9CC308B4213
:10B600000ADD410905EB810100F01F0C4B6902FACC
:10B610000CFC43EA0C034B61401CB842E3D300200E
:10B62000012F18BFA7F1010E3BD005EB4001B1F986
:10B630009A30B1F99820991A48BFD11A09B2DFF8A7
:10B640009CC1DCF800C0BCF9C4C08C4526DAB5F951
:10B65000E810B2EB010C48BFA1EB020C0FFA8CFC16
:10B660005A1A48BFCA1A11B28C450BDB420905EBC6
:10B67000820100F01F0C01224B6902FA0CF21A43FE
:10B680004A610BE0411C4B0905EB830201F01F0CE2
:10B690000121536901FA0CF119435161401C7045B5
:10B6A000C3D36969E869B14008432063A969286A7E
:10B6B000B140014361636869202E34BF20FA09F06C
:10B6C00000FA08F0084300E000E0606344480068C6
:10B6D000079010F0040F00F0BC8100202863E8629E
:10B6E000002E88BFDFF8F4E01BD9DEF8002005EB60
:10B6F0004001B1F95E11B2F9D8308B4203DCB2F9E6
:10B70000DA208A420ADA420905EB820100F01F0CB6
:10B710000122CB6A02FA0CF21A43CA62401CB04200
:10B72000E3D30020A8626862002F88BFDFF8ACE096
:10B730001BD9DEF8002005EB4001B1F98E12B2F9F9
:10B74000D8308B4203DCB2F9DA208A420ADA4209A5
:10B7500005EB820100F01F0C01224B6A02FA0CF289
:10B760001A434A62401CB842E3D300202864E863CD
:10B77000002E88BFDFF864E01BD9DEF8002005EB5F
:10B780004001B1F9AA11B2F9DC308B4203DCB2F905
:10B79000DE208A420ADA420905EB820100F01F0C22
:10B7A0000122CB6B02FA0CF21A43CA63401CB0426E
:10B7B000E3D30020A8636863002F88BFDFF81CE094
:10B7C00020D9DEF8002005EB4001B1F9DA12B2F918
:10B7D000DC308B4208DCB2F9DE2003E0D4810010BB
:10B7E000DC8100108A420ADA420905EB820100F08E
:10B7F0001F0C01224B6B02FA0CF21A434A63401CE5
:10B80000B842DED300202865E864A8646864002E8E
:10B8100088BFDFF850E71CD9DEF8003005EB4001A7
:10B82000B1F9F611B3F9E0208A4203DCB3F9E22062
:10B830008A420BDA410905EB810C00F01F0301215C
:10B84000DCF84C2099401143CCF84C10401CB0421D
:10B85000E2D30020002F88BFDFF808E71BD9DEF80D
:10B86000002005EB4001B1F92613B2F9E0308B421C
:10B8700003DCB2F9E2208A420ADA420905EB8201CE
:10B8800000F01F0C01224B6C02FA0CF21A434A64BE
:10B89000401CB842E3D3696AE86AB14040EA010E4D
:10B8A000C4F838E0A96A286BB1400843E063696ACC
:10B8B000202E34BF21FA09F101FA08F141EA000013
:10B8C000E0630590696BE86B01FA06F140EA01025A
:10B8D0002264A96B286C01FA06F140EA0100606459
:10B8E000696B34BF21FA09F101FA08F141EA00015C
:10B8F00061646B6CE86C03FA06F340EA0300A06431
:10B900000490AB6C286D03FA06F340EA0300E06490
:10B910006B6C34BF23FA09F303FA08F343EA00001F
:10B92000E0640290059832EA0E0521EA000C4EEA26
:10B9300005022564069240EA0C00C4F844C006EBF8
:10B940000701039008BFBCF1000F42D000231A4644
:10B950001846002988BF01273BD94FEA501804EB4D
:10B96000880800F01F09D8F8408007FA09F918EA9A
:10B97000090F03D0864294BF521C5B1C401C8142BD
:10B98000EBD8012B0FD105EA0A0040EA0E00A063B4
:10B9900005980CEA0B031843E06325EA0A002064CB
:10B9A0002CEA0B006064012A13D1226C0098A36B6F
:10B9B00010401843A063606C019BD4F83CC0034066
:10B9C00043EA0C03E363009B9A432264019A904389
:10B9D0006064069A049830EA0202A264069840EA7B
:10B9E000020CDDE9020320EA0300E064039B43EA62
:10B9F000000508BF002821D000231A461846002958
:10BA000088BF012717D94FEA501804EB880800F0C7
:10BA10001F09D8F8488007FA09F918EA090F03D076
:10BA2000864294BF521C5B1C401C8142EBD8002B09
:10BA300018BF002A02D10020A064E064079810F02B
:10BA4000010F06D0206B20EA0C002063606BA84336
:10BA50006063206B0099084203D1626B01990A422E
:10BA600003D0216941F01001216110EA0A0F04BFDF
:10BA7000606B10EA0B0F03D0206940F020002061BA
:10BA8000A06B0099084203D1E26B01990A4203D0EE
:10BA9000216941F04001216110EA0A0F04BFE06B07
:10BAA00010EA0B0F03D0206940F080002061206C69
:10BAB0000099084203D1626C01990A4203D02169BE
:10BAC00041F48071216110EA0A0F04BF606C10EA32
:10BAD0000B0F03D0206940F400702061A06C002897
:10BAE00004BFE06C002803D0206940F4806020612E
:10BAF00009B00120BDE8F08F2DE9F04FBDB016462A
:10BB00000D460446F5F782FFF5F75FF901004FF0A7
:10BB100011001DBF029001200390012108BFCDE953
:10BB20000210CDE93854F6F705FA0022002D88BF3F
:10BB300004A904D9835C8B54521C9542FAD8F6F7B9
:10BB4000FBF90021002C88BF04AA07D9435C02EB53
:10BB5000010C491C8CF820308C42F7D8F6F71DF9FF
:10BB600040F2012131900840F5F7F9FFFE480078D6
:10BB700010F0200F63D0F5F728F9FC49FC4A0028A3
:10BB80000CBFCDE90021CDE9001206F1EA003A90A0
:10BB900028303B90FF210F20F9F7DBFDF5F736FF4A
:10BBA0000025EA460DF1E8090DF1E00B02A85BF86B
:10BBB000257050F82500F6F7DDFC0024002F84BF27
:10BBC00004A800EB451818D918F90400262828BF46
:10BBD00000200BD2C10700EBD070890C401001EBA4
:10BBE00080005AF825104058F6F7CAFC59F825107D
:10BBF00021F81400641CBC42E6D36D1C022DD5D381
:10BC0000DC4804781D2C1AD100210A4614AD5BF8DB
:10BC100022300020002B88BF59F822C007D93CF8F9
:10BC2000107025F81170401C491C8342F7D8521C33
:10BC3000022AECD31D2C04BF2846FDF78BFECA4D0B
:10BC4000287810F00C0F00F0CB82F5F7BEF8CA4A46
:10BC5000CA4900280CBFCDE91412CDE91421C84807
:10BC6000F5F77DFF0120F5F717FB2D900120F5F783
:10BC700063FB2B900120F5F73DFE1B900298F5F732
:10BC800088FB28900398F5F784FB17900120F5F7BF
:10BC900015FC2E901120F5F711FC27900120F5F7E7
:10BCA0004DFC2C901120F5F749FC1D9024A8009024
:10BCB00022AB20AA1EA90298F5F763FD25A80090E3
:10BCC00023AB21AA1FA90398F5F75BFD0298F5F7AE
:10BCD000DAFD26900298F5F7D6FDA24C0190206877
:10BCE000B0F8E4100120F5F7E7FA00210120F5F79C
:10BCF000E9FD206890F8E6100298F5F75CFB2068F3
:10BD000090F8E6100398F5F756FB00210120F5F7AF
:10BD1000EEFB00211120F5F7EAFB00210120F5F7E9
:10BD200026FC00211120F5F722FC2068B0F8E8106D
:10BD30000298F5F756FD2068B0F8E8100398F5F77B
:10BD400050FD00210120F5F7EFFD2990864800788D
:10BD500010F0040F00F047812068B0F8EC1000915B
:10BD600090F8EB3090F8EA200B210298F5F7DBFC15
:10BD70002068B0F8EC10009190F8EB3090F8EA20D1
:10BD80000B210398F5F7CFFC00210120F5F7CCFD3E
:10BD900032A800F030FE3699002238AD002055F868
:10BDA0002230002B0ED902EB420C0CEB021C06EBEE
:10BDB0000C1C31F8027B0CEB4008401CA8F85E71AB
:10BDC0008342F6D8521C022AE8D30298F4F729FDE0
:10BDD0001C900398F4F725FD1A9000210298F5F7BE
:10BDE0005BFB189001210298F5F756FB1690002195
:10BDF0000398F5F751FB2A9001210398F5F74CFBC6
:10BE0000584C19902068B0F8EE10009190F8EB3083
:10BE100090F8EA200B210298F5F785FC2068B0F82D
:10BE2000EE10009190F8EB3090F8EA200B21039887
:10BE3000F5F779FC00240DF1080B00210120F5F73E
:10BE400073FD00210298F4F7D4FC00210398F4F765
:10BE5000D0FC5BF824000121F4F7CBFC38A80025C6
:10BE600050F8249014A8B9F1000F50F824002F9036
:10BE700049D904A800EB4410009004EB440000EB07
:10BE8000041006EB001A00980022114610F90580F4
:10BE90001046F5F757FDB8F1200F06DB0027A8F193
:10BEA0002001012000FA01F804E0012000FA08F75F
:10BEB0004FF000085BF824003A460021F5F7DAFA63
:10BEC0005BF8240042460121F5F7D4FA6FEA080234
:10BED000F9430920F5F736FD32AFF5F7ABFFFDF773
:10BEE00092F8012804D03846F6F7A6F900287DD04C
:10BEF000F5F78CFD2F9800880AEB45016D1CA1F821
:10BF0000AA014D45BFD3002211461046F5F71AFD90
:10BF1000641C022C91D31C990298F4F76AFC1A99BC
:10BF20000398F4F766FC0021189A0298F5F7A2FA34
:10BF30000121169A0298F5F79DFA00212A9A039892
:10BF4000F5F798FA0121199A0398F5F793FA054C39
:10BF50002068B0F8F010009190F8EB3090F8EA20EB
:10BF60000B210FE0D4810010DC810010B09D003067
:10BF7000189D003042810010CC0E0030CC090030FA
:10BF800001000E000298F5F7CEFB2068B0F8F01023
:10BF9000009190F8EB3090F8EA200B210398F5F728
:10BFA000C2FB01210846F5F7BFFC32A800F023FDD3
:10BFB0003699002238AC002054F822C0BCF1000FA2
:10BFC0000ED902EB420303EB021306EB031331F825
:10BFD000025B03EB4007401CA7F8F6518445F6D8F6
:10BFE000521C022AE7D3FE48007800E049E010F036
:10BFF000080F7DD0FB4D2868B0F8F210009190F842
:10C00000EB3090F8EA200B210298F5F78CFB2868BA
:10C01000B0F8F210009190F8EB3090F8EA200B2184
:10C020000398F5F780FB00210A4638AF002057F847
:10C0300021C0BCF1000F0CD901EB410303EB01134C
:10C0400006EB031303EB4004401CA4F84222844592
:10C05000F8D8491C0229E9D32868002490F8240163
:10C06000B4EB400F7CDA286890F82401A042D4BFDA
:10C07000012100210120F5F757FC32AFF5F7DAFE78
:10C0800002E0F9F711F92AE7FCF7BDFF012803D018
:10C090003846F6F7D1F860B3F5F7B8FC36994FF0AB
:10C0A00000090DF1E00E00225EF829701046002F05
:10C0B00005D931F91030401C1A448742F9D8B2FB37
:10C0C000F7F2781E3ED009EB490303EB091306EBA8
:10C0D000031A31F9103001EB400C3CF9028CB3EB40
:10C0E000080348BF5B4231F91080B8EB020801E059
:10C0F00036E01CE031F910804CBFA2EB0808A8EB39
:10C1000002083CF902BC3CF902CCBBEB020B4CBF71
:10C11000A2EB0C0CACEB020CE0450AEB400C09DD89
:10C12000BCF942824345C8BFACF8423208E0F9F797
:10C13000BBF8A9E7BCF940829845B8BFACF84032DB
:10C14000401EC6D109F1010901EB4701B9F1020F07
:10C15000A9D32868641C90F82401B4EB400F82DB5B
:10C1600001202D99F5F7A8F801202B99F5F7EFF8A4
:10C1700001201B99F5F7A6FB28990298F5F71BF902
:10C1800017990398F5F717F901202E99F5F7AFF9EC
:10C1900011202799F5F7ABF901202C99F5F7E7F96C
:10C1A00011201D99F5F7E3F924980090229B209A1D
:10C1B0001E990298F5F7B7FA25980090239B219ACB
:10C1C0001F990398F5F7AFFA26990298F5F709FB3E
:10C1D00001990398F5F705FB01202999F5F7A4FBD0
:10C1E0003198F5F7BCFC3DB0BDE8F08F2DE9F04F7C
:10C1F000ADF6844DFF224FF4056168460FF026FF2F
:10C20000FF224FF484610DF505600FF01FFFCDF89C
:10C2100050D86846FEF7FCFE714C208810F4804F21
:10C2200015D00025FF224FF4006114A804950FF0EB
:10C230000DFFADF82450ADF826500B950A950D95DD
:10C240000C950E950F951195109513951295DDF897
:10C250005018DDF85008DDF8503891F8211090F8AA
:10C260002000503301FB00FC03EB4C030DF505628D
:10C270004FF0000C002909D902EB4C0633F8025BA1
:10C280000CF1010CA6F8EA506145F5D84FF0000C0E
:10C29000002809D902EB4C0633F8025B0CF1010CC3
:10C2A000A6F812516045F5D815684FF0000C95F8C6
:10C2B0002250002D0CD902EB4C0633F8025BA6F895
:10C2C000BE5315680CF1010C95F822506545F2D863
:10C2D00015684FF0000C95F82350002D0CD902EB97
:10C2E0004C0633F8025BA6F8CE5315680CF1010C2E
:10C2F00095F823506545F2D84FF0000C002909D974
:10C3000002EB4C0633F8025B0CF1010CA6F87050FE
:10C310006145F5D84FF0000C002809D902EB4C0616
:10C3200033F8025B0CF1010CA6F898506045F5D883
:10C3300033F802CBA2F8E6C033F802CBA2F8E8C08B
:10C3400033F802CBA2F8E4C000254FF0000C00291E
:10C350000FD905EB450606EB051602EB860606EB44
:10C360004C0833F8027B0CF1010CA8F85E718C4587
:10C37000F5D34FF0000C00280FD905EB450606EB6E
:10C38000051602EB860606EB4C0833F8027B0CF12F
:10C39000010CA8F88E728445F5D36D1C042DD4D3FE
:10C3A000002516684FF0000C96F82260002E88BF1A
:10C3B00002EB05160CD906EB4C0833F8027BA8F803
:10C3C000DE7317680CF1010C97F822706745F2D8FC
:10C3D00016684FF0000C96F82360002E04E0000071
:10C3E000DC810010D481001088BF02EB05160CD947
:10C3F00006EB4C0833F8027BA8F8FE7317680CF1C3
:10C40000010C97F823706745F2D86D1C022DC8D334
:10C41000FEF754FFFE480125066816F4004F7DD153
:10C42000FC480DF505670025006890F8B40000F0A1
:10C430000F0401F020F8012809D00F212046F8F759
:10C44000DDFF012812D0002001F012F899E0002150
:10C450000846F5F7A7FBF4F79EFC50B1EE48D0F87C
:10C46000401341F48031C0F8401302E0012000F095
:10C47000FFFFEA4890F80080E94890F80090B9F191
:10C48000000F18BFB8F1000F79D0DDF85048002038
:10C4900084F8208084F8219084F8220084F8230016
:10C4A000F6F7A7F816F0100F09D0DE493A460878DB
:10C4B00084F82200497884F8231000F0E2FC16F09A
:10C4C0002C0F04D03A4649464046FFF715FB16F0BC
:10C4D000030F53D0CDF8707CF5F75FFC044600F4F1
:10C4E0008170F5F73CFBFF210F20F9F732F9F5F7E2
:10C4F0008DFA2046F5F733FBDDF850B80BF1500507
:10C50000F5F71AFD82460020F6F734F80026B9F157
:10C51000000F25D9002406EB460000E031E000EBD7
:10C52000061716E01AF90400262811D2C107890C53
:10C5300000EBD07001EB8701401001EB800000F1AF
:10C54000405000F500400068F6F71AF825F8020B95
:10C55000641C444538BF262CE4D3761C4E45D9D301
:10C56000B14800781D2804BF0BF15000FDF7E7F833
:10C5700049464046DDF8702CFEF7A0FE0125F5F790
:10C58000CDFB9DF82000CDF8740C9DF82100CDF86E
:10C59000780C002D1FBFDDF8740C0028DDF8780C36
:10C5A000002804BF0DF6844DBDE8F08F9848006860
:10C5B000CDF87C0C10F0020F00F00B81DDF8504834
:10C5C000DDF8786CDDF8741C206947F6FF7920F0FF
:10C5D0000F00206100200DF5056504F150076FEA9A
:10C5E0000908CDF86008CDF85C08CDF858088246F7
:10C5F000CDF85408002E4ED90AFB01F04FF0010C83
:10C6000037F91020002093465B46CDF8700C0129C5
:10C610001BD90AFB01C037F910009842C8BF034676
:10C620009042B8BF0246B0EB0B0E48BFABEB000E1A
:10C630000FFA8EFBDDF870ECF345C8BFCDF870BC87
:10C6400083460CF1010C8C45E3D34345C8BF9846A3
:10C650004A45B8BF9146981A48BFD01A02B26D48F1
:10C660000068B0F9C030934205DBB0F9C220DDF8B4
:10C67000700C90420BDD4FEA5A1005EB80000AF077
:10C680001F0C0122C36802FA0CF21A43C2600AF1BD
:10C69000010AB245B0D34FF0000A00294CD937F94E
:10C6A0001A20002093465B464FF0010CCDF8700C29
:10C6B000012E1BD90CFB01A037F910009842C8BF0E
:10C6C00003469042B8BF0246B0EB0B0E48BFABEB3F
:10C6D000000E0FFA8EFBDDF870ECF345C8BFCDF805
:10C6E00070BC83460CF1010CB445E3D34345C8BF8D
:10C6F00098464A45B8BF9146981A48BFD01A02B228
:10C7000044480068B0F9BC30934205DBB0F9BE2064
:10C71000DDF8700C90420BDD4FEA5A1005EB8000FB
:10C720000AF01F0C0122436802FA0CF21A4342601D
:10C730000AF1010A8A45B2D3E868002804BF2869D3
:10C74000002803D0206940F00800206168680028B4
:10C7500004BFA868002803D0206940F004002061CD
:10C760006968E868B1400843A062A9682869B140D7
:10C770000143E1626868202E39BFC6F12002D04033
:10C78000A6F1200290400843E062A4F82490A4F8A7
:10C790002680B5F9E410B8EB010048BFA1EB080012
:10C7A0001C490968B1F9B820904203DD206940F0C6
:10C7B00002002061B5F9E420B2EB090048BFA9EB03
:10C7C0000200B1F9BA10884203DD206940F001008F
:10C7D0002061DDF87C0C0E4D10F0050F07D00DF533
:10C7E0000562DDF8781CDDF8740CFEF7A8FED5F8BC
:10C7F000008018F0080F7CD0DDF850280DF505609A
:10C80000DDF8749C1169DDF8783C21F4C0510DE02D
:10C81000DC810010D481001000500040CC8000105A
:10C82000CD800010D48000103D8100104FF0000A30
:10C830001161CDF8B0A85146CDF8ACA8002B84BF4B
:10C84000DFF840B4012418D9DBF8006000EB410C9C
:10C85000BCF942C2B6F9266166450BDA4E0900EB17
:10C86000860C01F01F07DCF85C6004FA07F73E4312
:10C87000CCF85C60491C9942E6D3C0F858A000216E
:10C88000C0F854A0B9F1000F84BFFE4C012618D99E
:10C89000276800EB410CBCF972C3B7F926716745F4
:10C8A0000CDA4F0900EB870C01F01F0ADCF854701A
:10C8B00006FA0AFA47EA0A07CCF85470491C4945B7
:10C8C000E6D3916BD0F85CC041EA0C01D0F854C0BB
:10C8D0000CFA03FC41EA0C019163D16BD0F860C003
:10C8E00041EA0C01D0F858C00CFA03FC41EA0C0CE8
:10C8F00000E020E0C2F83CC0416D202B39BFC3F1FD
:10C900002003D940203B994041EA0C01D163416D9D
:10C91000002904BF816D002903D0116941F4006131
:10C920001161C16D002904BF006E002803D0106999
:10C9300040F48050106118F0100F18BF18F0050F68
:10C9400007D09DF823109DF822000DF5056200F038
:10C950007BF9287810F0400F2FD10598401C0590E6
:10C960000498002814BF0798069800F1010014BF2E
:10C97000079006900DF50560FEF7D1FB00200246FA
:10C980000390029869468C46B0F5056F94BF034644
:10C990004FF405630020B0EB930F06D25CF8204003
:10C9A000401C2244B0EB930FF8D35042C8604FF4C0
:10C9B00040304FF40562F6F783F941208DF8700C92
:10C9C0009DF810008DF8710C9DF811008DF8720C17
:10C9D0009DF812008DF8730C9DF813008DF8740CFF
:10C9E000002305220DF54761072000F0C3FC0DF67A
:10C9F000844DBDE8F08F70B505460024F5F71AFAAE
:10CA0000FCF701FB012804D02846F5F715FC20B1FE
:10CA10000124F4F7FBFF204670BDF8F745FCEFE773
:10CA20002DE9F74F84B04FF00008C2F82080C2F81B
:10CA30001C80059B934E01274146002B1ED902EB1B
:10CA40004103B3F97030002BB8BF5B421BB2D6F87C
:10CA500000C0BCF9CCC09C450CDD4B0902EB830344
:10CA600001F01F04D3F81CC007FA04F44CEA040CCC
:10CA7000C3F81CC0059B491C9942E0D30021012B3F
:10CA80001CBF059BA3F1010940D002EB4103B3F9A0
:10CA90007240B3F970C0B4EB0C0348BFACEB0403B5
:10CAA0001BB23568B5F9C6509D422CDAB2F9E630B2
:10CAB000BCEB030548BFA3EB0C052DB2B4EB030C94
:10CAC00048BFA3EB040C0FFA8CF39D420DDB4B091E
:10CAD00002EB830301F01F04D3F81CC007FA04F42F
:10CAE0004CEA040CC3F81CC00DE04B1C4FEA531C6D
:10CAF00002EB8C0C03F01F03DCF81C4007FA03F375
:10CB00002343CCF81C30491C4945BED3316891F809
:10CB1000CA30002B7DD091F8CB1014688B4288BFAF
:10CB200019460023DDF814C0BCF1000F84BF491C76
:10CB300000916ED94FF0010EDDF800C04FF00009F2
:10CB40000121CA46BCF1010F52D9DFF838C103FBFD
:10CB50000005DCF800C0CDF80CC0BCF9CEC00295D1
:10CB60000EFB0005019503FB001504EB4505B5F927
:10CB70005080B8F1000FB4BFC8F100054546AC4580
:10CB800036DB0EFB001504EB4505B5F95070002FA0
:10CB9000B4BF7D423D46AC452ADB029D6D1A04EBD5
:10CBA0004505B5F94E60002EB4BF75423546AC451B
:10CBB0001EDB019D6D1A04EB4505B5F94E50002DA5
:10CBC000B4BFC5F1000BAB46E34511DCA7EB080889
:10CBD000039FB7F9C8704745B8BF09F10109AD1BFC
:10CBE000BD42C8BF0AF1010A491C009DA942BAD33F
:10CBF000BAEB090148BFA9EB0A01DFF888C0DCF8ED
:10CC000000C09CF8CAC061450FDB590902EB8101E5
:10CC100000E015E003F01F064FF0010CCD690CFA9F
:10CC200006FC45EA0C0CC1F81CC005995B1C8B4244
:10CC300006D2002B18BFA3F1010E7FF47DAF79E778
:10CC400007B00120BDE8F08F2DE9F04FD2F800C009
:10CC500083B04FF00108DCF8103023F4E023CCF867
:10CC60001030094BD3F800E0064B1EF0010F1B6893
:10CC70002DD00024546625462746CDE90001002426
:10CC800004E00000D4810010DC8100105DF827B0C2
:10CC9000BBF1000F88BF02EB071A15D90AEB440657
:10CCA000B3F9D490B6F9BE63B14503DCB3F9D690BD
:10CCB000B14505DA566E08FA05F946EA09065666E0
:10CCC000641C6D1CA345E9D87F1C022FD7D31EF02E
:10CCD000040F71D00024946625462746CDE9000153
:10CCE0005DF827A00024BAF1000F88BF02EB4719B6
:10CCF00015D909EB4406B3F9D8B0B6F9DE63B345EC
:10CD000003DCB3F9DAB0B34505DA966E08FA05FB31
:10CD100046EA0B069666641C6D1CA245E9D87F1C8A
:10CD2000022FDDD30024D46625462746CDE9000135
:10CD30005DF827A00024BAF1000F88BF02EB471965
:10CD400015D909EB4406B3F9DCB0B6F9EE63B34587
:10CD500003DCB3F9DEB0B34505DAD66E08FA05FB9D
:10CD600046EA0B06D666641C6D1CA245E9D87F1CFA
:10CD7000022FDDD34418D2E91A5030EA050343EA02
:10CD80000506D36612D000210846002C0ED908FAF9
:10CD900000F73B4218BF491C401CA042F7D30129B1
:10CDA00004D145EA030090660020D0661EF0010F12
:10CDB00002D0506EB04350669CF820009CF82110C1
:10CDC0001EF0010F08441CBF516E00291AD0DCF878
:10CDD000101041F48031CCF81010536EDCF8301094
:10CDE00083401943CCF83010516E202839BFC0F170
:10CDF0002003D940A0F120039940DCF834301943D6
:10CE0000CCF83410916ED1B1DCF8101041F400313F
:10CE1000CCF81010936EDCF8381083401943CCF82E
:10CE20003810916E202827BFA0F120039940C0F14F
:10CE30002003D940DCF83C301943CCF83C10D16ECB
:10CE4000D9B1DCF8101041F48021CCF81010D36E69
:10CE5000DCF8401083401943CCF84010D16E2028F4
:10CE600027BF203801FA00F0C0F1200021FA00F0BD
:10CE7000DCF844100843CCF8440003B00120BDE8BE
:10CE8000F08F2DE9F04FABB091460D460446F4F714
:10CE9000BDFD0222209212222192CDE90645F4F72F
:10CEA0007CFF199000F48460F4F759FEFE484FF0BF
:10CEB0000107007810F0210F4ED0FC480090FC488C
:10CEC000019000212098F4F7E7FA029001212098C0
:10CED000F4F7E2FA039000212198F4F7DDFA0490C8
:10CEE00001212198F4F7D8FA0590FF210F20F8F7D7
:10CEF00030FCF4F78BFD002506A850F825B020A8DB
:10CF000050F82500F5F736FB002402A8264609EB69
:10CF1000051A00EBC50818E0600904F01F0158F875
:10CF2000200007FA01F108420ED0E007800C6108EA
:10CF300000EB81015DF825004058F5F721FB0AEB75
:10CF40004601761CA1F8BE03641C5E4538BF262C42
:10CF5000E2D36D1C022DCFD3D348007810F0040F1C
:10CF600000F0C481D3480C90D3480D900220F4F710
:10CF700093F927900220F4F7DFF925900220F4F7C7
:10CF8000B9FC1B902098F4F704FA1A902198F4F752
:10CF900000FA18900220F4F791FA26901220F4F784
:10CFA0008DFA1F900220F4F7C9FA24901220F4F7AA
:10CFB000C5FA1D900AA800900EAB08AA10A92098E7
:10CFC000F4F7DFFB0BA800900FAB09AA11A9219879
:10CFD000F4F7D7FB2098F4F756FC22902198F4F749
:10CFE00052FCB64D01902868B0F8E4100220F4F726
:10CFF00063F900210220F4F765FC286890F8E61038
:10D000002098F4F7D8F9286890F8E6102198F4F7FA
:10D01000D2F900210220F4F76AFA00211220F4F775
:10D0200066FA00210220F4F7A2FA00211220F4F798
:10D030009EFA2868B0F8E8102098F4F7D2FB286828
:10D04000B0F8E8102198F4F7CCFB00210220F4F7A7
:10D050006BFC23902868B0F8EC10009190F8EB304E
:10D0600090F8EA200B212098F4F75DFB2868B0F8CF
:10D07000EC10009190F8EB3090F8EA200B21219809
:10D08000F4F751FB00210220F4F74EFC12A8FFF741
:10D09000B2FC1799002206AC002054F822C0BCF163
:10D0A000000F88BF09EB421308D931F8026B03EB7C
:10D0B0004008401CA8F8DE638445F6D8521C022ABA
:10D0C000EAD32098F3F7ADFB1E902198F3F7A9FB64
:10D0D0001C9000212098F4F7DFF90290012120989C
:10D0E000F4F7DAF9039000212198F4F7D5F90490C8
:10D0F00001212198F4F7D0F905902868B0F8EE10D6
:10D10000009190F8EB3090F8EA200B212098F4F78A
:10D110000AFB2868B0F8EE10009190F8EB3090F818
:10D12000EA200B212198F4F7FEFA00250DF1800B7F
:10D1300000210220F4F7F8FB00212098F3F759FBB7
:10D1400000212198F3F755FB5BF825000121F3F747
:10D1500050FB06A8002450F8250029900CA826466C
:10D1600050F82500289002A800EBC50009EB451AED
:10D17000009044E0009861094FF0010850F8210048
:10D1800004F01F0108FA01F1084237D000221146CD
:10D190001046F4F7D7FB202C23BF0027A4F1200072
:10D1A00008FA00F808FA04F738BF4FF000085BF8F7
:10D1B00025003A460021F4F75DF95BF82500424668
:10D1C0000121F4F757F96FEA0802F9430920F4F74F
:10D1D000B9FB12AFF4F72EFEFBF715FF012804D0C0
:10D1E0003846F5F729F800285DD0F4F70FFC2898A9
:10D1F00000880AEB4601761CA1F8EE03641C29980E
:10D20000864238BF262CB5D3002211461046F4F7CB
:10D2100099FB6D1C022D8BD31E992098F3F7E9FA28
:10D220001C992198F3F7E5FA0021029A2098F4F767
:10D2300021F90121039A2098F4F71CF90021049A9E
:10D240002198F4F717F90121059A2198F4F712F9BA
:10D2500002202799F4F730F802202599F4F777F89F
:10D2600002201B99F4F72EFB1A992098F4F7A3F8E3
:10D2700018992198F4F79FF802202699F4F737F9C6
:10D2800012201F99F4F733F902202499F4F76FF96B
:10D2900012201D99F4F76BF90A9800900E9B089ADA
:10D2A000109920980CE027E0DC810010489E0030A7
:10D2B000E09E00304C1800304C1D0030D48100102E
:10D2C000F4F731FA0B9800900F9B099A1199219865
:10D2D000F4F729FA22992098F4F783FA0199219812
:10D2E000F4F77FFA02202399F4F71EFB1998F4F75C
:10D2F00036FC2BB0BDE8F08FF7F7D6FF6CE70000E7
:10D3000070474FF0FF3070475548406870475449A8
:10D310004860704710B582B007280BD14FEA111C46
:10D32000012404FA0CFC4E4C64681CEA040F04BF90
:10D3300002B010BD9B0100F00F0043EA800040F0F6
:10D3400001008DF800008DF801108DF80220100A00
:10D350008DF80300100C8DF80400100E8DF80500F8
:10D3600000208DF806008DF8070068460EF0DCFE00
:10D3700002B010BD10B59B0100F00F0082B043EA6F
:10D38000800040F001008DF80000072A88BF0722C6
:10D3900000206B46002A09D911F800C01C18401C57
:10D3A00084F801C09042F7D3072805D200211A184B
:10D3B000401C51700728FAD318460EF0B5FE02B093
:10D3C00010BD10B59B0100F00F0082B043EA800051
:10D3D00040F002008DF80000072A88BF07220020D5
:10D3E0006B46002A09D911F800C01C18401C84F8AB
:10D3F00001C09042F7D3072805D200211A18401C1B
:10D4000051700728FAD318460EF08EFE02B010BDF8
:10D4100070B5134E40EA012502283488224618BF11
:10D42000052803D1002918BF022900D12C46A242A9
:10D4300009D051B17088002344EA004290210720AE
:10D44000FFF768FF3480758070BDF6F732F844EA64
:10D450000042002390210720FFF75CFFF2E7000065
:10D46000E0810010FE4908707047FD480078704761
:10D47000FB4948707047FA48407870472DE9F04FF3
:10D48000F848F74E95B000687178836D0229C3F3B0
:10D4900003201AD0726812F4007F1EBFC3F3033159
:10D4A0000F29084612F0800F1EBFC3F303110F2986
:10D4B000084602F00701F7F7A1FF012814BF00207A
:10D4C0000220707040F046820DE000210846F4F71B
:10D4D00069FBF3F760FC30B1E348D0F8401341F446
:10D4E0008031C0F84013F4F758FC1090307910F0F8
:10D4F000100F18BFF5F75CF8307910F0080F03D162
:10D50000FF210F20F8F725F9D848DC49007805906D
:10D51000D74800781190D7480478D748057808781C
:10D52000009048780190119800281CBF05980028A9
:10D5300016D00EF0D6FD0EF0D9FD0020F7F7E8F872
:10D540000020F7F71EF90020F7F73AF9C4480079F0
:10D5500010F0100F0AD00120F7F744F9012009E07C
:10D56000002D18BF002CE4D100F0F4B90020F7F72B
:10D5700039F90020F7F736F9F3F70DFC10F0010F39
:10D5800004BF0120F3F779FEF4F71BFC1E20FCF723
:10D590002EF800210846FBF7A9FF83460121002051
:10D5A000FBF7A4FF119A05998246002001FB02F6C1
:10D5B000002E84BFB2494A0C06D92BF810102AF865
:10D5C0001020401C8642F8D81E20FCF7A9F9002143
:10D5D0000120FBF78BFF012112900846FBF786FF25
:10D5E0008146002065191CBFA54A510C07D0129B2B
:10D5F00023F8102029F81010401C8542F7D81E206F
:10D60000FCF7A8FA00210220FBF770FF80460121F9
:10D610000220FBF76BFFDDE90012074600208C18A3
:10D620001CBF97494A0C06D028F8101027F8102084
:10D63000401C8442F8D80020139089484088002874
:10D6400040F2DA80601C4008691C0C9048080E907B
:10D65000FBF7D9FC012800F0CF8006A8F4F7ECFD19
:10D6600000287CD00798F6F7F6FA0898002845D0ED
:10D670007B48007910F0100F08D0089801900EF048
:10D6800058FD01990EF05AFD019015E0002000238D
:10D69000019002900390049000901A461946089851
:10D6A0000EF051FD01906E48007910F0200F03D06C
:10D6B0000EF03FFD01900AE0F6F73DFB119A009253
:10D6C000019A01461046059B0EF042FD0198002884
:10D6D0001CBF0020002E11D901993BF9102031F90F
:10D6E00010108A42B8BF2BF810103AF910208A4265
:10D6F000C8BF2AF81010401C8642EDD8109810F0D0
:10D70000010F1CBF0A98002833D05548007910F04B
:10D71000400F0A9809D000231A4619460EF01DFD45
:10D720000EF020FD0F9020B30AE00F90F6F7CCFA30
:10D7300002220092DDE90E32014610460EF008FD8D
:10D740000020002D15D90F99129A31F9101032F9D5
:10D7500010208A42BCBF129A22F8101000E043E069
:10D7600039F910208A42C8BF29F81010401C8542A0
:10D77000E9D8109810F0200F1CBF0B9800282DD06E
:10D780003748808810F4807F0B9807D000210EF076
:10D79000EEFC0EF0F1FC0D9000B30AE00D90F6F7F0
:10D7A00079FA02220092DDE90C32014610460EF0B1
:10D7B000CFFC0020002C11D90D9938F9102031F937
:10D7C00010108A42B8BF28F8101037F910208A428A
:10D7D000C8BF27F81010401C8442EDD8F4F789FD2B
:10D7E0001398401C139002E0F7F75EFD13981C4954
:10D7F00049888842FFF42CAFF4F708F90EF076FC64
:10D800000EF079FC16491398498888427DD3109808
:10D8100010F0020F3AD000224FF6FF731046002E90
:10D820000ED93BF910103AF910C0A1EB0C0191424E
:10D83000C8BF0A469942B8BF0B46401C8642F0D882
:10D8400042208DF80000100A8DF80100180A8DF8AA
:10D8500002208DF8043000238DF80300052211E02A
:10D86000E8810010D481001000500040CC800010EE
:10D87000CD800010D1800010D2800010D480001024
:10D880000080FFFF69460720FFF774FD109810F035
:10D89000010F28D000224FF6FF731046002D0FD93C
:10D8A000129939F910C031F91010A1EB0C01914215
:10D8B000C8BF0A469942B8BF0B46401C8542EFD804
:10D8C00043208DF80000100A8DF801008DF8022029
:10D8D000180A8DF803008DF80430002305226946EC
:10D8E0000720FFF747FD109810F0200F29D00022E5
:10D8F0004FF6FF731046002C10D938F9101037F985
:10D9000010C0A1EB0C01914200E01AE0C8BF0A462A
:10D910009942B8BF0B46401C8442EED844208DF893
:10D920000000100A8DF801008DF80220180A8DF809
:10D9300003008DF804300023052269460720FFF715
:10D9400019FDFF20FBF753FEFF20FBF7E9FFFF2047
:10D95000FCF700F9F4F7E2F915B0BDE8F08F70B507
:10D96000224C00206070F4F7DFFAF4F7B2FA0546B3
:10D970000020F4F7A8FAFBF746FB012803D1F7F7DC
:10D980003BFC03281BD1207810F0010F07D0FEF7D5
:10D990002DFC207820F001002070FBF7EDFA2078B4
:10D9A00010F0020F07D0FFF769FD207820F0020089
:10D9B0002070FBF7E1FAF7F71FFC032807D0284691
:10D9C000F4F781FABDE870400120F4F7ADBAF7F73B
:10D9D0006BFCD0E705494860002048707047034859
:10D9E000406870470149488070470000E881001096
:10D9F000FB4908707047FA4800787047F848007A89
:10DA00007047F74800210172C1717047F4494872AC
:10DA10007047F348407A7047F14982B2CA61C0F357
:10DA20000742C0F303604A61487088700020886133
:10DA30007047EB4840797047E94A0028D16914BF24
:10DA400041F0020021F00200D0617047E448007FFD
:10DA5000C0F340007047E24A10F0010FD06914BFD4
:10DA600040F0020020F00200D0617047DC49002045
:10DA7000097FC1F34001002918BF01207047002829
:10DA8000D74AD16914BF41F0010021F00100D061F3
:10DA90007047D348007F00F001007047D0494A78B2
:10DAA0008A7048707047CE4840787047CC4880787C
:10DAB0007047CC480068406DC0F303607047012197
:10DAC0008140C7484269114041617047012181404E
:10DAD000C348426922EA010141617047C048406978
:10DAE0007047BF4880697047BD4910B58C6988612F
:10DAF0000246002381210720FFF70CFC204610BDC1
:10DB0000B748808BC0F380207047B5490120486238
:10DB10007047B349C872704710B5B14C60B906F090
:10DB200007F908281CBFE07A022805D00120E0721E
:10DB3000F4F7C6F9206210BD0020E07210BD2DE997
:10DB4000F041A74D0024E87A012802D02046BDE824
:10DB5000F081F7F751FB8046F7F754FB00260746A4
:10DB6000B8F1020F1CBF0124EE72EFD1F4F7A8F94F
:10DB70000146286A88429CBF081AB0F5966FE5D323
:10DB80000124022F14BFEE720024DFE79448C07A0C
:10DB9000012818BF002070479148007FC0F3800023
:10DBA00070478F48007FC0F3C00070478C48808B5F
:10DBB000C0F3002070478A48808BC0F34020704734
:10DBC0008748007FC0F3C0107047FCF70FBD844842
:10DBD000818B11F4005F04D1C07A01281CBF0020A2
:10DBE0007047012070477E48808BC0F3C02070478B
:10DBF0007B48808BC0F30030704770B5784E054687
:10DC0000C0F34020F469C4F3403188420CD0F0B92D
:10DC100006F08EF808281CBFF07A022817D00120E1
:10DC2000F072F4F74DF9306215F4807F14BF44F4BC
:10DC3000806124F4806115F4007F14BF41F400502A
:10DC400021F40050F061BDE87040FCF7B4BE002044
:10DC5000F072E9E770B5624E0446C0F38000F569E2
:10DC6000C5F3002188421DD00120F6F7C0FC14F056
:10DC7000040F07D005F0F1FF012839D005F0EDFFC2
:10DC8000082835D00120F4F71EF914F0040F03D052
:10DC900005F0E3FF01282FD0534890F86C00C0082E
:10DCA00002F067FF14F0040F08BF25F4807001D064
:10DCB00045F4807014F0080F14BF40F4007020F495
:10DCC000007014F0100F14BF40F4006020F40060E6
:10DCD00014F0400F14BF40F4805020F4805014F032
:10DCE000200F14BF40F0800020F08000F06170BD74
:10DCF0000020F4F7E8F8CBE7002002F03AFFD7E77E
:10DD00003748C169002011F0040F18BF012011F03D
:10DD1000080F18BF40F0020011F4807F18BF40F0D8
:10DD2000040011F4007F18BF40F0080011F4006FE8
:10DD300018BF40F0100011F4805F18BF40F04000A1
:10DD400011F0800F18BF40F0200070472448006B8E
:10DD5000704723498A6A10438862704770B5204E25
:10DD6000B06A40F400640020B062F56915F0040F59
:10DD700018BF44F0010415F0080F18BF44F0020466
:10DD800015F4807F18BF44F0040415F4007F18BF19
:10DD900044F00804FCF72AFC002818BF44F48074FF
:10DDA00015F4006F18BF44F0100415F0800F18BF71
:10DDB00044F0200415F4805F18BF44F0400415F4CB
:10DDC000005F02D1F07A012801D144F40074B169F6
:10DDD00044EA0140002918BF40F4805070BD0000A3
:10DDE000F0810010D4810010E4F80010FE49C862F0
:10DDF0007047FD4890F82C0000F001007047FA4889
:10DE000090F82C00C0F340007047F74890F82C00C1
:10DE1000C0F380007047002818BF0120F249487302
:10DE200070472DE9F041F14980000968896D21FAB8
:10DE300000F000F00F04C1F30327C1F30335C1F371
:10DE40000316BC4241D10F2D3FD0DFF89C83B8F8B8
:10DE50001C0010F4005F03D198F80B00012803D1D7
:10DE600005F066FF082810D1B8F81C00C0F30020A8
:10DE700038B105F0F2FE012807D005F0EEFE0828C3
:10DE800003D005F061FF022800D12C46D8F85000DD
:10DE9000A0421AD005F04CFF0146AC420CBF012055
:10DEA000002040EA012505F0D8FE45EA004505F0CE
:10DEB0004BFF45EA0062002384210720FFF72AFA7E
:10DEC0000020C8F85040F6F792FBF7F775FA20B13A
:10DED000BC4202D10F2E18BF34462046BDE8F08167
:10DEE0002DE9F047002586B02E46F7F785F9BF49A2
:10DEF000052808680CBF90F8F80090F8580000F06A
:10DF00000F094846FCF730FEB74F4FF0000A4FF0BC
:10DF10000108002808BF54460ED0446AB88BC0F3ED
:10DF2000002038B105F099FE092861D005F095FE72
:10DF30000A285DD087F80CA014F0010F14BF02244A
:10DF4000042444F400314846F7F758FA002804BF87
:10DF500006B0BDE8F08714F0040FA54C07D0F2F727
:10DF600042FC01462078814288BFF2F734FC012050
:10DF7000F3F783F9F3F75EFFFBF745F8012843D089
:10DF80006846F4F759F900283AD06846FBF704FFD1
:10DF90000198F5F760FE029880B1964821780078E4
:10DFA000400000FB01F2944802990EF02CF89348CF
:10DFB0000078492804BF9048FBF7C1FB049888B15A
:10DFC0008F48049C01788F4800780A185200214637
:10DFD0008D480EF018F88D4A1278492A04BF204661
:10DFE000FBF7B8FC87F80D80F4F783F901260BE006
:10DFF00014F0020F18BF24F0010487F80C809BE78F
:10E00000F7F752F9002DB7D0F3F700FDF7F765FBEE
:10E0100006B03046BDE8F0877348407B002818BF43
:10E02000012070472DE9F04F4FF0000A87B00446F9
:10E03000D146F7F7E1F80746F7F7E4F8DFF8A8B1BB
:10E040000690052F07D1FCF7C5F8002804BF002073
:10E050008BF80D0002D09BF80D0008B9FFF740FFC8
:10E06000052F0CBFDFF8A881DFF8A8810F2120461B
:10E07000F7F7C4F9002804BF07B0BDE8F08F0EF031
:10E0800030F8F6F753FA04007DD10125F2F783FE4C
:10E0900006460020F3F7F1F82846F3F7ABFE5248A6
:10E0A0000564F5F709FAA5F1010BFAF7ACFF0128B1
:10E0B0000AD0F7F7A1F8B84206D1F7F7A3F8069906
:10E0C000884208BF002C09D0F3F7A0FC464F16F099
:10E0D000010F7D7834D0012C27D031E06846F4F769
:10E0E000ABF8F8B116F0010F03D00120F5F728FCCA
:10E0F00082466846FBF750FE0198F5F7ACFD68468E
:10E10000C0470446F4F7F5F8002CCED115B90198B4
:10E110005845CAD1F3F778FC002804BF2846F3F726
:10E1200069FEC2E7F7F7B5F8BFE70120F5F708FC8D
:10E13000504505D2AAEB00010120F5F711FC8146FC
:10E14000F5F7DFF916F0010F29D0012C27D1B9F12D
:10E15000000F24D0F2F7D8FF0446F2F72DFE00EBB3
:10E16000800004EB40004844002144F20902904240
:10E1700084BFA0F580400938002D08BF43F639015F
:10E1800005D0022D00E00AE008BF41F6F9018842FF
:10E1900005D2091A0120F5F712FC0120B8720DF022
:10E1A000AAFFF7F79AFA07B0BDE8F08F2DE9F14F13
:10E1B00088B000260396049606960296F7F71CF898
:10E1C00001900C48B046C1460478094823460A49E4
:10E1D0000578089804FB05FA00EB4A07024600950B
:10E1E00038460DF0B5FF17E0F0810010D481001023
:10E1F000CD800010CC80001080FC00103D8100100C
:10E20000D2800010D18000107002011042810010F5
:10E21000D53100104D360010DFF8F4B39BF8000044
:10E22000492804BFFB48FBF78AFAF94800784C28D4
:10E2300004BF3846FBF783FA07EB4A0293464FF0D8
:10E24000000C002D25D90020611E13D007EB410ED4
:10E2500037F811303EF802ECA3EB0E031BB2002B93
:10E26000B8BF5B421BB222F811308342C8BF1846C8
:10E27000491EEBD10199022919D0108007EB440700
:10E2800002EB44024045C8BF80460CF1010CAC458E
:10E29000D9D3E148B0F9100005908045A4BF01260C
:10E2A0000396002E04BF0198022845D10BE002EB33
:10E2B000440131F9023C142BB9BF31F9041C142973
:10E2C00001260396D9E7D448007B00281CBF002212
:10E2D000002D88BF6B462FD902FB04F00BEB4000EA
:10E2E000018EADF80010818EADF80210018FADF8EF
:10E2F0000410B0F93C70ADF80670002003EB400C40
:10E3000033F81010BCF802C06144DDF814C009B243
:10E31000614503DB0126884602960AE0401C03287B
:10E32000ECDB36B9142F04DB0126BDF9068002961A
:10E3300002E0521CAA42CFD30BEB4A034FF0000C71
:10E34000002D25D90021601E022812D90BEB4002B6
:10E350003BF8107032F802EC32F8042C77443A445F
:10E3600012B223F810208A42C8BF1146401E02286C
:10E37000ECD800201980588098800BEB440B03EBFD
:10E3800044034945C8BF89460CF1010CAC45D9D3BB
:10E39000A14BB3F912209145A4BF01260496002E8B
:10E3A00014BF986CD86C00F1010014BF9864D86455
:10E3B00097480078FF2842D008980127002E20F8BF
:10E3C0003A600898039900EBCA0041800499818063
:10E3D0000299C18006990181996C4FEAE17C01EBB9
:10E3E0001C5C6FF30B0CA1EB0C014181D96C4FEA63
:10E3F000E17C01EB1C5C6FF30B0CA1EB0C01818148
:10E40000A0F80E80A0F81090197B418205998182B6
:10E41000C2824FF00208089907EB85032246CDF827
:10E4200000800CBF4E204D20FBF72BF907EB850336
:10E430002246CDF8008047200899FBF722F909B061
:10E440003046BDE8F08F754870472DE9F04FDFF892
:10E45000C8A183B083460025BAF91080714872497B
:10E460000095007809782E466D4C4718F3F795FC17
:10E4700001906E48A4F174090078492804BF484609
:10E48000FBF768FA0020002F09D93BF8101039F883
:10E490001020891A24F81010401C8742F5D8DFF8A4
:10E4A0008C9199F800004C2804BF2046FBF752FAE3
:10E4B000019810F4007FA7F1010011D0002818BFC7
:10E4C000BAF9123025D034F910100029B4BF4A42ED
:10E4D0000A469A42BCBF0D44761C401EF3D118E098
:10E4E000002818BFBAF9123013D004EB400234F8F8
:10E4F000101032F8022C891A09B224F810100029E1
:10E50000B4BF4A420A469A42BCBF0D44761C401E24
:10E51000EBD1002EC8BF95FBF6F52EB2268099F8F8
:10E5200000004F2804BF2046FBF714FA0025781E90
:10E530000ED034F81010891B09B224F810100029ED
:10E54000B8BF494209B28D42B8BF0D46401EF0D156
:10E550002580BAF81C00C0F3002048B105F07DFB0F
:10E56000012803D005F079FB082801D14FF00508F8
:10E57000454506DD0120009099F800004D2807D19F
:10E5800003E099F800004E2802D12046FBF7E2F99B
:10E5900099F80000472804BF2046FBF7DBF90098F4
:10E5A00003B0BDE8F08F2DE9F04F87B0FBF7DAFF3D
:10E5B0001F480068B0F93610B0F934000DF073FD53
:10E5C0000120F6F714F8144FB88BC0F3002038B1CF
:10E5D00005F043FB01282DD005F03FFB082829D08A
:10E5E0000120F3F770FC387D10F0100F06D00420E6
:10E5F000FFF717FC0F2818BFF5F7DDFFFF20B871F4
:10E6000008F028FEF6F7F8FD022815D0AEE000006D
:10E610003D81001080FC0010F0810010700201109C
:10E62000E4020110D2800010D1800010428100105D
:10E63000D48100100020D4E7DFF8A4A1DFF8A4B152
:10E640004FF000084FF0E0297C78C7F8388020466A
:10E65000C7F83C80FFF7E5FB054621460220FEF7A0
:10E66000D7FE052C75D2DFE804F06D0303037100BB
:10E670007E780F212846F6F7C1FE002869D00DF0FC
:10E6800030FD0DF033FDF5F751FF05002FD138783F
:10E6900000281CBF0001F2F74BFD0024F3F77DFBBF
:10E6A0000690F2F778FB10F0010F0ED0F2F7DFFDC5
:10E6B00002280AD3B87A40B1069840F40030F3F744
:10E6C0004EFA0124F3F7B6FB01E0F3F77AFB87F883
:10E6D0000A8087F80380FAF796FC012807D0F6F73E
:10E6E0008BFD022802BF7878B042002D06D00DF0D5
:10E6F000FDFC0DF000FDF6F7F0FF2AE06846F3F7A9
:10E700009BFDE0B12CB1641E0698F3F728FAF3F7ED
:10E7100058FB6846FBF740FB0198F5F79CFA684602
:10E720000DF02FFD05469AF8000028B1D9F8180021
:10E73000CBF80000C9F81080F3F7DBFDCBE7F6F764
:10E74000B3FDC8E728460DF0E0FC02E02846FFF7DD
:10E7500069FCFAF758FC012803D1F6F74DFD0228B1
:10E7600004D1F6F749FD02283FF46EAF0AF0CCF968
:10E77000F5F73CFF07B0BDE8F04FFBF7F3BE4A00EA
:10E78000014619480DF03FBC10B58168044679B1C7
:10E790001648174A007812784000424315480DF099
:10E7A00032FC15480078492804BF1248FAF7C7FF21
:10E7B000246984B111480178114800780A18520080
:10E7C000214609480DF01FFC0E4A1278492A04BF61
:10E7D0002046FBF7BFF801200B49487310BD00002D
:10E7E000208000108880001070020110CC80001082
:10E7F000CD80001080FC00103D810010D280001000
:10E80000D180001042810010F08100103E4A30B4E7
:10E81000146894F86CC01CF0040F1ABF012222EA9D
:10E820000C050CF00105B0F90030B1F900201DB164
:10E83000E58AAA1A521E12B21CF0020F03D0A48A53
:10E84000E31A5B1E1BB21CF0040F19BF02800B8081
:10E8500003800A8030BC70474FF6FF71A0F8B010FB
:10E86000A0F8B210A0F8B410A0F8B61070472DE9C7
:10E87000F05F16468A46834605F0BAF9074605F06A
:10E88000AFF900F15009002E18BF002588BF4FF6E0
:10E89000FF780FD098BFBDE8F09FC5EB051007EBE0
:10E8A000001494F8E000012804BF94F893000028B5
:10E8B00012D103E0BDE8F05F02F0C4B8A4F8B08064
:10E8C000A4F8B280A4F8B480A4F8B68023464A46DF
:10E8D0005146584602F000FE94F8ED00022818BF99
:10E8E00003280DD0B4F8B000A4F8B400B4F8B20016
:10E8F000A4F8B600681CC5B2B542CED3BDE8F09FFF
:10E90000204601F0CAFEF5E7EC820010FE48407890
:10E91000002818BF01207047FC48006890F870007C
:10E9200000F001007047F94909680A6F60F30002BE
:10E930000A6770472DE9F001F4491025402680242C
:10E94000F14A09684FF0200C670010B301284ED03F
:10E9500002281CBFBDE8F0017047488A322300FB43
:10E9600003F84B8BB8FBF3F808FB08F8C2F81080EB
:10E9700000EB001808EB4010B0FBF3F0404350618F
:10E98000486F000F062821D2DFE800F0201C202568
:10E99000292D488A4B8B4FEA0018C000B8FBF3F8CA
:10E9A000B0FBF3F008FB08F84043C2E90480B1F87B
:10E9B0007400C0F30330062808D2DFE800F0070334
:10E9C000070C10145580BDE8F0017047A2F802C092
:10E9D000BDE8F00170475680BDE8F00170475480F3
:10E9E000BDE8F00170475780BDE8F0017047488AE4
:10E9F000498BC0EB00135B00B3FBF1F35B43136186
:10EA000000EB4003C3EB4010B0FBF1F0404350611A
:10EA10005480BDE8F001704710B5BC48BA4C00689E
:10EA200090F87C20418A408B4A43B2FBF0F201EB24
:10EA300081014900B1FBF0F04043E260A061002099
:10EA4000FFF778FF04F120014FF6FF70088048803F
:10EA5000091F4FF0FF30088048800020207010BD53
:10EA60002DE9F04F8DB01F46DDE916860D460446B0
:10EA700005F0B6F8029005F0CFF80B90A2484FF4DD
:10EA8000A051A24AB0F802A0CDF8288001910169F6
:10EA9000049140690390029890F80C801068B8F1D6
:10EAA000000F418A26D0408BC900B1FBF0F04043F3
:10EAB000089010686421428A438B5143B1FBF3F103
:10EAC0004943079102EB8201B1FBF3F149430991FC
:10EAD00094F899C08E491CF801900A31B9F1000FE1
:10EAE00010D0B9F1010F11D0B9F1030F08BF1CF814
:10EAF00001100FE0408B01EB4101B1FBF0F040430E
:10EB00000890D6E71CF8011021B904E01CF80110A8
:10EB100001292FD001210091DFF8F88194F8ED1040
:10EB2000A8F10A03A3F10A0902291CBF94F8BB103B
:10EB3000012934D0784901EBCC0252E90212B5F830
:10EB400000C0CDF818C0B5F802C0CDF814C094F8D4
:10EB5000CCC0BCF1000F57D094F89AC0CCEB0C1B82
:10EB6000DDF82CC00CEB0B1C9CF8CCC0BCF1000FEA
:10EB700039D06CE001210091B8F1000FCCD002EB4C
:10EB8000C20101EB0211B1FBF3F14943049102EB25
:10EB90004201C900B1FBF3F149430391BCE7298865
:10EBA0006A884FF0000B0CF809B094F899C00CF883
:10EBB00003B094F899C00CF808B094F899E0DFF825
:10EBC0005CB1DDF804C00BEB4E0B2BF802CC94F8D3
:10EBD00099C0BCF1010FB2D1DFF82CB14FF0000C9D
:10EBE0008BF801C0ABE794F899B0DFF830C10CEBBB
:10EBF0004B0C3CF802BCB34529D92CF8026C94F8B4
:10EC0000CCC0BCF1000F22D1DDF81CC0674594F8E0
:10EC1000EDC015D3BCF1020F12D0DDF81CC0674562
:10EC200015D394F899E0DFF8F4B094F8CCC00BEB6E
:10EC30004E0B3BF802ECB64588BF2BF8026C08E09F
:10EC40004FF4A06B4FF0020CCDF804B001E094F843
:10EC5000CCC0DDF820B05F4538BF4FF0020CDFF8C4
:10EC6000A8B09BF801E0BEF1000F01BF94F899E055
:10EC7000BEF1010F94F8CCE0BEF1030F0DD14FF0BF
:10EC8000010E8BF801E0DFF894B0BBF800B0B3459B
:10EC900084BFDFF888B0ABF80060DDF810B05F45E6
:10ECA0001DD3BCF1020F1CBFDDF800B0BBF1000F9B
:10ECB00015D094F899E04FF0000B0EF803B094F8DB
:10ECC00099E00EF808B094F899B01BF809E0BEF18D
:10ECD000640F3CBF0EF1010E0BF809E053E0DDF8C4
:10ECE0000CB05F4502D2BCF1020F37D1DDF800B0A5
:10ECF000BBF1000F32D0DDF80CB05F4524BFDDF86A
:10ED000010B0BB453CD90BE044820010EC820010EF
:10ED1000D9030110BB03011058030110C6030110F1
:10ED2000BCF1020F51D094F899B01BF808E0BEF185
:10ED3000000F28D04FF0000E0BF809E094F899B0BE
:10ED40000BF808E094F899B01BF803E0BEF1640FEB
:10ED500019D20EF1010E0BF803E014E094F899E0DB
:10ED60004FF0000B0EF809B094F899E00EF808B0D7
:10ED700094F899B01BF803E0BEF1640F03D2E8E702
:10ED8000BCF1020F21D094F899B01BF8033093B373
:10ED9000DFF8DC9406EB460309EB4B0838F802BCBD
:10EDA0009B4508D9DDF808B09BF80CB0BBF1000F0B
:10EDB00008BF28F8023C94F8993009EB430838F86A
:10EDC000023CB34230D365D94DE094F899E04FF05E
:10EDD000000B0EF809B094F899E00EF803B094F81F
:10EDE00099B01BF808E0BEF1640F3CBF0EF1010EB4
:10EDF0000BF808E0C7D30BF0FF0313F80990B9F143
:10EE0000000F33D0DFF8689409EB430838F8023C70
:10EE1000B34206D9DDF808B09BF80CB0BBF1000F87
:10EE200006D00A9EB3421DD2534428F8023C31E07A
:10EE3000A3EB0606A3EB66039BB228F8023C94F80A
:10EE400099604FEA132309EB46064FF6FF7826F840
:10EE5000023C94F8996008EA032309EB460626F879
:10EE6000023C17E016D9A3EB0A03DEE713F80860AB
:10EE7000012E0FD9FE4EDDF8048006EB430636F86E
:10EE8000023C434588BFA3EB0A0338BF534401D07B
:10EE900026F8023C94F89930F54E009306EB4303B4
:10EEA00033F8023C002B08BF00207AD01E46B3F591
:10EEB000807F3CBF4FF480763346BCF1020F1CBF0D
:10EEC000DDF824C067456DD81F0A029B360A93F807
:10EED0004230022B1CD3B0F818A0069BB0F810905B
:10EEE0000AFB03F3B3FBF9F3B0F81AE0DDF814C042
:10EEF000B0F812800AFB01FA0EFB0CFCBAFBF9F920
:10EF0000BCFBF8FC0EFB02FABAFBF8F88B461BE0E0
:10EF1000B0F814A0069BB0F810900AFB03F3B3FB03
:10EF2000F9F3B0F816E0DDF814C0B0F812800AFB6F
:10EF300001FA0EFB0CFCBAFBF9F9BCFBF8FC0EFB6A
:10EF400002FABAFBF8F88B46A6F1010A0AFB09336C
:10EF5000B3FBF6F6A7F1010303FB08C3B3FBF7FC11
:10EF6000078A07FB06F308D3078BB0F812A0B3FBA0
:10EF7000F7F30AFB0CF7408B07E0878AB0F812A082
:10EF8000B3FBF7F3C08A0AFB0CF7B7FBF0F04E4572
:10EF900018BFC44535D14E4508BF5B46C44508BFC0
:10EFA00010462EE0B0F81480078ADDF818C008FB80
:10EFB00001F108FB0CFCBCFBF7F9B0F816C0B1FB83
:10EFC000F7F1408AA6F5807B0BFB01F101EB0921EB
:10EFD000DDF814A0B1FBF6F10CFB02F20CFB0AFA0F
:10EFE000B2FBF0F2BAFBF0FAA3F58076724302EBC3
:10EFF0000A22B2FBF3F279435043B1FBF8F3B0FBC2
:10F00000FCF09C49009A01EBC20242F8083C94F8DB
:10F01000992001EBC20141F8040CAB80E8800DB0EF
:10F02000BDE8F08F2DE9F84F9349944B01444FF020
:10F03000000E01F801EC0344012103F8011C904982
:10F04000744601EB401100918E49724601EB401B62
:10F0500001F5A07101EB4019009800210BEB041899
:10F0600009EB041700EB0416002008EBC10307EBC3
:10F07000C10C06EBC10503EB800A4AF8202C0CEB0F
:10F08000800A4AF8202C05EB800A401C00B24AF89E
:10F09000202C0228EFDB481C01B20229E4DB601CB3
:10F0A00004B2022CD8DB7848784E0021D0F800C09A
:10F0B000A6F110070BEB0E1809EB0E1A002006EB59
:10F0C000C10908EBC1050AEBC10407EBC10381428A
:10F0D00007D1BCF87A2043F82020BCF8782049F802
:10F0E000202053F8202005EB800B02EB8202520017
:10F0F0004BF8202C04EB800B401C00B24BF8202C6A
:10F100000228E4DB481C01B20229D7DBBDE8F88FF6
:10F1100010B490F899C05E4C00230CF8043090F8BD
:10F1200099C00A340CF80430574B90F899C01B680A
:10F1300093F87430C3F303131B02153404EB4C0C27
:10F140002CF8023C90F899C0A4F16E0303EBCC0CB0
:10F150004CF8081C90F8991003EBC10141F8042CFD
:10F1600090F8990010BC5DE710B5044604F054FD1A
:10F1700001464848C26894F8ED00022804BFB4F87C
:10F18000B410B4F8B60009D094F89A00C0EB00109F
:10F1900001EB0010B0F8B410B0F8B60094F8CC3021
:10F1A000022B18BF10BDB4F8B4C0BCEB010348BFBC
:10F1B000A1EB0C03934228BF10BDB4F8B6C0BCEB62
:10F1C000000348BFA0EB0C0393423CBFA4F8B4106B
:10F1D000A4F8B60010BD2DE9F04F83B0044604F04A
:10F1E0001BFD2948B4F8B690B4F8B4A00068DFF865
:10F1F000A8B0B0F81880078A468B458A09FB06F24A
:10F2000092FBF5F00AFB08F191FBF7F194F8ED2081
:10F21000ABF1200E022A68D09EF800C0BCF1000FAE
:10F2200000F0EF80BCF1020F7ED2BBF8002001920B
:10F2300002FB08F292FBF7F9BBF80220009202FBF6
:10F2400006F292FBF5FAB1EB090348BFA9EB010303
:10F25000B0EB0A0248BFAAEB0002142BB8BF142A75
:10F260007EDADFF838B0BBF900E0AEF57F4B17E08F
:10F27000C603011058030110F8080110020901101B
:10F28000B807011038050110EC820010A0820010B0
:10F29000A7030110448200106482001060820010F5
:10F2A000BBF1FF0B6CD04945FC4981FB03314FEAB0
:10F2B0006103A3EBE1730199D4BFC91A1944F84B58
:10F2C0005045F648198080FB02104FEA6001A1EB1F
:10F2D000E0710098CCBF0844401AF14948800846C4
:10F2E0000188A4F8B410408875E0BBF800C00CFB9E
:10F2F00008F292FBF7F7BBF8028008FB06F292FBDC
:10F30000F5F5CA1B48BF7A1A431B48BF2B1A142AAB
:10F31000B8BF142B30DAACF57F46FF3E2CD0B94293
:10F32000DE4981FB022100E034E04FEA6102A2EBFA
:10F33000E171D4BFACEB01016144D94AA842D7487E
:10F34000118080FB03104FEA6001A1EBE070CCBF9D
:10F350004044A8EB0000D24948800846018800E0FC
:10F360000EE0A4F8B4104088A4F8B60001208EF88E
:10F37000000003B0BDE8F08F00208EF8000040E0F0
:10F38000C84ABCF1010F04BF0223137003D003B0BD
:10F39000BDE8F08F2FD1DFF80893B9F90020B9F953
:10F3A000023002FB08F2734392FBF7F293FBF5F392
:10F3B000B1EB020C48BFA2EB010CC11A48BF191AED
:10F3C000BCF1060FB8BF06290ADAB9F80000A4F8A4
:10F3D000B400B9F80200A4F8B60003B0BDE8F08F9D
:10F3E000B4F8B400A9F80000B4F8B600A9F8020017
:10F3F00003B0BDE8F08FBCF1000F1CBF03B0BDE847
:10F40000F08FABF800A0ABF8029003B0BDE8F08F2E
:10F410002DE9F04F90F899C08FB04FF48063002928
:10F420000CBFA14CA14C04EB4C14A14D029205EB76
:10F430004C1705F5A5756544203C15F8015C07EBF4
:10F44000051606EBC10858F8206C921B039290F841
:10F45000ED20022A1CBF90F8BB0001287DD058F88F
:10F460001C8C04EB051206EB0809CDF83890D2F895
:10F470000490D6689568106809EB0602DFF83492AC
:10F4800028441044D9F800A035445044D9F804A0C9
:10F49000DFF824B25244D9F808A0D9F80C905544AA
:10F4A0004E44DDF808A0DDF83890AAEB0909CDF844
:10F4B0002090DDF80C90A9EB0809CDF82C90DBF832
:10F4C00000908144CDF82890DBF8049009EB020A03
:10F4D000DBF80890DBF80CB0A9440BEB060EDDF866
:10F4E00028B00BFB0EFB0AFB19BB9BFBF3FBBBF12C
:10F4F000000F08BF4FF0010B4FEA8E2E4FEA8A2A09
:10F500009AFBFBFA4FEA892999FBFBF99EFBFBFE6C
:10F51000CAF1000ACDF834A0DDF828A0C9F100092D
:10F520004FEA8A2A9AFBFBFB00FB0EFA02FB09AAB0
:10F530009AFBF3FACDF828A0DDF834A000FB0AFA14
:10F5400002FB0BAA9AFBF3FACDF824A005FB0EFAF6
:10F5500006FB09A999FBF3F900E05BE0DDF834A0B4
:10F56000CDF8309005FB0AF906FB0B9999FBF3FBEC
:10F57000DDF828A0DDF820900AFB09FEDDF824A0C4
:10F58000DDF82C900AFB09EEDDF820A0DDF83090C4
:10F590009EFBF3FE09FB0AFADDF82C900BFB09A990
:10F5A00099FBF3F9DDF838A0C844F244CDE900A88E
:10F5B000DDF828A0CBF5806ECAF5806808FB00FB5B
:10F5C000DDF824A0DDF83090CAF1000AC9F1000985
:10F5D0000AFB05BB08FB02F809FB00F00AFB0688E2
:10F5E0000EFB05009BFBF3FB98FBF3F890FBF3F09D
:10F5F000CDF810B0CDE9058009FB02F00EFB060046
:10F6000090FBF3F007902D480022E84604AE00EB93
:10F610000C0315E0294A00206244039012F8012CE3
:10F6200002AB07EB021202EBC10253F8204002EBDF
:10F630008005401C00B245F8204C0228F5DB20E094
:10F6400013F8015C58F8220007EB051505EBC1051E
:10F6500005EB820545F8200C002006EBC20513F8E7
:10F6600001AC55F8209004EB0A1A0AEBC20A4AF8DA
:10F670002090401C00B20228F1DB501C02B2022A8A
:10F68000DEDB0E48604410F8010C07EB001000EBC5
:10F69000C10050F8200C0FB0BDE8F08F67666666B9
:10F6A00060820010448200103805011078060110B5
:10F6B000B807011090820010A0820010F808011015
:10F6C0000288438862F30F01808863F31F419A42E6
:10F6D00084BF63F30F0162F31F410A0C824288BFAB
:10F6E00060F31F4188B20A0C904284BF62F30F019D
:10F6F00060F31F41080C704730B51546024690F87C
:10F70000EDC090F89900FE4B2C88698800EB400012
:10F7100003EB8000BCF1020F1CBF92F8BB20012A52
:10F7200020D0844630F80A0C2CF8080C3CF80C0C5D
:10F730002CF80A0C2CF80C4C3CF8040C2CF8020C9D
:10F740003CF8060C2CF8040C2CF8061CACF10C0050
:10F75000FFF7B6FF0446ACF10600FFF7B1FFAC803F
:10F76000E88030BD20F8084C20F80A4C20F80C4CFA
:10F7700020F8021C20F8041C20F8061C0846EEE7BE
:10F7800030B4002488B0A44601EB001101EB4C001A
:10F7900030F8100C04440CF101001FFA80FCBCF19D
:10F7A000080FF3D3E4081C60002318466D4601EBF4
:10F7B000400C3CF810CCACEB040C0CFB0CFC45F8FA
:10F7C00020C0401C80B263440828F0D3D80831F828
:10F7D0000A3C31F8101C591A4943116008B030BC7A
:10F7E0007047C84A0021024402F8011CC64A02447C
:10F7F00002F8011CC54A024402F8011CC44A02EB8B
:10F80000800242F8041CC34A02EB800242F8041C46
:10F81000C14A02EB800242F8041CC04A02EB80029B
:10F8200042F8041CBE4A02EB400020F8021C418052
:10F8300070472DE9FF4FE1B053B200225792B94A09
:10F840001F461268B2F812C0528BCCEB0C1CBCFBEA
:10F85000F2F25092AD4ADFF8B0C2024412F8016CE5
:10F860000CF10202844402441CF8015C12F8014CC1
:10F8700000EB800C01EB0C1C002E7DD00CEB450145
:10F8800031F8505C5495B1F85010539112F8011CA6
:10F89000143949B20029BCBF283149B20CEB4101EF
:10F8A00031F8502C5292B1F850101E2251910CEBAD
:10F8B0004401052A31F8504C5994B1F85010589130
:10F8C00040F2E6819249EE4601EB800151F8044C8A
:10F8D00090495E9401EB8000012150F8040C5B908C
:10F8E000844268DD649800885A90501E58BF744660
:10F8F00012D40CEB430544F8201004EB80065B1E89
:10F9000035F8505C5BB2C6F8A050002BB8BF272377
:10F91000401E00B20028ECDA00210C46B846501E0A
:10F9200058BF754616D40CEB480355F82060B3F861
:10F9300050307343A8F1010659184FFA86F844EB8A
:10F94000E374B8F1000FB8BF4FF02708401E00B2B3
:10F950000028E8DA00252E46501E58BFF1467DD417
:10F960000CEB470309EB8008B3F85030D8F8A080BF
:10F970007F1E03FB08F300E00BE05D197FB246EB4E
:10F98000E376002FB8BF2727401E00B20028E7DA31
:10F9900067E0611CCAB23CF8501C5491BCF850108E
:10F9A000539125F00101614431F8505C5295B1F852
:10F9B000501051917BE76E9800885A90501E58BFA6
:10F9C000744612D40CEB430544F8201004EB800677
:10F9D0005B1EB5F850505BB2C6F8A050002BB8BF04
:10F9E0002723401E00B20028ECDA00210C46B9465D
:10F9F000501E58BF754616D40CEB490355F82060CD
:10FA000033F8503C7343A9F1010659184FFA86F9AF
:10FA100044EBE374B9F1000FB8BF4FF02709401E63
:10FA200000B20028E8DA00252E46501E58BFF146E5
:10FA300017D40CEB470309EB800833F8503CD8F897
:10FA4000A0807F1E03FB08F35D197FB246EBE376CF
:10FA5000002FB8BF2727401E00B200E001E00028B9
:10FA6000E7DA0027B8463846002AC8BFF4460ADD60
:10FA70005CF8203000F101005B43DF1948EBE378CC
:10FA800000B28242F4DC0023CDE955331846002A47
:10FA9000C8BFF44615DD0CEB80095CF82030D9F8BE
:10FAA000A09003FB09F3DDE955A94FEAE37B13EBD3
:10FAB00009034BEB0A09401CCDE9559300B2824281
:10FAC000E9DC4FF0000AD1465046002AC8BFF34691
:10FAD00010DD0BEB80035BF820C0D3F8A03000F101
:10FAE000010003FB0CF313EB0A0A49EBE37900B2C4
:10FAF0008242EEDC4FF0000CE3466046002A13E041
:10FB00000C0901104A820010488200104C8200103B
:10FB100080820010888200106882001070820010BD
:10FB200078820010EC8200100EDD6B4603EB800340
:10FB300000F10100D3F8A03000B25B4313EB0C0CD2
:10FB40004BEBE37B8242F0DCA7FB0C32CDE95CCBD4
:10FB500008FB0C2207FB0B2CDDE95520A0FB0ABE9D
:10FB6000CDE95F2002FB0AE200FB0922B3EB0B00A8
:10FB70006CEB0202CDE95520104304BF4FF0000B9F
:10FB8000594632D0DDE95C03A0FB012C5C9103FBFC
:10FB900001C100FB0411DDE95F30A0FB05CB03FBD5
:10FBA00005B300FB0633B2EB0C0061EB0301DDE9AA
:10FBB00055320CF02DFA8346A7FB050108FB051111
:10FBC00007FB06125C99AAFB013C09FB01C10AFB79
:10FBD0000411C01A62EB01010904DDE9553241EA62
:10FBE000104100040CF014FA01465A9848431BEBEC
:10FBF000204048BF00205B9B5E9A9A4224DD549AC5
:10FC0000539B4A430BEB2242D31A44BF539B9B1A8C
:10FC1000509A93423CD2529A5143519A0BEB214154
:10FC20008A1A44BF519A521A50998A4230D258992E
:10FC3000091A44BF5899411A509A914228D26E9994
:10FC400008800120579023E0539A549B4A430BEBC2
:10FC50002242D31A44BF549B9B1A509A934217D204
:10FC6000519A5143529A0BEB21418A1A44BF529A3E
:10FC7000521A50998A420BD25999091A44BF59997C
:10FC8000411A509A914203D26499088001205790FA
:10FC9000579865B0BDE8F08F2DE9FF4F8DB09A46BB
:10FCA0008B46054603F09CFF0190007BD8B11420E1
:10FCB00002900220009095F89940022C94BF4FF0DA
:10FCC00001094FF0000995F8760001281CBFFE4895
:10FCD000806914D0039095F8ED00FC4B4FF00008BC
:10FCE000022846D115E03C200290019890F842008D
:10FCF00002282EBF03200F200090DCD3DAE7F4485F
:10FD000064220068418A408B5143B1FBF0F04043CC
:10FD1000E0E71819B9F1000F00F8018CED48204414
:10FD200000F8018C80F80980EB48204400F8018C31
:10FD300080F80980E94800EB440020F8028CA0F824
:10FD40001280E7488BF8CC80204485F8CC8000F8FE
:10FD5000018CE448204400F8018CE348204400F87A
:10FD6000018CE248204400F8018C1CBF2046FFF7BC
:10FD700038FD0F981919B9F1000F0288DC48059178
:10FD800000EB0410079011F8011C049100EB4100F6
:10FD900020F8102CBAF80010A0F8901072D0D548B6
:10FDA000D54900EB040E21441EF8010C01F8010CAA
:10FDB000D2492144069111F8011C01B3411CC9B27A
:10FDC000282927D3CE4904EB840201EB021101EB71
:10FDD000400231F850CC32F8503CACEB030CC94B2C
:10FDE00003EB840343F804CCB2F85020B1F8501070
:10FDF0008A1AC54901EB840141F8042C25E0C14968
:10FE000001EB840141F8048CBF4901EB840141F806
:10FE1000048C1AE0BA4A04EB840302EB031202EBEF
:10FE2000410131F8502C31F8523CD31AB54A02EB5B
:10FE3000840242F8043CB1F85020B1F84E10521A36
:10FE4000B14901EB840141F8042C0F9904EB8403C0
:10FE500027280A88AA4901EB031101EB400121F888
:10FE6000502CBAF80020A1F8502003D1069A0121A5
:10FE700002F8011C401CC0B20EF8010C282828BF53
:10FE80000EF8018C95F8ED00022800F089810498A5
:10FE90000799C01D4FF0000E00F007000F9ACDF833
:10FEA00018E001EB4000128830F8101CB0F8900008
:10FEB000511ABAF80020101AB9F1000F36D08F4A43
:10FEC000224412F801CC914ABCF1000F02F1080360
:10FED0004AD002EB840C00295CF8046CACBF0A46E3
:10FEE0004A42164403EB84034CF8046C53F8047C38
:10FEF0000028B4BF424202463A4443F8042C174655
:10FF0000804A02EB840252F8042C002AB8BF524205
:10FF1000B21A4CF8042C7C4A02EB840252F8042CEE
:10FF2000002AB8BF5242BA1A43F8042C684A126831
:10FF3000138B5943138A91FBF3F6518B4843518A33
:10FF4000B9F1000F90FBF1F704D06C48204410F891
:10FF5000010C08B3002E3DDD60484FF0020100EBBC
:10FF6000440020F8028C4DE002EB8402002952F894
:10FF7000046CB4BFC1F1000C8C46B44442F804CC0C
:10FF800003EB8402002852F804CCB4BF434203467A
:10FF9000634442F8043CC9E75D48002E00EB44008E
:10FFA00030F8022CB4BF714231468A4205DA002E85
:10FFB000ACBF3146714220F8021C4288002FB4BF0A
:10FFC000794239468A42C5DA002FACBF39467942B8
:10FFD0004180BFE706DA4148012100EB440020F8E8
:10FFE000028C0FE03C48204410F8011C3B4800EB19
:10FFF000440030F8022C642A04D2521C20F8022C4F
:020000021000EC
:100000004FF0010E002F07DD344A4FF0040002EBE1
:100010004402A2F8128015E007DA304A4FF00300DC
:1000200002EB4402A2F812800CE02C4A2A4802EBB0
:1000300044022044538A407A642B03D25B1C5382CF
:1000400001220692244A224412F8013C13B38B4247
:1000500021D1224B03EB440333F802CC029B9C4595
:100060001C4B234496BF13F801CC03F8018CBCF160
:10007000640F51D2BEF1000F4ED10CF1010C0CF007
:10008000FF0C03F801CCBCF10A0F45D3144B2344F9
:1000900003F8018C40E00F4B234413F801CCBCF172
:1000A000050FDFF83CC0A44436BF1CF801EC0CF887
:1000B000018CBEF1640F05D20A2EA4BF0EF1010E11
:1000C0000CF801EC26E0000044820010C40A011084
:1000D000EC820010E20A0110CE0A0110F60A0110AB
:1000E0001E0B0110280B0110320B01102E05011000
:1000F00084090110488200104A8200104C820010CE
:10010000EE030110688200107082001080820010DF
:100110007882001003F8018C537A23B3834223D1F1
:10012000FD4B03EB4403B3F812C0029B9C45FB4B11
:10013000234496BF93F809C083F80980BCF1640F8B
:100140002BD2DDF818E0BEF1000F26D10CF1010C26
:100150000CF0FF0C83F809C0BCF10A0F1DD3F04B63
:10016000234403F8018C18E0EC4B234493F809C0B6
:10017000BCF1050FDFF8A8C3A44436BF1CF801EC9E
:100180000CF8018CBEF1640F05D20A2FA4BF0EF14A
:10019000010E0CF801EC83F8098002F8011C507282
:1001A00004980599401CC0B201F8010C08280AD334
:1001B000059800F8018C9BF8CC00002804BF0120B2
:1001C0008BF8CC0006E09BF8CC00002808BF85F82F
:1001D000CC8037D00AAB08AAD2492046FFF7D0FA24
:1001E00083460BAB09AAD0492046FFF7C9FA039909
:1001F0008B4598BF88420CD9032085F8CC00CB48AA
:100200000121204400F8018CC948204400F8011C59
:1002100014E0C248204410F8011C08299CBF407A11
:1002200008282AD9032085F8CC00C048C0492044BA
:10023000214400F8018C012001F8010C95F8CC0054
:10024000032807D0BB48204400F8018CB448204460
:1002500000F8018CB84802212044029000F8011CEB
:10026000B648B9F1000F00EB040B0BF8011C26D0C7
:1002700095F8CC0003281CD01EE0AC48204410F8B0
:10028000011CC8293CBF491C00F8011CA849214495
:1002900011F8011C012908D110F8011C00988142B5
:1002A0009CBF032085F8CC00D4D9022085F8CC006F
:1002B000C8E703F0D5FC88B12046FFF792FA95F81D
:1002C000CC0003281EBF042811B0BDE8F08F012028
:1002D000019981F8200511B0BDE8F08F98482044BD
:1002E00010F8010C012808D00028E8D195482044D6
:1002F00010F8010C401C0728E1D3282ED8BF282F66
:1003000009DC914800EB440030F8021C28299CBF0E
:10031000408828280AD90198007B0028CFD002996C
:10032000032001F8010C0BF8010CC8E78548CDF853
:1003300000A02044854910F8012C20460F9BFFF7B0
:1003400078FA012805D0029800F8018C0BF8018C8E
:10035000B5E70299012001F8010C0BF8010CAEE79A
:10036000B0F8B030B1F8B0C0B3EB0C0248BFACEBA2
:100370000302B0F8B230B1F8B210581A48BFC81A28
:1003800002FB02F100FB0010704770B50D460446F9
:1003900003F026FC94F8ED006D4E02281DBF94F882
:1003A000BB000128012DB4F8B4000FBFB4F8B6208B
:1003B00094F8990006EBC00151E90202322131257F
:1003C000B4F8B4C0B4F8B63005FB00C0B0FBF1F02F
:1003D00005FB0232B2FBF1F194F8992006EBC20260
:1003E00042F8080C94F8992006EBC20242F8041C6B
:1003F000A4F8B400A4F8B61070BD2DE9F007554C70
:10040000DDE9078C24681F8890F8ED30658A648BDD
:10041000C5EB0515AD00B5FBF4F90E881588B8F8E5
:100420000040032B3BD190F89930DFF82CA10AEB68
:10043000430333F8028CB8F1050F30D2B8F1000F46
:100440001AD0A1F800C02B1B1480002BB8BF5B4250
:100450004B459CBFBDE8F007704767451CBFBDE832
:10046000F0077047052190F899000AEB400020F84A
:10047000021CBDE8F00770474FF0010823F8028C1A
:100480002B1B1C04A6EB070894FBF8F47443A5EBA4
:100490002445A1F800C005EB24411180D5E7A1F85F
:1004A00000C0BDE8F00770472DE9F04786B00C4664
:1004B000074603F0B1FB804600F0BEFA064600F0A6
:1004C000BEFADFF890A0054694F89A00DAF800101A
:1004D000C0EB001008EB0010B1F81280B1F81090DA
:1004E0003988ADF808107988ADF80C10B0F8B41060
:1004F000ADF81010B0F8B600ADF8140000F033FB02
:1005000060B3BDF80800B04238BF3046ADF808000F
:10051000BDF80C10A94222E0F60A0110E20A01100F
:10052000280B011084090110240A0110320B01105C
:100530002E0501101E0B0110DA030110E403011057
:100540004C8200104A82001078820010EE030110E5
:100550003C0B0110EC8200108C0B01101CE038BF2A
:100560002946ADF80C10A9EB0602531E8342B8BF12
:100570001846ADF80800A8EB0500421E8A42B8BF35
:100580001146ADF80C10BDF80800B880BDF80C009D
:10059000F88006B0BDE8F08794F8ED0002281CBF93
:1005A00094F8BB0001281ED16078FE4A60B1DAF8E9
:1005B00000108B795B1E98421CBF2078002803D066
:1005C000C979491E884207D194F89910052002EB99
:1005D000410121F8020C06E094F89910002002EB8A
:1005E000410121F8020CBDF80800B04208D205A86C
:1005F000CDE9000604AB03AA02A92046FFF7FDFEE1
:10060000BDF80C00A84208D204A8CDE9000505AB4E
:1006100002AA03A92046FFF7F0FEA9EB0600BDF8E9
:100620000810401E884209DA80B205A9CDE9001001
:1006300004AB03AA02A92046FFF7DFFEA8EB0500E2
:10064000BDF80C10401E88429DDA80B204A9CDE9A5
:10065000001005AB02AA03A92046FFF7CEFE92E7E1
:1006600030B490F8ED20052490F89010DFF838C3EE
:1006700090F89930022A1BBF90F8BB20012A0A4645
:1006800013F80C20042505FB021191FBF4F103F88B
:100690000C1080F8901030BC70472DE9F04F87B0F7
:1006A000044600F0C9F9824600F0C9F9814603F01A
:1006B000B3FA059003F094FA0746007B94F899800A
:1006C000DFF8E8B200281CBF387D0128DBF80010F5
:1006D0007ED0086FC0F3C0420192C0F34042C0F325
:1006E000804004920090486FC0F303410E02B0496D
:1006F000414411F8011C02290EBF4FF44075C0F3AC
:10070000035005020220FEF715F9A848006890F88A
:10071000700010F0010F00F07F8194F89A00B4F897
:10072000B010ADF80810B4F8B210ADF80A10C0EB74
:100730000011059802AA00EB011B59462046FEF75E
:10074000DBFF019838B1BDF80C00ADF80800BDF82A
:100750000E00ADF80A0094F8ED00022819BF94F8D5
:10076000BB0001284046FEF75DFCBDF808200021D3
:100770002046FEF74DFE0190BDF80A2001212046DB
:10078000FEF746FE01990029B8BF00210028B8BF36
:100790000020DFF818C2DCF80030B3F91020A2F115
:1007A000010E8E45B8BF7146B3F91220531E834225
:1007B000B8BF184689B283B27E48ADF80C1000EB82
:1007C0000802ADF80E300A3012F801CC404400E0C7
:1007D00028E010F801EC02F801EC00F801CC0098D8
:1007E00000281CBFADF80810ADF80A300DF10E035B
:1007F00003AA59462046FFF74FFAB4F8B020BBF8D9
:10080000B000111A48BF811AB4F8B230BBF8B22058
:10081000981A48BFD01A494300FB0013387B0028C0
:100820003ED053E091F87000C0F3C0020192C0F3D3
:100830004002C0F3800004920090387D01281BD054
:1008400003F00EFA38B103F008FA01281BD003F0C8
:1008500004FA082817D003F0A8FA002818BF03F0FC
:1008600067FADBF8000090F8740001070E0DC0F382
:1008700003100502002046E7B1F87400C0F303201E
:1008800006023546F6E7DBF80000B0F87400010711
:100890000E0DC0F30320000200F58075012032E741
:1008A0004548404410F8010C012807D070B943486E
:1008B000404410F8010C401C282807D9BDF80C0052
:1008C000ADF80800BDF80E00ADF80A00CDE90065EE
:1008D00097F8422002A92046FEF7C2F8049868B1B2
:1008E000BDF80C00ADF80800BDF80E10ADF80A1008
:1008F000A4F8B400BDF80E00A4F8B60003F0B0F9F7
:10090000012804BF94F8E500012807D1B4F8B0002D
:10091000A4F8B400B4F8B200A4F8B600234D2868D7
:1009200090F8700010F0200F0FD097F842100129B6
:100930006ED023484FF0FF3101804180080C2149DF
:1009400008804880002020390870B4F8B400ADF861
:100950000800B4F8B600ADF80A00214602A8FFF777
:10096000A3FDBDF80C00ADF80800BDF80E10ADF801
:100970000A1094F8ED2005230B49022A1BBF94F8B6
:10098000BB20012A94F8902094F8992018BF525C5B
:1009900094F890C0042606FB02C292FBF3F294F88E
:1009A000993011E08C0B01109F0B0110EC820010AC
:1009B000DA030110F80801104C8200104A8200107E
:1009C00060820010648200105A5484F89020BDF8B0
:1009D0000A105045B8BF50464945B8BF49462B6834
:1009E000B3F91020A2EB0A02A2F1010C8445B8BFB2
:1009F0006046B3F91220A2EB0902531E8B42B8BF26
:100A00001946A4F8B400A4F8B61007B0BDE8F08FFA
:100A10002046FEF7E0FB98E7B4F8B000A4F8B40075
:100A2000B4F8B200A4F8B60007B0BDE8F08F00003B
:100A3000FE487047FE487047FE4800787047FD4802
:100A400040787047FB48142181801221C180704793
:100A50000346002002460029D8BF704753F822C041
:100A6000521C60449142F9DC70472DE9F05F0E465C
:100A7000054603F0E1F8044603F0DAF8310291FB91
:100A8000F0FC290291FBF4F3DFF8A8A30021DFF8C2
:100A9000A893BAF80480BAF806704FEA6C264FEAB9
:100AA000632B002CC8BFE24D0BDD01FB03F20BEB07
:100AB000222245F8212049F82120491C09B28C4204
:100AC000F3DC0021DFF874B30028C8BFD74D0BDD7D
:100AD00001FB0CF206EB222245F821204BF82120E5
:100AE000491C09B28842F3DC0CFB08FC4FEA6C316C
:100AF0007B43CAF808105A139AF802504FEA6C3C2C
:100B00005B13CDB1D9F800300BEB80009B1AC9F80C
:100B1000003009EB840353F804CC624443F8042CFE
:100B2000DBF80020521ACBF8002050F8042C1144B6
:100B300040F8041CBDE8F09FD9F800500BEB800092
:100B4000AA1AC9F8002009EB840252F8044C234485
:100B500042F8043CDBF80020511ACBF8001050F8A2
:100B6000041C6144E4E7B3488078012818BF0020E2
:100B700070472DE9F047DFF8C89204461226D9F8ED
:100B80000000AC4D478AB0F810801420142C03D21A
:100B9000A4F10F01052902D2A880EE801BE0A4F188
:100BA0000A0105293CBFA880E88014D3611F0529EC
:100BB00003D21620A880E8800DE0052C28BFA8806D
:100BC00008D203F04DF800281DBF1820A880E88047
:100BD000AE8000D1EE800021002C06BF0120A8705D
:100BE000A970D9F80000428A408B6243B2FBF0F052
:100BF0002870697041463846BDE8F04735E710B5C2
:100C0000012907BF8F4C14218F4C1221142803D2C5
:100C1000A0F10F02052A01D2218010BDA0F10A0225
:100C2000052A38BF14200CD3421F052A38BF1620CE
:100C300007D30528F0D203F013F8002814BF1820BA
:100C40001220208010BD7E497A4A0128096807D009
:100C5000488B5278498A5043B0FBF1F0C0B27047DC
:100C6000088B1278098A5043B0FBF1F0C0B270478C
:100C7000734810B502684FF0140C92F86C30508A2B
:100C8000118ADB08528B4343B3FBF2F3694A1370BA
:100C900000235370A2F804C04FF0120CA2F806C053
:100CA0009370FFF7E2FE694900204FF6FF7221F8CA
:100CB000202001EB8003401C80B25A800A28F6D322
:100CC00010BD2DE9FF4FADF5037D1C46164698215A
:100CD00068460BF08EF950214CA80BF08AF9982148
:100CE00026A80BF086F9502160A80BF082F902F0DB
:100CF00093FF814602F074FF074602F083FF78906D
:100D0000503081900A20809002F092FF054602F058
:100D100093FF80464A480068418A7591008A769020
:100D2000607800281BBFA8F1010188424248404872
:100D30007790207800281BBF691E88423F483B48B7
:100D4000749002F08DFFDFF8ECA0012810D102F0C2
:100D500084FF01280CD11820AAF80400DDE97501F0
:100D6000FFF783FE3548DAF80820C16B1144C163F0
:100D70009AF802007F90012803D12F487790983885
:100D8000749094F8EBC0DFF8C8A0BCF1000F0FD14D
:100D9000E088401DAAFB0010C00800FB05F1A088F8
:100DA000401DAAFB002006EBD000085C00F03F0CC1
:100DB00094F89A0094F899202449C0EB001001EBB4
:100DC000820309EB001033F8049CA9F57F41FF3939
:100DD0001DBF33F8022CA2F57F41B1F1FF018188DC
:100DE0000CBFC2884946B4F804B0CDF8E8B10BF1A5
:100DF000050BAAFB0BEBCBF3CF0BCDF8F8B1B4F896
:100E000006B0CDF8E4B10BF1050BAAFB0BEBCBF36D
:100E1000CF0BCDF808B201F1050BAAFB0BEBCBF31E
:100E2000CF0E02F1050BAAFB0BBA13E0AC0B0110BD
:100E3000440C0110B08200102C0D0110940C011014
:100E4000EC820010B4820010B68200107C0D0110FC
:100E5000CDCCCCCCCDF8ECE1DDF8E8B14CF6CD4E04
:100E60000BFB0EFB4FEADB4BCDF8F0B1DDF8E4B144
:100E7000CAF3CF0A0BFB0EFB4FEADB4BCDF8F4B104
:100E800001FB0EFB4FEADB4BCDF8E8B102FB0EFB9A
:100E90004FEADB4BCDF8E4B1DDF8ECE1DDF8F8B179
:100EA000F34504BFDDF808B2D3450BD0DDF8E8B157
:100EB000DDF8F0A1DA4515D1DDF8F4B1DDF8E4A1F3
:100EC000D3450FD197F842A0BAF1020F0AD3DDF84B
:100ED000E0B19BF842B0D34504BF94F898A0BAF1B2
:100EE000020F4CD04FF6FF7023F8040CF94994F828
:100EF000992001EB820121F8020C207B7990607B24
:100F00007890A27B94F80F907898EB4648452AD8C1
:100F100000FB05F189B27A91799991421FD87A9BA9
:100F200003EB010A839B33F91A3016F80AA00AF082
:100F30003F0AE2450FD1DDF800A253450BDB5BF819
:100F400021A09A444BF821A00DF5987A5AF820E098
:100F500073444AF82030491C89B29142DFD9401CC1
:100F600080B24845D4D9387B00287DD097F82F052A
:100F7000002804BF97F83304012852D08CE0DFF832
:100F800054A34FF6FF7BD94504BF33F8029CD945E3
:100F900007D123F8041C94F899100AEB810121F879
:100FA000022C017B227B914238BF2173417B627B03
:100FB000914238BF6173817BA27B914288BFA1734C
:100FC000C17BE27B914288BFE173217B799194F8E8
:100FD0000DA0CDF8E0A194F80F90A27B90F8EBB0B3
:100FE000CA4591D80AFB05F080B27A907998904270
:100FF00010D87A99819B01445B5C03F03F0EDE457B
:1010000004D123F03F0343EA0C037354401C80B225
:101010009042EED90AF101001FFA80FACA45E1D9DF
:1010200072E794F8E860012E07D835D197F84C1391
:10103000849830F911001E282EDD50214CA80AF0AA
:10104000D8FF07EB460197F8422091F8E20391F8A8
:10105000E313012A13D10A1A521C0A2A0FDD07EBE7
:10106000860292F8483300E016E0DA1EDB1C82426A
:10107000C8BF1046C0B29942C8BF1946C9B288421B
:1010800098BF4CAA08D8849B33F9103042F820301E
:10109000401C80B28842F6D900216A460846002DDD
:1010A00040F3F58052F82030401C1944A842F9DB87
:1010B000002940F3EC8000214CAA0846B8F1000F4B
:1010C0007BDD52F82030401C19448045F9DC0029B2
:1010D00073DD002026AE002D88BF59460BD9749AC7
:1010E00051F8203052F820205A4346F82020401C66
:1010F00080B28542F3D80020B8F1000F84BF4CA91C
:1011000060AB0CD9779A51F820C052F820200CFB24
:1011100002F243F82020401C80B28045F2D8002122
:1011200032460846002D05DD52F82030401C194497
:101130008542F9DC00226B461046002D05DD53F890
:1011400020C0401C62448542F9DC91FBF2F094F827
:101150007610012904BF7F9900296AD1DFF878C190
:10116000F0280CEB8503DCF8007053F8044CBCBF8E
:101170008020CCF800002EDBA0F1F001DC2938BF84
:10118000C02007D3A0F5E671B1F5967F38BF4FF4C4
:10119000807002D2CCF800001DE0A0F5B8413039D3
:1011A000B1F52F7F3CBF45F6E06043F8040C12D345
:1011B000A0F5BC41EC39642900E068E038BF45F691
:1011C000407006D345F650718842A8BF4FF4BF4027
:1011D00001DB43F8040C0020002D88BF59460CD9D0
:1011E000749A51F8209052F8202009FB02F246F838
:1011F0002020401C80B28542F2D8002132460846A9
:10120000002D05DD52F82060401C31448542F9DC98
:1012100000226E461046002D05DD56F82090401C39
:101220004A448542F9DC91FBF2F0CCF8007043F8B7
:10123000044C002260AB1146B8F1000F05DD53F8F5
:1012400021C0491C62448845F9DC00230DF5987CD7
:101250001946B8F1000F05DD5CF82140491C234414
:101260008845F9DC92FBF3F10028B8BF0020002983
:10127000B8BF0021769A521E9042C4BF7698401E95
:10128000759A521E9142C4BF7599491E01E0002013
:101290000146909A1080919801800DF5077DBDE878
:1012A000F08F2DE9F84F1D4616460C46834602F096
:1012B000B3FC014694F89A000022C0EB001001EB49
:1012C00000130648BBF1010F0AD0BBF1080F28D06C
:1012D0004AE000007C0D0110940C0110EC8200101B
:1012E00000686E2140F2D34AB0F812C0078B0CFBA5
:1012F00001F8418B008AB2FBF7F900FB0AF0B0FB62
:10130000F7F0B8FBF1F840F231570CFB07FCBCFBDF
:10131000F1F11FFA80FA80B21FFA88F88FB20090BC
:1013200022E001684FF448700F8AB1F818C0784382
:10133000B0FBFCF01FFA80F9488A07EB8717C0EB77
:1013400040187F0108EB8018498BB7FBFCFC1FFAA3
:101350008CFA40F2415C00FB0CF0B8FBF1F8B0FBFA
:10136000F1F01FFA88F887B2A4F8B060A4F8B25080
:101370004E4538BFA4F8B09003D3B24538BFA4F8A7
:10138000B0A0454538BFA4F8B28003D3AF4238BF00
:10139000A4F8B2700120BBF1080F15D0BBF1010F0A
:1013A00018BFBDE8F88F4E4522BF0099B1424545B0
:1013B00003D3BD4298BFBDE8F88F94F8ED10022921
:1013C00018BFBDE8F88F1CE04E4528BFB24504D3D6
:1013D000454524BFAF42BDE8F88F94F8ED100229CF
:1013E0000FD084F8E50093F8E510012918BFBDE897
:1013F000F88F84F8E40084F8E02084F8ED20BDE85C
:10140000F88F84F8E40084F8E02084F8ED2084F874
:10141000E520BDE8F88F2DE9F04385B01C4616465F
:101420000F46804602F0DCFB02F0ECFB02F0F4FB1E
:1014300094F89A10C1EB011100EB011502F0FCFBCE
:10144000814602A903A8CDE9000123463246394668
:101450004046FFF736FCBDF80C00A4F8B000BDF81C
:101460000800A4F8B20002F0F8FB012803D002F053
:10147000F4FB08280BD102F0F3FB40B102F0EDFBC6
:10148000BDF80830BDF80C202146FFF70AFF95F89B
:10149000BB00032807BF2878002805B0BDE8F0830B
:1014A000687800281CBFA9F101018842A4BF05B0DB
:1014B000BDE8F08394F8BB0001281CBF05B0BDE86F
:1014C000F083B5F8B000A4F8B000B5F8B200A4F805
:1014D000B20005B0BDE8F0839DE700002DE9F041C2
:1014E00014460D46074602F07BFB02F0A1FB0646C0
:1014F00002F0A2FBD5E9071380462869002510B346
:1015000001EB810189004000B1FBF0F203EB8301A4
:101510008900B1FBF0F1FE48A0FB02C34FEAD30CF7
:10152000A0FB0130C308701E84459CBFA8F10100D8
:10153000834208D803FB06C02280618037F8100080
:10154000A080BDE8F08125806580A580BDE8F081A0
:101550002DE9F0410446DDE90606089F0D46002806
:101560001CBF002081F8290002D00020BDE8F081D6
:10157000286820606868E060106851686060A16059
:101580008422194604F114000AF02EFDA868206197
:101590002869A061A889A082A88CA4F8700095F899
:1015A000280084F8E10095F82A0084F8E200012080
:1015B00084F8E00095F82B0084F8E70084F8E370E5
:1015C00095F82C0084F8E80095F82D0084F8E900DF
:1015D00095F82E0084F8EA0095F82F0084F8EB00C7
:1015E0003078401CC0B230700A2828BF0120BCD31C
:1015F000BDE8F0810028DCBF002070474FF4807107
:101600004FEA002C00200B129CFBF3F30A469918BA
:1016100001EBD1714910531A48BF8B1A802B02DBA2
:10162000401C6428EFD3081270472DE9FF4F85B0A6
:101630001F4616460D46002402F0FAFA0190B6F94C
:1016400000E0B6F902000290287903906A79E879FF
:1016500095F806A0A446654666460090824229DCBD
:101660000398504521DC029902EB8203C1EB43034E
:1016700003FB03FB019902FB0108059931F91810DE
:101680000A290EDD00EB8008CEEB480808FB08F9BC
:1016900003FB08F809FB01CC0BFB015508FB0166B5
:1016A0000C44401C00B25045E4DD501C02B20098CE
:1016B0008242D5DDDFF85C8288FB0C104111A1EB82
:1016C000E07188FB05204211A2EBE07288FB063036
:1016D0004311A3EBE0734CB1080211021A0290FB14
:1016E000F4F091FBF4F192FBF4F202E000200146E9
:1016F000024600FB01F302FB12320844C0F1000C69
:101700001412A0000CFB0CF1C0EB212000124100D0
:101710000029D8BF002014DD0D024FF48070002195
:10172000031295FBF3F30246981800EBD0704010BB
:10173000131A48BF831A802B02DB491C6429EFD39C
:101740000012000200EBD070DCEB60010CEB6000DB
:10175000C0F100027C6148BF4942F960002AB8BF6D
:10176000524201EB8100400088FB0030C310A3EB24
:10177000E0703A61FF28C8BFFF2049115211FF29CC
:1017800088BFFF21FF2A88BFFF22002912BF002A3D
:1017900001210A46002808BF012087F87C0087F84D
:1017A0007D1087F87E2009B0BDE8F08F70B5044643
:1017B00002F03EFA054602F03FFA2178024600297F
:1017C0001CBF681E814206D0607800281FBF511ED2
:1017D0008842002070BD012070BD2DE9F05F9A465F
:1017E00090460E46054602F0FBF9044602F00AFA5E
:1017F00083464FF0000902F01BFA074694F84A03AB
:101800000023012842D1207B00283FD0D4F82805AE
:10181000DBF82815404A884206D2D2F800C0C943F6
:1018200061440844106003E0401A116808441060E5
:1018300094F82605012808D094F8300400281CBF2D
:1018400094F8180500281DD10AE094F83004002807
:101850001ABF94F8180500284FF0010912D1EBE7E0
:10186000BAF1030F24BF207D00280BD194F8240582
:1018700094F82215401A072804DB012084F8260575
:10188000136056E01068B0F5616F02D984F8263510
:1018900002E0B9F1000F4CD102F087FA18B102F062
:1018A00047FA082803D102F04FFA02282BD17379A6
:1018B00096F807B04FF000099B453AD3B07996F8F7
:1018C00004A0441E5046844216DB03FB070235F990
:1018D000121005EB4202B2F90220B1EB020C48BF34
:1018E000A2EB010CBCF1230F02DD4FF0010903E074
:1018F000401C80B28442E8DA581C83B29B45E1D296
:10190000B9F1000F15D0B6F902005A2814DA05E033
:10191000CDCCCCCC1F85EB51BC820010B0898C287B
:101920009CBF98F87D00FA283CBF98F87E00FA2802
:1019300002D30120BDE8F09F0020BDE8F09F2DE913
:10194000FF4F89B017460C46FE48D0E90012CDE99A
:101950000212D0E90210CDE904100020009001909D
:1019600002F03EF95030069002F062F9804602F033
:1019700063F9B4F902100791237861784FF00009F8
:101980004A465C1EA1F1010C4D46A8F1010EA0F1E2
:10199000010BEA4602A925F00100095A21440CB2C4
:1019A00004A9002C085A60440FFA80FCA8BFA64581
:1019B00034DBBCF1000FA8BFE3452FDB0CFB084074
:1019C000069900B2095C49B3099931F91060002EFB
:1019D000D8BF01261698032120F8126006EB0900F3
:1019E0000FFA80F903E0481E10F0FF0105D00AEB62
:1019F000410030F9020C8642F5DC0223022909D2AB
:101A00000AEB430030F8020C2AF81300581EC3B248
:101A10009942F5D3501C2AF81160C2B2681CC5B2B5
:101A2000082DB7D3BDF80000BDF80210BDF8043092
:101A300001441944A7F87A100C990A7007990844D0
:101A4000A7F84A00A7F878900DB0BDE8F08F2DE90F
:101A5000F04186B014460D468046002702F0C0F8DB
:101A600002A8009001AB224629464046FFF767FFD7
:101A7000002084F85A7084F85F00687840B102F062
:101A8000DBF86978401E88421CBF06B0BDE8F081D3
:101A9000012084F8760006B0BDE8F0812DE9F04120
:101AA00017460E4602F09CF8044602F0ABF8217D82
:101AB000002599B9B1891E2981BF97F87D104B295E
:101AC000F18C072906D897F87D10642984BFF18C22
:101AD000062903D9217B0125022907D002F06AF9E2
:101AE000002808BF00252846BDE8F08194F82E158F
:101AF000012919BF90F84200002800202073EDE76B
:101B00002DE9F74FAEB0804602F072F82A9002F04D
:101B100067F80027259030988DF890703E463D4636
:101B20000028C8BF4FF0010940F337812F9805EB1B
:101B3000450100EB011494F82900012840F02781A9
:101B4000842101A80AF055FA01A822974FF0000B52
:101B500023972B9002F044F826A800902CAB214646
:101B600040462B9AFFF7EBFE00208DF85EB08DF813
:101B70006300607828B102F05FF8411E607881420E
:101B800001D18DF87A9002F02BF802F051F88246DC
:101B900002F052F88346D4E90712206920B301EB22
:101BA000810189004000B1FBF0F102EB820292005A
:101BB000B2FBF0F0644AA2FB01C3A2FB00C2DB0847
:101BC000D208AAF1010C63459CBFABF1010C624540
:101BD0000AD8ADF8881002FB0A31ADF88A0038F84F
:101BE0001100ADF88C0005E0ADF88870ADF88A7092
:101BF000ADF88C7001AB22AA21464046FFF715FDD7
:101C000001F0EEFF824601F0FDFF01469AF8140054
